:1010000000000420B5120000DD120000DF12000015
:10101000E1120000E3120000E512000000000000F1
:10102000000000000000000000000000E7120000C7
:10103000E912000000000000EB120000ED120000B9
:10104000558A0000E9C70300658A0000EF1200001E
:10105000EF120000EF12000071870000EF12000095
:10106000EF120000EF120000EF120000EF1200007C
:10107000EF120000018B0000EF120000EF120000E1
:10108000EF12000081500000EF120000EF1200008C
:10109000EF120000EF120000EF120000EF1200004C
:1010A000EF120000EF120000518D0000EF1200005F
:1010B000EF120000EF12000000000000000000002E
:1010C000EF120000EF120000EF120000EF1200001C
:1010D00015F60300EF120000EF1200000D9D000056
:1010E000EF120000EF120000EF12000000000000FD
:1010F00000000000EF12000000000000EF120000EE
:1011000000000000000000000000000000000000DF
:1011100000000000000000000000000000000000CF
:1011200000000000000000000000000000000000BF
:1011300000000000000000000000000000000000AF
:10114000000000000000000000000000000000009F
:10115000000000000000000000000000000000008F
:10116000000000000000000000000000000000007F
:10117000000000000000000000000000000000006F
:10118000000000000000000000000000000000005F
:10119000000000000000000000000000000000004F
:1011A000000000000000000000000000000000003F
:1011B000000000000000000000000000000000002F
:1011C000000000000000000000000000000000001F
:1011D000000000000000000000000000000000000F
:1011E00000000000000000000000000000000000FF
:1011F00000000000000000000000000000000000EF
:1012000010B5054C237833B9044B13B10448AFF340
:1012100000800123237010BD200600200000000084
:101220003C7D040008B5034B1BB103490348AFF3F1
:10123000008008BD00000000240600203C7D040062
:10124000154B002B08BF134B9D46A3F5803A002198
:101250008B460F461348144A121A3EF06EFD0F4B90
:10126000002B00D098470E4B002B00D09847002051
:10127000002104000D000D48002802D00C48AFF3F7
:1012800000803EF0DFFC2000290009F043F83EF02A
:10129000B3FC00BF000008000000042000000000B4
:1012A000000000002006002060A9002000000000CF
:1012B000000000000649074A074B9B1A03DD043B68
:1012C000C858D050FBDC09F08DF8FFF7B9FF0000DB
:1012D0006C7F04000800002020060020FEE7FEE7E7
:1012E000FEE7FEE7FEE7FEE7FEE7FEE7FEE7FEE7D6
:1012F0007047000007B5044B0093044A802300F0B8
:1013000032F803B05DF804FB111300003D06002025
:101310002DE9F84389461446B2B10F4B0F4E032511
:10132000002743F00108224609EB0701002008F0DE
:101330004BFF0744241A48B933782BB14FF47A4055
:10134000C047013D02D13570BDE8F88301233370F9
:10135000002CE8D1F8E700BF802104003C06002003
:10136000704708F065BFF0B595B008460D461646C3
:101370001C4606F0C3FC1A9A0D920023082205A908
:1013800028460A938DF82C300C93CDE9086406F0BA
:10139000D3FC079B0293BDF81830ADF80C30BDF8B4
:1013A0001A30ADF80E3001238DF811309DF814304D
:1013B00003F00302012A1DD1BDF81440059EC3F3BA
:1013C000C203C4F383148DF81030A20008230EA9C1
:1013D000284606F0B1FCC6F3952608AB00932246DA
:1013E00002AB0EA9304600F045FF284606F08AFC05
:1013F00015B0F0BD022AF8D1BDF81640C3F3C20300
:10140000A4098DF810300827082C264628BF082686
:101410003B4632460EA9284606F08EFCA41B08ABBC
:1014200002AA31460EA8374400F088FF002CEBD109
:10143000DBE7000008B5FFF794FF0421034800F044
:1014400077FE034B01225A7108BD00BF407D0400A6
:101450000800002000230428CB604B6098BF044B99
:10146000044A98BF53F820308A600B60704700BF71
:101470006823040044230400CB6800225A7170479B
:10148000C368DB6800225A717047CB6801225A7129
:101490007047C368DB6801225A717047104A8A603E
:1014A000F0B5104A104C0023121BCB604B600B6050
:1014B00022F00F021D46264693420DD006EB030C88
:1014C000E718DCF80CC09CF804C0BCF1FF0F05D095
:1014D000854202D1BB680B60F0BD01351033EBE7EC
:1014E0007C230400607D0400407D04002DE9F74F5B
:1014F000174E184D0093AD1B52F8043C07468A4620
:10150000904625F00F050024B146A54207D1124AA6
:101510000221384603B0BDE8F04F04F049BC09EBA6
:1015200004011846896801933FF03EF906EB040B6D
:10153000019B10340028E8D1DDED007A17EE90CA47
:10154000434652465946384603B0BDE8F04F60471F
:10155000407D0400607D0400B4240400014BFFF7CB
:10156000C5BF00BF751B0000014BFFF7BFBF00BF29
:1015700079140000014BFFF7B9BF00BF8B140000C6
:10158000014BFFF7B3BF00BFAD190000037813F0A4
:10159000040216D003F00303012B03D0022B09D061
:1015A000012070470A6800880232C0F383100244A9
:1015B0000A60F5E70B684288023303EB92130B6075
:1015C000EEE71046704700002DE9F04F484C87B019
:1015D0000F460546861C0020019203F003FC236899
:1015E0003B60D4E901231344226801339B1A04F2BF
:1015F0001C4704F5836A04F21448B34219D3019AD4
:101600000023002A6CD0012262F3010343F004039B
:1016100065F389132168A2680A4003320E44002052
:1016200044F82230266003F0DFFB012007B0BDE85C
:10163000F08F0121384603F02BFF504603F041FFA5
:10164000404603F03EFF0DF118096068D4F808B079
:1016500049F8100D00EA0B00033004EB8000494606
:10166000FFF794FF029BB0B90BEA030204EB82027E
:10167000D16803919A1C013303EA0B0B04EB8B0C2A
:1016800001F00303012B0292DCF80CB020D0022BF6
:1016900004D083460BE00BEA0300DDE7BDF80E3013
:1016A0009B0903334FEA1B4B02EB93030293404623
:1016B00003F00AFF08B1029B63605946384603F005
:1016C000E7FED4E901231344226801339B1A94E70F
:1016D000BDF80C30C3F383134FEA1B4B1344E5E70B
:1016E000022262F3010343F0040365F39F5391E781
:1016F00058080020012907B5034604D08168D1F8B5
:101700005413890707D500221146184603B05DF827
:1017100004EB05F007BD53680193054B0093136874
:10172000044A022104F044FB03B05DF804FB00BF4F
:10173000AE210400A42104002DE9F3478368D3F807
:101740005443C4F34004074634B10022114602B0AA
:10175000BDE8F04705F0E6BC144D154EDFF85880A3
:10176000DFF85890DFF858A0761B26F00F06B44239
:1017700002D102B0BDE8F0872B19DA689B681179B5
:10178000FF2906D10B4A0821384604F011FB10341A
:10179000EDE75279002A0CBF42464A46CDE90021C6
:1017A00038465246082104F003FBF0E7407D040070
:1017B000607D0400C3210400464D0400EF4C04008A
:1017C000E221040030B50A4B0A4A0B49D21AD2086A
:1017D00000239A4201D1052006E031F82350046825
:1017E000A54202D10360002030BD0133F1E700BF04
:1017F0000C7E04002C7F0400EC0400208368D3F8E6
:1018000054339B0703D50022114605F08BBC024AD6
:10181000022104F0CDBA00BF032204008368D3F88C
:1018200054339B0703D50022114605F07BBC024AC6
:10183000022104F0BDBA00BF032204002DE9F84FD5
:10184000224B2348FF229A600022C3F81824C3E9E0
:101850000022C3F8142483F8202406F008FA8046F6
:1018600088B91C481C4E1D4DDFF874A006F07DFCA5
:10187000AD1BED084446AC4208D100231849194875
:101880001A469C421BD14046BDE8F88F4FF0000934
:101890004F4606EBC40BBC420AD0142256F8371050
:1018A000DBF800003EF09AFF0028C8BF09F10109EB
:1018B0000137BD42EFD12AF824900134DBE701EB78
:1018C000830540F823206A800133DAE758080020B6
:1018D0002C7F0400382304000C7E04002C7F0400BD
:1018E000EC0400207C05002007B5019031B9019A75
:1018F000064B53F8320003B05DF804FB01A8FFF774
:1019000061FF0028F3D00020F5E700BF0C7E040043
:10191000002310B5CB604B60034B8B600C4601215C
:10192000FFF7E2FF206010BD44230400094B01399A
:1019300003EBC000032909D8DFE801F00A0204061E
:101940000420704700797047407970470020704745
:10195000022070470C7E040030B5124C00EB4000B2
:1019600054F821508240072303FA00F06A400240F5
:101970000D4B6A40C2F3821044F8212003EB810131
:10198000C2F3C203834238BF0346C2F342208342FC
:1019900002F0070238BF03469A4238BF1A464A800F
:1019A00030BD00BF7C050020EC0400202DE9F74F7E
:1019B00006461D469046002A50D0CB6828684B4901
:1019C00093F8049007223EF009FFD0B9B8F1010F57
:1019D00007D1474A0221304603B0BDE8F04F04F07A
:1019E000E7B9444F04460A2257F8241068683EF0CD
:1019F000F5FE002873D00134052CF4D16B683E4A03
:101A000013E008223D4928683EF0E8FE58B9B8F1D5
:101A1000010F04462BD00127394A3A4B9B1A4FEA53
:101A2000D30A934645E02B68374A0221304603B07B
:101A3000BDE8F04F04F0BCB908EBC5039B79A342A5
:101A40000FD200212846FFF74FFF524603460221DE
:101A5000304604F0ADF90135BD42EDD103B0BDE82B
:101A6000F08F224629464846FFF776FFF3E7244BDE
:101A7000244FDFF89CA0FF1AFF0800259846EBE7EB
:101A8000184600210193FFF72FFF009920223EF016
:101A9000A5FE019B014608B1013310E00BEBC30228
:101AA0009279A24215D3224619464846FFF754FFC1
:101AB00001374745D2D255F82730009300239A4585
:101AC000DED155F82730114A0221304604F070F972
:101AD000EEE71846FFF708FF0D4A0346F4E7B8F1B2
:101AE000020FE4B2C3D0022796E700BF142204001D
:101AF0001B220400542304007E220400ED45040050
:101B00000C7E04002C7F0400322204006A220400B0
:101B10004722040013460A46C168FFF747BF00008A
:101B200013B504460191A3B162B9019A0F4B04EBBE
:101B30004404072053F82230A0401840E040C0B2CF
:101B400002B010BD01A8FFF73DFE0028EDD0002037
:101B5000F6E72AB9019A064B03EBC2039879EFE73F
:101B600001A8FFF72FFE0028F1D1F3E77C05002044
:101B70000C7E04002DE9F04F274B284A9B1A4FEAB0
:101B8000D309CB685B7985B005460E461BB9244A5C
:101B9000022104F00DF9234B234A244F0821284643
:101BA00004F006F9224A0821284604F001F900242D
:101BB0004C4502D105B0BDE8F08FF36893F804807E
:101BC00001231A4621464046FFF7AAFF012221467B
:101BD000834600234046FFF7A3FF0328034628BFA0
:101BE00003235FFA83FA804601212046FFF77CFE3B
:101BF00057F82A3001930F4A0F4B57F82B100091DA
:101C0000D04598BF134602930C4A03460821284644
:101C100004F0CEF80134CBE72C7F04000C7E0400E6
:101C20009D220400B0220400BC22040054230400BE
:101C3000DA2204003C3104009B2204001723040034
:101C400013460A46C168FFF795BF000037B5164B2B
:101C500093F8203404460BB918B90024204603B089
:101C600030BD3EF0B3FD02AA013042F8080D012359
:101C700001A90E4806F087FA05460028EDD1214655
:101C8000009A01983EF035F8DDE900231344074837
:101C900003F8015C009906F0ADFA0099034806F0DC
:101CA000C2FA019CDAE700BF58080020382304007C
:101CB000034BD3E90030C31A58425841704700BF64
:101CC000580800202DE9F04F85B0FFF7F1FF0646D8
:101CD000002840F018818D4DC5F81804BFF34F8FD0
:101CE0006868AC6804AF47F8100D2040033005EB7E
:101CF00080003946FFF74AFC009B18B1D5F818243C
:101D0000002A66D004EA0302991C013305EB820223
:101D1000234005EB8303D268DB68029302F00303E0
:101D2000022B0192009169D1BDF8063078489DF8E8
:101D300004604FEA931ABAF1A00FD14628BF4FF0C2
:101D4000A00969F38F1309F10801ADF8063005F019
:101D5000A6FFC6F3C2068046002800F0BB8005F04F
:101D6000CDFF01A900230822404605F0DAFF0099C3
:101D700024EA01070137BF00B94538D95FFA89F96C
:101D800097B3FFB2A9EB0709214003315FFA89FB42
:101D9000B946604F05EB810108234A46404605F0ED
:101DA000C0FF37B109F108035A463946404605F0ED
:101DB000B8FF009B0AF1030A03EB9A030093D5F8DE
:101DC0001834002B50D1D5F81044DFF85C91072768
:101DD0006FE02A689A4204D86A60304605B0BDE8D0
:101DE000F08F04EA030081E74A49BB46D4E721406B
:101DF000033108234A4605EB8101D7E7012B69D15E
:101E0000BDF804604248C6F38311062928BF0621A5
:101E100061F3891602318900ADF8046005F03FFFD7
:101E2000C6F3C2068046002854D005F067FF0023A1
:101E3000082201A9404605F074FF0027BDF80420E0
:101E4000C2F38312BB1C97424FEA8303B7D20099B7
:101E50004A1C21400331009205EB810104224046D7
:101E600005F05FFF0137E9E7404605F04BFFFFF75C
:101E70001FFF80F00100C6B2AFE7E3685A79B2B144
:101E80001B79BDF8081003EB430259F8211007FA3B
:101E900002F3052E03EA010323FA02F308BF032627
:101EA000B34204D3236841461B6820469847E36841
:101EB0001C68002CE1D1404605F024FF204602F0CA
:101EC00091FFD5F818340BB9009B6B60002002F02D
:101ED0008BFFCCE7D5F8104474B90F4B5B88012B0E
:101EE000C5D90E4B0E480F49C01AC008000440F077
:101EF000020000F073F8BAE7236820469B68984711
:101F0000E3681C68E8E7002667E700BF5808002080
:101F10002C7F0400640800200C0500200C7E0400C7
:101F20004C7E0400DC2404007C0500202DE9F74FE2
:101F3000284C80460F46924601A9012218469B462E
:101F4000D4F80890FFF740FB88B3019D0026A91C38
:101F50005E4506EB010234D100211F4803F062FA0E
:101F600080F310006A1C02EA090204EB82020004FA
:101F700005EA0903033340EA1840D06014F823202F
:101F800068F3C50204F8232034F8232066F389128D
:101F900024F8232054F82320012167F39F2244F8DA
:101FA000232061F301026FF3820204F8232094F8E6
:101FB00020341BB1FFF786FE0028FBD103B0BDE83B
:101FC000F08F09EA020204EB82025AF82630D3604D
:101FD0000136BDE758080020740C002000231A4683
:101FE000FFF7A4BF13B502AC012344F8042D224629
:101FF000FFF79CFF02B010BD07B5CDE90023022317
:102000006A46FFF793FF03B05DF804FB1FB5CDE907
:102010000123069B039301AA0323FFF787FF05B063
:102020005DF804FB1FB5CDE90023069B0293079BD7
:1020300003936A460423FFF779FF05B05DF804FBBC
:102040007FB5CDE90123089B0393099B04930A9B69
:10205000059301AA0523FFF769FF07B05DF804FBAC
:102060002DE9F3478046304CD01C8A46174601A91B
:1020700000228008A568FFF7A7FA002840D0DDF805
:102080000490A66809F10200019001362840361A32
:10209000B6000330B74204EB80003BD83A465146C5
:1020A0003DF027FE0021214803F0BCF980F3100029
:1020B00009F101032B4004EB83034FEA184242EA83
:1020C0000040D86005EA0903033304EB830214F8E7
:1020D000231068F3C50104F8231034F823106FF3BC
:1020E0008F1124F82310518867F38F11518014F851
:1020F0002320022161F301026FF3820204F82320FE
:1021000094F820341BB1FFF7DDFD0028FBD102B0AD
:10211000BDE8F087324651463DF0EBFDBA1B0AEBB5
:10212000060104F10C00BBE758080020740C0020E5
:102130002DE9F8431F4B8846D3F8101405460024B8
:102140000A469AB9E9680C71D3F81014A1B9C3F81A
:102150001054EB681A60184F184EF61BF6084FF033
:102160000009B14511D12046BDE8F883D268107945
:10217000A04218D01268E4E7C968EA6809681160EB
:10218000D3F81034DB681D60E5E707EBC903494667
:10219000DA79EB68424528BF42461879FFF7DCFB45
:1021A00009F10109DDE701340A2CC9D14FF0FF34F0
:1021B000D9E700BF580800200C7E04002C7F0400E3
:1021C00010B5037A052B0C460FD0437A23B1084A89
:1021D0000849204605F049F90749204605F045F928
:1021E0002046BDE8104005F035B9002AF8D0F3E7E5
:1021F0005B27040037310400322F040073B5C38815
:1022000004460D4633B1144A00921449144A284634
:1022100005F02BF9217A05291CD0637A4BB1A088EF
:10222000FFF784FB0F4B104953F82020284605F098
:102230001CF9227A0D4BA08853F822600021FFF789
:1022400053FB0B4903463246284602B0BDE87040B6
:1022500005F00BB902B070BD5B27040068270400CD
:10226000602704002C270400373104008C27040069
:10227000802704002DE9F04385B01F460C9D002304
:1022800006460C46904695F80C902B732946384626
:10229000FFF7B4FFB8F1060F09D8DFE808F0041221
:1022A000181F283340003146284605F0DEF800228A
:1022B00029463846FFF784FF85F80C9005B0BDE845
:1022C000F08322683146284605F0CFF8EFE7D4E9DD
:1022D00000233146284605F0C8F8E8E7A3680093D4
:1022E0003146D4E90023284605F0BFF8DFE7E3686C
:1022F0000193A36800933146D4E90023284605F0F2
:10230000B4F8D4E723690293E3680193A3680093C8
:102310003146D4E90023284605F0A7F8C7E76369EA
:10232000039323690293E3680193A3680093314602
:10233000D4E90023284605F098F8B8E708292DE9E4
:10234000F84F80460E4617461C4635D8002593F8B0
:102350000C901D7319461046FFF750FFDFF88CA054
:10236000DFF88CB0AE4229D918F80520594620462E
:1023700005F07BF80135082DF4D11A49DFF874B067
:10238000204605F072F84FF0000A564524D918F897
:102390000A507E2D17D92E225946204605F065F8A1
:1023A0000AF1010ABAF1080FEFD10122214638469D
:1023B000FFF706FF84F80C90BDE8F88F51462046E1
:1023C00005F053F8D6E73DF065FC2844427812F05A
:1023D000970FE0D02A46DFE70349204605F045F88D
:1023E000DEE700BF56270400165804001458040006
:1023F0005027040058270400074B1B5C1F2B86BF87
:1024000003F01F0305494FF0A041012202FA03F334
:10241000C1F80C35704700BFD827040000030050F6
:10242000074B1B5C1F2B86BF03F01F0305494FF0B2
:10243000A041012202FA03F3C1F80835704700BF3A
:10244000D82704000003005008B50020FFF7E8FF7C
:102450000120FFF7E5FF0220FFF7E2FF0320BDE8C0
:102460000840FFF7DDBF0000C10710B5044642D5A4
:102470004FF08043D3F84036DA072ED54FF01023C3
:10248000D3F8043303F00703072B26D11D4B012299
:10249000C3F80425D3F80024002AFBD04FF0102104
:1024A000D1F8042322F0070242F00402C1F8042309
:1024B0000022C3F80425134AD2F80034002BFBD0C5
:1024C000BFF34F8F1049114BCA6802F4E062134307
:1024D000CB60BFF34F8F00BFFDE74FF0A0420C4928
:1024E0000323C2F81837C2F82037C1F82437C2F8DE
:1024F0003037FFF7A9FFA30742BF054B0C22C3F8F3
:10250000182710BD00E0014000ED00E00400FA05CE
:10251000000300500D4930B5A1F5BC72022591426F
:1025200001D800200EE08B1ADB1093FBF5F302EBD1
:10253000C30452F83330834205DC02DA04F10802A6
:10254000EDE7606830BD2146E9E700BF702C04006C
:1025500008B5FFF7DFFF024B002808BF184608BD8B
:10256000DC27040013B502AC002304F8053D0193F9
:102570009DF80330032B08D904210DEB010005F071
:1025800091FF30B9019802B010BD204605F080FFE0
:10259000EEE70020F7E708B500F08EFA00F078F8D3
:1025A000002005F055FF20B1852802D000F0C6F8C4
:1025B000FCE7FFF7D7FF3DF0EFFF05F081FF10B913
:1025C00000F0BCF8FCE708BD08B500F0B7F8FCE780
:1025D00062B6704772B67047FFF7C4BF00F0B2BA78
:1025E000034A431A934288BF0B1A1846704700BF2C
:1025F000FEFFFF7F10B5044600F0A4FA241804D3B0
:1026000000F0A0FA8442FBD310BD00F09BFA844294
:10261000FBD8F9E738B50D4614465AB151B148B167
:1026200005F092FF2946204605F064FF10B900F03E
:1026300085F8FCE738BDEFF30580003018BF0120B6
:102640007047000000000000F7B54FF080530025F0
:102650001C6E596E04F0FF0745EA010206A5D5E994
:10266000004502A9224347EA050361E90223082243
:102670003DF03FFB03B0F0BD000000000036CEF49B
:1026800000487047140D0020704705F061BB70478B
:1026900008B514F095F948B9054B1B7813B9054BEB
:1026A0001B781BB1BDE8084014F090B908BD00BF0D
:1026B00091010020940100202DE9F84307460E46C1
:1026C00014F07EF958B1184C184BDFF86890DFF819
:1026D0006880E41AE408240444F003040EB9BDE859
:1026E000F883D9F80000C0F10805B542A8BF354607
:1026F0002A46394640443DF0FCFAD9F800202A44E5
:10270000082AC9F800202F44A6EB0506E6D1084B9D
:102710005B88022B03D941462046FFF7A1FC00232A
:10272000C9F80030DAE700BF047F04000C7E040023
:1027300068050020600D0020580D002010B50C4CDD
:10274000226882B10B4B5B88022B0AD90A480B4BDB
:102750000B49C01AC008000492B240F00300FFF712
:102760007FFC00232360BDE81040FFF7ABBA00BF39
:10277000600D002068050020047F04000C7E04002A
:10278000580D002040F6F8731868431C04BF054B31
:1027900018684FF08053411C1A695B6908BF03FB3E
:1027A00002F070471410001008B5FFF7EBFFA0F51A
:1027B000104008BD0378022B01D814F015B97047FA
:1027C00010B5FFF7DFFF094C2061FFF7EDFF084B65
:1027D000E06000220749C3F80821204605F008F808
:1027E00018B1BDE81040FFF7EFBE10BD0C06002089
:1027F000640D00208C3304004FF4804070470220A9
:10280000704708B513460A4631B143B10146184630
:102810003DF06FFA002008BD6FF00A00FBE76FF093
:102820000B00F8E70128F8B507460C4616461D468A
:1028300010D80B44B3F5804F0FD28AB19DB1FFF78A
:10284000B3FF04EB873101442A4630463DF051FA8C
:102850000020F8BD6FF03800FBE76FF01600F8E7D6
:102860006FF00B00F5E76FF00C00F2E70128F7B509
:1028700007460C4616461D4624D80B44B3F5804F38
:1028800023D22AB3AB0826D0FFF78EFF04EB8734A0
:10289000044414F0B1F807460028FAD114F09CF86B
:1028A000214600972B4632460C4804F0DDFF0446D3
:1028B00014F0A2F80028FBD1201C18BF01204042D0
:1028C00003B0F0BD6FF03800FAE76FF01600F7E7DD
:1028D0006FF00B00F4E76FF00C00F1E70C0600203E
:1028E00001282DE9F041064624D8FFF75DFFDFF807
:1028F000508000EB863505F5804714F07DF80446DE
:102900000028FAD114F068F82346012229464046EF
:1029100005F06AF888B914F06FF804460028FAD177
:1029200005F58055BD42E8D1304614F06DF82046DB
:10293000BDE8F0816FF03800FAE74FF0FF30F7E7BD
:102940000C06002010B5084CD4F8083153B19BB2E6
:102950002246D4F8041194F80001FFF787FF002302
:10296000C4F8083110BD00BF640D00202DE9F84304
:102970001C4C1E46D4F8083181460F4690466BB178
:1029800094F80021824207D1D4F804211A449142DC
:1029900002D1B3F5807F01D1FFF7D4FFD4F808014D
:1029A00018B984F80091C4F80471C0F58075B54277
:1029B00034BFADB235464DB12A46414620443DF0C4
:1029C00098F9D4F808312B44C4F80831761BB6B214
:1029D00016B93046BDE8F883FFF7B4FF2F44A8448A
:1029E000DCE700BF640D002007B50C4B18680090B1
:1029F000FFF7DAFE042200F500410DEB02003DF086
:102A000078F9042269460DEB02003DF063F9B0FA53
:102A100080F0400903B05DF804FB00BF762C040091
:102A200038B505460C46FFF7BFFE00F500402A46C4
:102A300021460430BDE83840FFF7E3BE70B50646D6
:102A40000D461446FFF7B0FE04F500440434324648
:102A500029462044BDE87040FFF7D3BE00487047C8
:102A60007C2C0400042203210270817000220621C4
:102A70004270C17042607047B0F5A27F01D113F07F
:102A8000C5BF704710B5084CFFF7A4FD2378012B94
:102A900005D1FFF7E3FF06F0E7F800232370BDE858
:102AA0001040FFF795BD00BF700E0020014B187855
:102AB000704700BF700E00201FB502A8FFF7D2FFBD
:102AC000FFF7CCFF104A02A906F048F808B1FFF75B
:102AD0007BFDFFF7C3FF0368D3F81045FFF7BEFF88
:102AE000E2B24FF47031012421FA02F202232146AE
:102AF000009406F015F9FFF7B1FF06F09BF8034BC1
:102B00001C7004B010BD00BF792A0000700E0020B8
:102B100008B5FFF75FFD0A4B1B782BB9FFF7CCFF19
:102B2000BDE80840FFF754BDFFF798FF06F0C4F872
:102B30000028F5D1FFF792FF06F07CF8F0E700BF20
:102B4000700E002038B5FFF745FD0B4B1B78012BAD
:102B50000FD1FFF783FF022106F0BAF8044618F000
:102B600015FA0546FFF734FD4FF4705000FB0540A1
:102B700038BD0024F3E700BF700E00201F2886BF79
:102B800000F01F00044A4FF0A042012303FA00F0B6
:102B9000C2F80C05704700BF000300501F2886BF15
:102BA00000F01F00044B4FF0A04300F5E07003223B
:102BB00043F82020704700BF0003005008B51620DE
:102BC000FFF7ECFF1320FFF7E9FF1720FFF7E6FF01
:102BD0001120FFF7E3FF1420FFF7E0FF2D20FFF7A0
:102BE000DDFF13490223C1F838372F20FFF7D6FF46
:102BF0001520FFF7D3FF1620FFF7C0FF1320FFF7C4
:102C0000BDFF1720FFF7BAFF1120FFF7B7FF142011
:102C1000FFF7B4FF4FF40053C1F808354FF40043F9
:102C2000C1F808351520BDE80840FFF7A7BF00BF71
:102C30000003005030B50F4D8BB038F0E3FA0FCDE4
:102C400001AC0FC40FCD0FC42B68236001A83BF06B
:102C500013F9FFF719FD012038F04EFB38F0F8FAB0
:102C6000032801D138F000FB012038F049FB0BB0FC
:102C700030BD00BF842C040038F0C0BA07B502ABE9
:102C800023F8020D184638F0B7FA03B05DF804FBDC
:102C900007B502AB23F8020D184638F0B1FA03B0BD
:102CA0005DF804FB10B54FF470544443204638F0EF
:102CB00000FB0028FAD010BD38F086BA38F095BA7B
:102CC00010B5044638F093FA207010BD003018BFDC
:102CD000012038F013BB003018BF012038F00CBBC6
:102CE000003018BF012038F005BB08B938F0BFBA72
:102CF00038F0C5BA08B538F0ABFAC31E584258418F
:102D000008BD08B538F0A4FA023818BF012008BD84
:102D100013B50446032C104608D0042C10D0012C07
:102D200014D138F0FEFA204602B010BDA1F59C4245
:102D30000093203A44F62063002138F0B2FAF3E71A
:102D4000002102B0BDE8104038F09FBA0020EBE748
:102D500010B50C46FFF794FC036A0133036220466A
:102D6000BDE810400CF0E8BD38F0A8BA10B50C462C
:102D7000072942D8DFE801F004171D23292F353B2E
:102D8000FFF77EFC436A01334362012000FA04F43A
:102D900014F0DA0F03D114F0240F2ED00420BDE874
:102DA00010400CF003BEFFF76BFC836A01338362B3
:102DB000EBE7FFF765FCC36A0133C362E5E7FFF7A2
:102DC0005FFC036B01330363DFE7FFF759FC436BE1
:102DD00001334363D9E7FFF753FC836B013383630C
:102DE000D3E7FFF74DFCC36B0133C363CDE7FFF7B8
:102DF00047FC036C01330364C7E710BD2DE9F041C4
:102E000005460E4617469846FFF73AFC046801341B
:102E1000046043463A4631462846BDE8F0410CF08E
:102E2000E9BD000008B506280AD8DFE800F0040D67
:102E300013191F252B00FFF723FC43680133436060
:102E4000134B00221A6008BDFFF71AFC8368013398
:102E50008360F5E7FFF714FCC3680133C360EFE755
:102E6000FFF70EFC036901330361E9E7FFF708FC94
:102E7000436901334361E3E7FFF702FC83690133F0
:102E80008361DDE7FFF7FCFBC3690133C361D7E76B
:102E900098990020003218BF012211B1114638F074
:102EA0003ABA114638F02EBA08B5002038F036FA92
:102EB0000120BDE8084038F031BAF0B58BB01C46AF
:102EC0000546164612F0E7FD0146284612F0CDFEF3
:102ED000022C074621D0032C24D064BB4FF6FF738D
:102EE000ADF8263000230122CDE906230593149B7B
:102EF0000493BDF84C300393BDF8483002939DF81D
:102F0000443001939DF8403000930DF12602234692
:102F10003946284619F0AAF910E03378727843EA66
:102F20000223DDE7304612F0E1F94FF6FF739842D5
:102F3000ADF8260004D1284612F0A8FC0BB0F0BD75
:102F40000224CFE71FB50021039001AA44F201003B
:102F5000CDE90111FFF79BFB05B05DF804FBD0E95B
:102F60000223D1E90201994208BF90422CBF0120FF
:102F7000002070472DE900480C4802F06DF80C4B1A
:102F8000D3E9002312EB000B43F1000C094BD3E90A
:102F900000239C4508BF93455846614603D21BF168
:102FA00080704CF10001BDE8008800BF24000020C3
:102FB000780E0020E00E002037B505460C460A4882
:102FC00001A902F0BAF960B10570446001A9064890
:102FD00002F0DDF918B1054802F042F8002003B014
:102FE00030BD0420FBE700BF1000002024000020BB
:102FF0002DE930481A4B1B7804461BB9002528469A
:10300000BDE830880028F9D090F8203003F0FF05A3
:10301000002BF3D0FFF7AEFFD4E90223994208BF9B
:10302000904217D323690BB984F82030D4E90530D6
:10303000984721690029E1D094F8203003F0FF057A
:10304000002BDBD0D4E9022312EB010B43F1000C7F
:10305000C4E902BC2146034805F0F9F8CFE700BFF8
:10306000800E0020DC2C040013B5114B11491868A8
:10307000019008235822104802F04CF9044698B9F0
:103080000E4A0F4801A901F0BFFE044660B90121B4
:103090000B4801F0C1FF01230A4A0948194601F013
:1030A0001FFF094B01221A70204602B010BD00BF5D
:1030B000D82C0400840E00201000002021310000D4
:1030C00024000020FFFF7F00800E00203AB103683B
:1030D0005A614A1E51425141196100207047072030
:1030E000704738B590F8203004460D4683B98261A8
:1030F000FFF740FF421941F10003C4E902232369AD
:1031000003B1256121460020BDE83840FFF754BFD8
:10311000002038BD014801F09FBF00BF24000020FF
:103120002DE9F74F064601F080FF40B15A49D1E939
:10313000002312F1807443F10005C1E9004500212C
:10314000304601F082FF38B1544C236823B1206827
:10315000FFF74EFF002323600121304601F075FF89
:1031600020B1FFF707FF4E4BC3E9000101A94D480D
:103170004A4D4D4C4D4F02F01AF9002845D1DFF869
:1031800028A1464CDFF82CB1504605F076F82368AC
:10319000002878D083B12368D0E90201D3E9022363
:1031A000994208BF90422DD2236893F820301BB17A
:1031B0002168504605F04BF8504605F058F8D0E924
:1031C00002890746FFF7D6FEB8EB000869EB010954
:1031D00040464B46012873F1000347DB344DA845B8
:1031E00042D9FFF797FF42194FF496030021584642
:1031F00001F09AFE002841D1236813B9304601F04E
:1032000067FE276003B0BDE8F08F0378012B20D064
:103210000BD3022B14D14FF00008204605F027F8FD
:10322000002836D080F82080F7E7436893F8202004
:1032300032B9012283F820204168204605F007F8C2
:1032400001A9184802F0DEF801A9164802F0AFF80B
:1032500093E741682B68994202D100232B60EFE786
:10326000204605F00DF8EBE7BA68BDE700215846A7
:1032700001F0E0FE3846FFF7BBFE01E00D28F9D073
:103280000023236080E7002BBCD1304601F024FEF0
:10329000B8E701233B70D3E7780E0020E80E00204A
:1032A000E00E002010000020DC2C0400800E002026
:1032B000FFFFB4002400002043681B68184700008B
:1032C000024B5B6803B11847704700BFEC0E00204B
:1032D000020600F00F034CBF02480348DB0018440D
:1032E000704700BFF80E0020400F002008B5FFF720
:1032F000EFFF016009B9416008BD4B681B6843607E
:10330000FAE70000024B01465A681868104700BFF0
:10331000400F00200378052B0CD1084AD2F88434E2
:10332000D2F8802412F0FF0F04D1054ADBB2052B3E
:1033300008BF1046034B1B68184700BF00700240CF
:103340001C2D0400EC0E0020012806D002D3022818
:1033500005D070470348FFF7DDBF0348FBE703488C
:10336000F9E700BF102D0400142D0400182D0400EF
:10337000FFF7D0BF0148FFF7CDBF00BF202D0400ED
:1033800038B5831EDBB2062B98BF194A194C98BF7B
:10339000D25C2378A3F10203DBB288BF0022062BA4
:1033A0009ABF1349CB5C00239342054603D0A2B1D8
:1033B000114804F0D7FF022D01D0082D10D10123B0
:1033C0002278022A01D0082A0CD101229A4202D086
:1033D00053B106F0FDF9257038BD04F0EDFFEAE7C2
:1033E0000023EDE70022F1E706F0E8F9F3E700BF7C
:1033F000042D0400910F00202C0000202DE9F04F37
:1034000087B006AC002644F8106D05468946924602
:1034100098466B6800225F68294601232046B8471A
:1034200040B98DF80600049004460746BE4203D812
:1034300005202AE00136ECE76B680DF10602D3F8AF
:1034400004B02946012304A8D8476B680DF1070290
:10345000D3F804B02946012304A8D8479DF80730C3
:103460004B459DF8063015D1544511D1109A136083
:1034700088F8003088F801906A68023B5468294651
:1034800008F1020204A8A047002007B0BDE8F08FB1
:103490000134E4B26A68023BD2F804B02946002243
:1034A00004A8D8479DF806301F44BFE72DE9F7432D
:1034B00005462E4806F0A2F9044600283AD12C4BC6
:1034C00018702C4B18602C4B0146186048222B4872
:1034D0003CF033FC4822214629483CF02EFC294B85
:1034E00065BB294A1D72C3E900251A680AB9264A34
:1034F0001A60002004F074FF18B1852801D0FFF78E
:1035000021FD224E96F80890002506F10908ECB23C
:10351000A14504D904EB440414EB080423D102A907
:103520000B2301F8043D1948FFF7C6FE044608B115
:1035300006F00EF8204603B0BDE8F08395E80700DA
:1035400083E80700D1E73146E05CFFF7CFFE637800
:10355000FAB2934205D9A3781344DC4207F101077C
:10356000F1D10135D3E70027F1E700BF7133000047
:10357000910F0020880F00208C0F0020F80E0020F3
:10358000400F0020EC0E0020BD3800004C2D040040
:1035900010B506F0C1F808B9082010BD06F0C4F84F
:1035A00004460028F8D1044804F035FF0028F4D080
:1035B000FFF7C8FC2046F0E70C2D040005F0D2BF51
:1035C00006F0A4BC4FF08043D3F83824920702D50C
:1035D0000348FFF79FBED3F83824D107F4D47047CF
:1035E000212D040007B502A8822300F8043DFFF74F
:1035F00091FE03B05DF804FB2DE9F341037A00F17D
:1036000009040325064615FB03452746AC4231D085
:103610001CB394F80180002106E0E05CFFF758FE3F
:1036200003680131002B36D1CBB2984503D9A3787A
:103630000B44DC42F1D10334E8E73146E85CFFF7A4
:1036400055FE6A785FFA88F39A4205D9AA7813443E
:10365000DD4208F10108F0D10134337AE5B2AB4222
:1036600003D905EB45057D1901D10C4B05E04FF061
:103670000008E6E70024F0E713681A68002AFBD187
:1036800002A91E600B2301F8043D3046FFF714FE2B
:1036900002B0BDE8F0811120FAE700BF880F0020DA
:1036A000024B1878003018BF01207047900F00209F
:1036B00000F00F03072B10B5044604D806F0BEF93E
:1036C000204606F0E1FC2046BDE8104006F090BC24
:1036D00006F05CBC014B1868704700BF880F0020E3
:1036E00070B50A4B1B687BB11E7A0022D5B2B54279
:1036F00001D31B68F6E7013202EB42041C44A479B3
:103700008442F3D101B10D70184670BD880F0020BE
:103710001146FFF7D1BD08B500F00F03082B07D8FD
:10372000FFF7D6FD006818B1BDE80840FFF7C4BD3B
:10373000102008BD38B5054B05461C6804B938BDD6
:1037400029462046FFF7B8FD2368F6E7880F0020DA
:1037500038B5074B05461C680CB9062038BD29460C
:103760002046FFF7A9FD0628F8D12368F3E700BF3C
:10377000880F002038B504460D4606F080F848B1A1
:10378000054B1B78022B05D129462046BDE8384061
:1037900006F078B8082038BD910F002038B50446EF
:1037A0000D4606F06CF848B1054B1B78022B05D18D
:1037B00029462046BDE8384006F0D6B8082038BD76
:1037C000910F0020F8B543689B6805460C461646E5
:1037D00013B92EB1072002E098470628F9D0F8BDAA
:1037E0002B7AA34213D9093504EB44042C4467789F
:1037F000F3B29F4201D80020F1E762789A4208D9DB
:10380000A219A378D05CFFF753FF0136F0E7737875
:10381000FFDE00231B78FBE770B54368DB680546D5
:103820000C4603B198472B7AA34213D9093504EB10
:1038300044042C4400256678EBB29E4200D870BD4B
:1038400062789A4209D96219A378D05C06F09EFB8F
:103850000135F1E700235B78FFDE00231B78FBE7EF
:1038600043681B6903B118471846704770B5084B89
:103870001C6804B970BD267A0025E9B2B14201D3B3
:103880002368F5E700222046FFF79CFF0135F4E7A7
:10389000880F002070B5084B1C6804B970BD267AEB
:1038A0000025E9B2B14201D32368F5E72046FFF7CE
:1038B000B3FF0135F5E700BF880F002038B5047865
:1038C000092C054620D023D8032C00F0BC8012D848
:1038D000012C00F0A68040F28D800320FFF750FD00
:1038E0000220FFF7EDFC2846FFF724FF2846BDE83D
:1038F0003840FFF707BD052CF8D0C0F0B380062C88
:1039000000F0BF80082C13D12046FFF7D9FC95E0CA
:10391000812C0ED005D80F2CF6D0802C44D00A2C48
:10392000F1E7832C4CD021D3842C53D0852CDDD0CF
:1039300038BD5E48FFF7E6FC5C48FFF7FBFE0D2054
:10394000FFF7BEFCFFF7A6FF00F05BFF584B1B68BC
:1039500053B9584B187A00F0010005F0B3FE01206E
:10396000BDE83840FFF70CBD0120F4E7FFF792FFF8
:1039700006F0AEFA0020FFF703FD4F48FFF7DAFE2E
:103980004D48FFF7BFFC0E20FFF79AFC4B4B1B780E
:10399000023BDBB2062BCBD8494AD35C002BC7D005
:1039A000BDE8384004F008BD444B1B78062B05D019
:1039B000072B01D0052BBBD10220D1E70820CFE790
:1039C0003E4B1B78032BB3D106F0BAFA0028AFD0D8
:1039D0000420C5E7394B1B78032B05D106F0B0FA5C
:1039E00010B10420FFF7CCFC05F0B6FE00289FD0F4
:1039F0000620B5E7314B1B78032B01D0082B02D1F1
:103A00003048FFF75BFF0020FFF75AFC284B1C688B
:103A1000002C8DD020462946FFF74EFC23685C68B9
:103A2000F6E7FFF737FF00F0E3FE0220FFF7A8FC00
:103A30002046FFF745FC2846FFF764FC2846BDE812
:103A40003840FFF777BE1D4B1B78082B06D10220AC
:103A5000FFF796FC05F0C6FE0320EAE70520FFF716
:103A60008FFCF9E70320FFF72BFC1748FFF74AFC10
:103A70001548FFF75FFE114B1B78062B9CD10720E2
:103A80006EE78078FFF724FC294643680068984772
:103A900000283FF44DAFA87800F00F03013B062B40
:103AA0003FF646AFBDE8384005F0A2BF222D040026
:103AB0008C0F0020EC0E0020232D0400910F00201D
:103AC000042D0400242D0400252D0400C36903B136
:103AD00018477047036800221A845A62DA62C3E901
:103AE0001E22C3E9202203F134025A677047436063
:103AF000CA699A4227BF8A69026001F128020260FE
:103B000026BF0B67CB618B6700207047F0B5BE4DB9
:103B10000C7A2C70046840F24636B44200F0CD8234
:103B200000F2DD80B4F54A7F00F0428270D8B4F52F
:103B3000467F00F0008226D840F21536B44200F0ED
:103B4000DF810AD8002C00F0C981B4F5457F00F070
:103B5000CD81002303601846C7E140F21636B44217
:103B600000F0DC8140F21736B442F2D100240AB1F1
:103B700006791655013402269C420671C0F0DC819C
:103B80004FF44673AFE140F21B36B44200F0EC81D3
:103B9000B4F5477F15D240F21936B44200F0D78110
:103BA00040F21A36B442D4D100240AB1067916552F
:103BB000013400269C420671C0F0D78140F21B33CD
:103BC00091E140F22236B44200F0E58140F2233622
:103BD000B442BED100240AB1067916558B4E0F7A35
:103BE0003678DFF82CC2B74204F1010440F2558365
:103BF00001F1090706EB460607EB060E9C42BE5D87
:103C0000CCF800E00671C0F0D4814FF44A736AE149
:103C100040F23536B44200F00A8239D840F22E36EE
:103C2000B44200F0E0811DD840F22936B44200F0E1
:103C3000CB8140F22A36B4428BD100240AB10679F6
:103C40001655734E0F7D36683678B74204F101047D
:103C500040F0E28102269C420671C0F0C58140F22C
:103C60002E3340E140F22F36B44200F0C881B4F563
:103C70004C7F7FF46EAF00240AB1067916550134EB
:103C80000026A342067100F2EC8140F23E332AE1A5
:103C900040F23E36B44200F0E38108D840F23636B6
:103CA000B44200F0D08140F23736B442E1E7B4F5D7
:103CB000517F00F0EA8100F2F48140F24336B442D1
:103CC0007FF447AF00240AB1067916550134242643
:103CD0009C420671C0F0DA814FF4517303E1B4F5F0
:103CE000567F00F054826BD840F24E36B44200F05A
:103CF0001C8232D840F24B36B44200F0FD81B4F55C
:103D0000537F16D240F24736B44200F0E28140F2CF
:103D10004A36B4427FF41DAF00240AB10679165525
:103D2000013424269C420671C0F0E78140F24B33F7
:103D3000D9E000F0ED8140F24D36B4427FF409AF96
:103D400000240AB10679165501348E7D06719C4215
:103D5000C0F0EC8140F24E33C5E040F25336B4423D
:103D600000F0FC81B4F5557F16D240F25136B442D2
:103D700000F0E78140F25236B4427FF4EAAE00240C
:103D80000AB106791655013402269C420671C0F02C
:103D9000E68140F25333A6E000F0EC8140F2573662
:103DA000B4427FF4D6AE00240AB106791655013428
:103DB00024269C420671C0F0EB814FF4567392E0CA
:103DC000B4F55D7F00F0288248D840F25B36B442FB
:103DD00000F0F681B4F5577F1CD240F25936B44258
:103DE00000F0E18140F25A36B4427FF4B2AE0024D2
:103DF0000AB10679165501348E7D06719C42C0F0D9
:103E0000E08140F25B336EE0940F0020930F0020BE
:103E1000980F002040F26F36B44200F0F081B4F504
:103E20005C7F7FF496AE00240AB106791655AF4E3A
:103E3000AF4F36683F7896F801C0BC4504F10104E5
:103E400040F2308296F802C03E449C4216F80C6064
:103E50000671C0F0E2814FF45D7344E040F28536B4
:103E6000B44200F0F98115D840F27936B44204D05A
:103E700040F27E36B4427FF46CAE00240AB106797B
:103E8000165501344026A342067100F2E68140F245
:103E9000853328E040F28B36B44200F0F481B4F56B
:103EA000647F00F0F08140F28636B4427FF451AE78
:103EB00000240AB1067916558C4E0F7D3668367887
:103EC000B74204F1010440F0D4810E6A9C42367876
:103ED0000671C0F0D98140F28B3304E008240471EC
:103EE00023B94FF4457303600120F0BD0AB1047992
:103EF00014700B24012B04710ED840F21533F2E735
:103F000000240AB10679165501340E7D06719C42D3
:103F100005D340F21633E6E70124F2E700240AB1A4
:103F200006791655013402269C420671FFF41FAE35
:103F300040F21733D7E700240AB106791655013449
:103F400002269C42067103D340F21933CBE70024CA
:103F50000AB10679165501344E7E06719C42FFF473
:103F600024AE40F21A33BEE700240AB10679165592
:103F7000604E0027013437705E4E37782E78B74296
:103F800002D340F29B33AEE70926A342067103D861
:103F900040F22233A7E700240AB10679165501340E
:103FA00004269C420671FFF416AE40F223339AE7D2
:103FB00000240AB106791655013400269C42067188
:103FC00003D340F229338EE700240AB1067916554F
:103FD000464E36680134767806719C42FFF42EAE68
:103FE00040F22A337FE700240AB1067916550134DE
:103FF00002269C42067103D340F22F3373E700245C
:104000000AB10679165501344E7E06719C42FFF4C2
:1040100033AE4FF44C7366E78F7DB7427FF430AE1A
:104020000A269C42067103D340F235335BE7002435
:104030000AB106791655013400269C42067103D355
:1040400040F236334FE700240AB1067916550134A1
:1040500000269C420671FFF40FAE40F2373342E770
:1040600000240AB106791655204E0F7D3668367841
:10407000B74204F1010440F0A88005269C42067175
:10408000FFF421AE40F243332DE700240AB1067954
:104090001655013400269C42067103D340F2453385
:1040A00021E700240AB106791655013410269C42F6
:1040B000067103D340F2463315E700240AB10679AE
:1040C0001655013401269C42067103D340F2473352
:1040D00009E700240AB106791655013405269C42E9
:1040E0000671FFF41AAE40F24A33FCE6980F002046
:1040F000950F0020930F002000240AB10679165571
:10410000013401269C42067103D34FF45373EAE64F
:1041100000240AB106791655013403269C42067123
:10412000FFF40FAE40F24D33DDE600240AB106790C
:104130001655013404269C42067103D340F25133D4
:10414000D1E600240AB106791655013424269C4292
:104150000671FFF415AE40F25233C4E600240AB1F2
:1041600006791655013402269C42067103D34FF49A
:104170005573B8E600240AB10679165501340526B0
:104180009C420671FFF410AE40F25733ABE60024B8
:104190000AB106791655013406269C42067103D3EE
:1041A00040F259339FE600240AB1067916550134CE
:1041B0000E7D06719C42FFF41BAE40F25A3392E62C
:1041C00000240AB1067916550134374E36687778DF
:1041D000364E3770364E00273770354E3778334EAF
:1041E0003678B74204D3334F3E7801363E70C3E68B
:1041F0000726A342067103D840F26F3373E600240A
:104200000AB106791655013405269C420671FFF461
:104210000BAE4FF45C7366E600240AB106791655BE
:10422000214E0F7D36683678B74204F1010407D17C
:1042300003269C420671FFF421AE40F2793352E628
:104240008F7DB7427FF41EAE02269C420671FFF4BA
:1042500015AE40F27E3346E600240AB106791655C3
:10426000013400269C420671FFF423AE40F28633EF
:1042700039E68F7DB7420BD100269C42067103D3ED
:104280004FF464732FE600240AB106791655013401
:10429000074F3E7801363E709FE70023CCF8003090
:1042A0001B78FFDE0023FBE7980F0020920F002011
:1042B000950F0020930F00204360CA699A420ED3E5
:1042C0008A6902608A69C8691A448A610A6FC01AD9
:1042D0001A44C86100300A6718BF0120704701F115
:1042E000280202608B670020704710B5044658B959
:1042F0000868037B202B09D100F10E01072218303A
:104300003BF0F7FC204610BD0320FCE70620FAE74F
:10431000037A012B08D9427B012A00F10C0306D94C
:10432000827B13445878704700235B78FFDE0023BC
:104330001B78FBE72DE9F0430B7889B005460E4664
:104340000E2B1AD8DFE813F05C0041015C005C0022
:1043500019000F00A600190019003E0119005C00A9
:104360005C005C005C004A78D1094FEA521330D0FF
:1043700013F0030303D0012B21D006241BE002F02D
:104380001F02012AF9D1B478062CF6D105A80393AF
:1043900000F0B4FC03ABF278317900930746034692
:1043A0002846FFF72BF8052805D0039A3946701CDC
:1043B00000F042FA0446204609B0BDE8F083B37825
:1043C000212BDAD1B6F80720072AD6D10168183197
:1043D000EDE7012BD1D1B3780768202B12D0222B27
:1043E000CBD1B6F80730002BC7D197F82030B6F8FC
:1043F00003403C8403F0010304F00104A34223D1F1
:104400000024D8E7B6F80720072AB6D13B73B6F8E0
:1044100007300024DBB27B7320460E37CDE90573ED
:10442000079400F0DFFC204605A9FFF7A3F9044636
:1044300030B96B4B03A9CDE9033500F0EBF9044625
:10444000002000F0D1FCB6E7A4B2002C0CBF032181
:104450000221FFF73BFB002CD2D12B7A012B40F23B
:10446000B8806B7B05F10C02002B00F0B480AB7BB5
:10447000D05C05F00FFC2846FFF74AFF05F00AFC68
:1044800007F134037C62FC62C7E91E44C7E920449B
:104490007B6790E7037A002B00F09F80837A00F11E
:1044A0000901002B00F09780C27AB3788A5C9A42A7
:1044B000A6D01B06F4780AD524B1032C0CBF002427
:1044C000032478E701212846FFF700FB73E7012C5E
:1044D00096D003D3032C93D003246CE70668FFF730
:1044E00017FF404B059306F10C030693B76A80460D
:1044F000B7B9F36FF46AB767C6E91F736CB106F119
:104500002C0103C906F1240383E80300F76205A91F
:104510004046FFF743F9044600E074620021D2E709
:10452000D6F88490706A4F4528BF4F4606F1340490
:104530003A4621463BF0DDFBF36F3B44C6F8803042
:10454000A9EB0703B367F36A00223C44F267746780
:10455000002B35D006F12C0999E8030006F1240759
:1045600087E803001446F262B36F706A1BB9746A7D
:10457000002CCCD1D2E7B26A716F9A4216D83BF0C8
:10458000B8FBB36AB26FC6F88030D21AB267726FE6
:104590001A44726700212846FFF798FAF36A7BB144
:1045A00099E8030087E80300F462DDE71A463BF070
:1045B000A0FBB26FB36AF2679B1AB362736A1344CB
:1045C0007362D4E70321FFF781FA2846FFF782FAE6
:1045D00016E76378FFDE1B78FCE75B78FAE700BF3D
:1045E000EB420000B94200001FB503681B8CDC07DA
:1045F00014D5037A012B13D9437B00F10C0493B13A
:10460000837BE05C9306CDE901120CBF01230023FC
:1046100001A90393FFF7AEF804B010BD0820FBE733
:1046200000235B78FFDE1B78FCE70368D3F880008B
:10463000704700002DE9F3410468238CDB07064630
:104640008846174631D5002000F0CCFBA56FBDB1E0
:10465000BD4228BF3D46616F2A4640463BF049FBBC
:10466000A36FC4F880505B1BA367636F2B44636721
:104670000024002000F0B8FB204602B0BDE8F08125
:10468000636A83B9C4E909873046FFF741FE0C34F9
:10469000074B019469460093FFF780F8002814BF88
:1046A00004469224E5E71124E3E70824E4E700BF89
:1046B000EF3A0000002070472DE9F04F87B04B68BB
:1046C000029281460C465BB90B681B681B683BB9BC
:1046D0008D682DB9C0E90055284607B0BDE8F08FB8
:1046E00005F082F9E768029B9F4228BF1F464FF002
:1046F000000804F110038346019746460125039301
:10470000019B002B2DD0A368019A616893429A46C1
:1047100028BF924641B352460BEB06003BF0E9FA44
:1047200000236360A268E3680199A2EB0A02A3EB8D
:104730000A03A1EB0A01A260E360019156440ABB9F
:10474000B8F1000F38D02268126812682260002B7E
:1047500030D02368D3B963601EB1029BB34288BFD7
:104760000025C9E900B6B7E7002BDBD02168039824
:104770004B680BEB0602D3F804805346C0474FF05A
:104780000108CFE7002B08BF0025B9E70DF1180A93
:1047900000234AF8083D21684B685B6800221F46E9
:1047A00050460123B84708B92061A9E7A36801333F
:1047B000A360F0E71D46A3E7002BCAD145469FE75B
:1047C000084B1A7882420CD0052818BF064A187088
:1047D00018BF137805481CBF23F002031370FFF7BE
:1047E0006DB87047A80F0020C40F00205C2D040096
:1047F00008B50020FEF75CFF8020BDE80840FEF70A
:1048000057BF08B50020FEF763FF8020BDE80840D1
:10481000FEF75EBF38B505460C4605F08BF9A84299
:1048200003BFD4E90001034BC3E90001102008BF16
:10483000002038BDC80F00207FB5C38893421D46B5
:1048400028BF154693420E46144620D9802005F015
:1048500011F8B4FBF0F303FB1040B0FA80F040090C
:1048600003900020CDE9016500F0BCFA01A9802089
:10487000FEF780FF044620B906498020FFF7CAFFF3
:104880000446002000F0B0FA204604B070BD0020BD
:10489000E6E700BF902D04002DE9F04F0C78062CC0
:1048A00087B00E4600F0FC8120D8022C3DD003D802
:1048B000012C32D00624EDE1032C32D0052CF9D1A5
:1048C0000DF10D00B04D8DF80C4005F0C7F8002338
:1048D0002B609DF80D3003F01F02032A00F2848143
:1048E000DFE812F02D001D01790165000D2C00F0AC
:1048F000C58107D80B2C18D00C2CDBD10020FFF77A
:104900005FFF12E00E2C00F0C981852CD2D19F4BA5
:104910001B78032BCED1042000E00320FFF750FFCB
:10492000C8E79B4800F0D0FD08B90024B2E1994BDC
:1049300001221A60BFF36F8FBFF34F8FF5E7C3F308
:104940004116A6BBDB099DF80E1000F0A2800629D7
:1049500016D0082900F0908049BB8F4C02222046D7
:104960003BF0EBF9237843F0010222708B4A127876
:10497000910744BF43F003032370022286490EE0EF
:104980009DF81030022B16D0032B65D0012B0ED1D1
:10499000BDF81330002B00F06E81814912220DF119
:1049A0000D00FFF749FF0446062C40F0258103A8BF
:1049B000FEF7CEFE0DE1BDF81370002F00F05B8115
:1049C000092F28BF0927FEF785FE4FF00908044686
:1049D000B14654BB704C73493A4620463BF089F9C6
:1049E0002671A4F80280FEF75BFE18B1E37943F06C
:1049F0002003E371FEF76EFE6B4BC3E900049F607A
:104A0000BDF81320DA60002000F0ECF9674980203F
:104A1000FEF7C4FE044620B965498020FFF7FAFE80
:104A20000446002000F0E0F9BEE7CDF804904FF016
:104A3000000A63680022D3F804B02146012301A8CC
:104A4000D84730B9237A1E442368D044F6B21C6894
:104A5000BFE70AF1010AECE7BDF81330002B00F0C4
:104A60000A81BDF811109DF80F0000F095F901467C
:104A700000289CD0027892E7444A1278052A03D194
:104A8000454A1370012279E7042A90D1424B1E70E7
:104A9000F8E703290FD009292BD0012987D1BDF8C8
:104AA0000F30012B83D1FEF7FBFD60B13B4A137839
:104AB00023F002030FE0BDF80F30012B7FF477AF36
:104AC000FEF7EEFD18B90F2405F031F8E2E0334AA5
:104AD000137843F0020313702B68002B00F0CB8097
:104AE00005F028F8044600287FF41FAF04F0DCFF2F
:104AF000D0E0264B1B78043B012B01D90824E3E7C7
:104B00009DF80F302BB9FEF7C5FE0420FFF758FEC5
:104B1000E2E7012B56D1FEF7A9FE0520F6E701A931
:104B20009DF81100FEF7DCFD074608B91024CBE71D
:104B300003AA9DF80410FEF7EBFD062804465BD19E
:104B40009DF80D2012F0600FBED1104B9DF804109F
:104B500018789DF80E30D6092CD073B10A2BB3D13A
:104B60000528CBD13846FEF77BFE0B49324608704C
:104B70000DF10D00FFF760FE2BE00528BED10649C0
:104B80000B800222F4E700BFC80F0020A80F00200E
:104B9000D00F00205C700240D40F0020C40F002012
:104BA0007C2D04005D2D0400AC0F0020A82D040016
:104BB000902D04000B2B87D105289FD1BDF80F3015
:104BC000FF2B01D907247FE79DF80F203846FEF719
:104BD000F9FD044610E09DF81100020706D19DF88A
:104BE0000D3013F0600F0BD006246DE703A9FEF71C
:104BF00092FD06280446F2D0002C3FF46DAF63E727
:104C00009DF80E20384B9DF811401B78012A1ED0CC
:104C100012D3032AE8D104F00F02072AE4D8BDF822
:104C20000F100029E0D1052B02D0002A7FF466AFD7
:104C3000204604F0DDFE4FE7052B02D023077FF46A
:104C40005DAF204604F0E0FE2849088099E704F0B3
:104C50000F02072AC8D8BDF80F100029C4D1052BB0
:104C600002D0002A7FF44AAF204604F0E7FE204637
:104C700005F00AFA30E704F057FF56E64FF080439C
:104C8000D3F8384414F0010401D0022037E60120A3
:104C9000FFF796FD204607B0BDE8F08F01202EE615
:104CA000C8780328F6D0124D2B68D3B100222A60B1
:104CB00069689847044600287FF406AF2B6823B143
:104CC000B378002B7FF431AE10E70A4B1B68082B3A
:104CD00004D1094B1B68002B3FF427AE04F024FFDE
:104CE000D8E70E24F0E600BFA80F0020D40F002064
:104CF000C80F0020300100103401001008B140231B
:104D000003600148704700BFD40F002070B54FF01A
:104D1000805286B0D2F8A830D2F8A42000926FEA70
:104D200083436FEA934302AD9BB2094A094E0D21BA
:104D300028463BF089FC002428463BF047FD84428E
:104D400001D306B070BD2B5DA3550134F4E700BF5D
:104D5000B02D04005C87002010B50E4B53F82040A6
:104D600023780BB9A01C10BD0020FFF7C7FF224617
:104D7000E4B2131B12F8011BDBB231B901335B0043
:104D8000DBB243F440730380EDE7131BDBB220F882
:104D90001310EEE7082E040008B9FFF7DDBF052861
:104DA00007D8054A105C20B1044B53F82030002B83
:104DB000F3D10020704700BF202E0400082E04000D
:104DC00072B6024A13680133136070471410002052
:104DD000034A1368013B136003B962B6704700BF12
:104DE00014100020FFF7ECBFFFF7F2BF435882B06A
:104DF0003BB10023435043580193019B012002B073
:104E000070471846FBE7000070B5284C4379284DE1
:104E100044F82320274C04EBC3031B7973B16B8840
:104E2000012B09D92448254B2549C01AC008000484
:104E300040F00200FDF7D2F8082070BD03680A8830
:104E4000C3F8082590F904308A78002B4FEA421203
:104E5000AFBF03F1604303F00F031A49D2B2A9BFF9
:104E600003F56143CA54D2B283F8002390F90430A9
:104E700015495E09012203F01F0302FA03F341F80A
:104E80002630437904EBC30144F833006B880A7180
:104E9000022B09D90848094B0C49C01AC008000464
:104EA00040F00300FDF79AF80020C6E7201000202C
:104EB00014050020181000205C7E04000C7E040005
:104EC000362E040014ED00E000E100E0582E04004E
:104ED000036801221A607047036801225A60704714
:104EE000F7B505684FF480348C40C5F80843056871
:104EF000C5F848438D0005F5A0750668ADB20027DA
:104F0000775175590195019D056801F5A87122F049
:104F10007F4245F821200268C2F8444313B1036878
:104F2000C3F8044303B0F0BD2DE9F34799464FF4AD
:104F30008038036808FA01F8C3F848830368C3F8A7
:104F4000088322F07F4502688E000F46D2F80415D0
:104F5000324406F5A076D2F84035C2F84015B6B214
:104F600002684FF0000A42F806A05B1A92590092BC
:104F700023F07F43012B0446009A0BD1254B4FF4BD
:104F8000806043F001039847236843F806A09B59CB
:104F90000193019B2368D3F80465C3F84483AB1BDA
:104FA00023F07F43012B07F5A877236819D101353A
:104FB00043F82750174B4FF4806043F001039847A4
:104FC0002368D3F804359E4209D12368C3F844838B
:104FD00023680020C3F8048302B0BDE8F0870D20E9
:104FE000FAE743F827502068D0F804156A1A013A06
:104FF000C9F1FF1322F07F4203F57F439342EED3C2
:10500000002AE2D1013540F827502368D3F804354F
:105010009942D9E7302E040002680223C2F84433D3
:1050200011B10268C2F8043370474FF4827100680E
:10503000FFF7DCBE4FF4803303FA01F10368C3F8D5
:1050400048130368C3F808137047890001F5A0717D
:1050500089B20068FFF7CABE0368D3F80405704739
:1050600090F9043001215A0903F01F0301FA03F3F8
:105070004032024941F82230704700BF00E100E0B1
:10508000024B034A1B681068184700BF201000201D
:105090001810002038B50B0704460FD53AF0FAFD7A
:1050A000651C435D03F00303012B07D13AF0F2FDC9
:1050B000435D03F00303012B08BF2034204638BDB5
:1050C0002DE9F04F87B08A4614460293064618B978
:1050D000012007B0BDE8F08F0029F9D0029B002B1A
:1050E00000F0138102F004030D460493214630784A
:1050F000FFF7D0FFC7B23F2F06F1010823D00BDC2A
:10510000D7B12A2F38D021462878FFF7C3FF87422E
:1051100005F101061FD0DBE75B2F7DD05C2FF2D1BC
:10512000E307F0D421467078FFF7B4FFC7B2002F31
:10513000E9D006F10208E6E7E106287839D52F28FC
:1051400037D10020C5E72B78002BC1D02F2B05D1FC
:10515000A207BDD46E1C35464646C7E72E2BF9D1B3
:10516000049B002BF6D05545B2D0A307F2D515F815
:10517000013C2F2BEED1ABE770782146FFF78AFF79
:10518000C1B22A2919D02B782E2B09D1049B3BB10F
:1051900055459DD0A70703D515F8013C2F2B97D077
:1051A00079B9A607CDD5E406CBD42F2128463BF00C
:1051B000EEFA003018BF01208BE7214618F8010FE6
:1051C000DCE72F291FD0029B24F004095F1E04F0A6
:1051D000020AAB4621469BF80000FFF75BFFC6B210
:1051E0000135002E3FF474AF3B464A4659464046CF
:1051F000FFF766FF01287FF46CAF2F2EE9D1BAF1DB
:10520000000FE6D064E7A007DDD528463BF0BFFAE3
:10521000064600289FD15BE7287800283FF458AF66
:105220002F2802D1A1073FF553AF2146FFF732FFE8
:105230008346B8F1000F3FF44BAF7378212B01D0B8
:105240005E2B25D1023601230122019304EA0203D9
:105250004FF000090393214630780592FFF71AFFBB
:10526000C3B25D2B06F10107059A14D112BB019B55
:105270004B453FF42DAF002F3FF42AAF7A1C04D1E9
:105280002B785B2B7FF424AF47466E1CB84662E751
:1052900046460023D8E72F2BF2D05C2B07D1039A88
:1052A00042B921467078FFF7F5FEB71CC3B2002B58
:1052B0003FF40EAF3A782D2A21D121467878059314
:1052C000FFF7E8FEC0B2059BC8B15D2817D05C2887
:1052D00007F102060BD1039A4AB92146B878FFF7C5
:1052E000D9FEC0B200283FF4F3AE059BFE1C9B45DF
:1052F00003DB8345D8BF4FF001090022ABE73E46F0
:105300009B4508BF4FF00109F7E70320E1E6402382
:10531000FFF7D6BE10B561B1B2FBF3F403FB142462
:10532000A4B244B9C0E9001484608281C3812046DC
:1053300010BD0E20FCE70920FAE737B550E8013F21
:105340009DB2C48925448489A54228BF2D1B0489A8
:10535000A54202BFBFF32F8F002207E0C5EA030575
:1053600040E80154002CE9D14FF001028DF80320F0
:105370000193019B9DF803200B6002F0FF0322B113
:105380000B880068184403B030BD1846FBE70A8854
:105390004B889A4209D150E8012FC2EA024240E804
:1053A0000123002BF7D1012070470020704737B54B
:1053B00050E8023F1FFAA3F5C488A54202BFBFF31D
:1053C0002F8F00220DE0C48925448489A54228BF7F
:1053D0002D1BC3EA054540E80254002CE8D14FF0EC
:1053E00001028DF803200193019B9DF803200B60BF
:1053F00002F0FF0322B14B880068184403B030BDAF
:105400001846FBE70A884B889A4209D150E8022FD8
:10541000C2EA224240E80223002BF7D10120704764
:105420000020704750E8002F0B4640E8003C9CF0FD
:10543000000FF7D11046704750E8002F42EA0103F1
:1054400040E8003C9CF0000FF6D11046704750E851
:10545000003F43EA010240E8002C9CF0000FF6D127
:105460001046704750E8002F02EA010340E8003C74
:105470009CF0000FF6D11046704750E8003F03EA59
:10548000010240E8002C9CF0000FF6D11046704756
:1054900050E8003F03EB010240E8002C9CF0000FB5
:1054A000F6D11046704750E8003FA3EB010240E8F8
:1054B000002C9CF0000FF6D1104670470121FFF739
:1054C000BBBF0121FFF7C3BF0021FFF7CBBF002106
:1054D000FFF7D3BF2DE9F0438368D3F85463C6F3D5
:1054E000400689B0074636B10022114609B0BDE832
:1054F000F04301F017BE012906D91E4A022109B066
:10550000BDE8F04300F054BC1B4C1C4DDFF870901C
:105510001C23E2182D1B4FF06408B5FBF3F503FBC9
:1055200005251C34AC4202D109B0BDE8F08354F823
:105530001C0C54E90623017900689A1A1B1ADBB285
:10554000039308FB03F3B3FBF2F3CDE9016334F8F3
:10555000043C0093CDE9061254F8083C11FB08F115
:105560003846B1FBF2F1CDE904214A46082100F0AA
:105570001FFCD6E7942E04002C7F0400647F0400F7
:10558000A72E040010B590B1D0E9012301689B1A41
:10559000DBB20A60013BDBB2FF2B026802D10020C4
:1055A000107110BD11684C1C14600B70F2E70E20D6
:1055B000F7E738B504460020FFF714FC226861685D
:1055C00013688B4215D9591E116013F8015C228BA8
:1055D000E36802FB05352268A36811685B1A11793C
:1055E000DBB2994200D213710020FFF7FDFB284681
:1055F00038BD0025F8E738B5054600200C46FFF712
:10560000F1FB2A681368591C1160E968641A298B38
:10561000B4FBF1F41C700020BDE83840FFF7E4BB98
:1056200030B18A68B2F8543343F02003A2F85433FF
:10563000704710B543689C686068036801219B68E7
:105640009847A36810B903221A7010BD0422FBE723
:10565000096800683BF0A8B808B13BF0B7B87047DC
:1056600010B50446FFF7F8FF23462044834201D1DA
:10567000002010BD13F8012B3F2A01D02A2AF5D1B2
:105680000120F6E738B50546836800681C8DFFF7F2
:10569000E3FFAB68DA8B2044B0FBF2F302FB1300AC
:1056A000B0FA80F0400938BD10B584680068FFF793
:1056B000D3FF238DE28B84F82000C0B2034493FB18
:1056C000F2F102FB11330133A382E38C0131184460
:1056D000218390FBF2F3591C02FB13030133618316
:1056E000E38204F1140010BD38B5054683680068F4
:1056F000DC8CFFF7B1FFAB68DA8B2044B0FBF2F330
:1057000002FB1300B0FA80F0400938BD2DE9F047E4
:10571000089C1E4609BB1B4F1B4CE41BE40894422B
:10572000B94606D91948E50000EB82080C46A542A7
:1057300001D100230EE009EB0403D8F800005B68F8
:1057400019683BF031F807EB040A08340028EED161
:10575000DAF804303360BDE8F0870028E9D001783A
:10576000436839B12146104698472368002BE0D0A2
:105770003460F0E7120199189B58002BD9D03160A2
:10578000E9E700BFB47D0400FC7D0400C8040020EC
:1057900030B50368D3F84C5385B00446EDB100230F
:1057A0000A2201A9284602F0C7FA2368029AC3F820
:1057B0004C2300210A2201A83AF0BFFA00230A2252
:1057C00001A9284602F0ADFA284602F052FA2368F1
:1057D000D3F84C0318B9C3F8480305B030BD01A98C
:1057E00000230A2202F0A8FA206800230A2201A955
:1057F000D0F84C03019302F094FAEEE707B5836802
:10580000C9B193F822208A4212D00D4A0092332265
:105810008DF8042001F12F028DF805206D22ADF8DE
:10582000062083F822106A460649006901F01DFE31
:1058300003B05DF804FB83F82210034AF4E700BFCD
:105840001B5B313B37310400C82F040007B5836868
:1058500093F823208A4214D045F61B32ADF800207D
:1058600034228DF8022001F12F0283F823108DF8E5
:1058700003206D22ADF80420034900696A4601F057
:10588000F4FD03B05DF804FB37310400014901F079
:10589000ECBD00BF3B310400014A024901F0E5BD07
:1058A000BE2F0400373104002DE9F84F00250746CC
:1058B000884614460560267866B13AF0EBF9304424
:1058C000437813F008030CD00023237001343B68A5
:1058D0000B2BF0D93B68002248F823202846BDE86E
:1058E000F88F3A68511C396048F822401D4694F8F8
:1058F0000090B9F1000FEAD0002D40F08A80B9F194
:10590000270F05D0B9F15C0F0ED0B9F1220F79D174
:105910002046FFF7A1FE611C024620463AF0F4F94A
:105920004D4626463446E2E7661C2046FFF794FEC5
:105930003146024620463AF0E7F9F3E7B9F15C0F49
:1059400001D0661CEEE760788542EED0302825D184
:1059500002234FF00009E05CA0F13001C9B2072931
:105960005FFA83FA17D8013341EAC901052B5FFAC0
:1059700081F9F0D19A462046FFF76EFE0AF1FF3B0F
:10598000A344821CA2EB0A02594620463AF0BCF915
:1059900084F80090C6E7BAF1020FECD17828D0D194
:1059A00002214FF00009635CA3F13002D2B2092A50
:1059B000C8B214D842EA091303295FFA83F90CD15B
:1059C0004FF0040B2046FFF747FE0BF1FF3AA244CD
:1059D000821CA2EB0B025146D7E70321E3E7A3F1B8
:1059E0006102052A03D8573B43EA0913E4E7A3F110
:1059F0004102052A01D8373BF6E70228A1D04FF033
:105A0000030BDFE73AF046F9484443781B0798D583
:105A10005DE7A94504F1010690D12046FFF71CFE81
:105A20003146024620463AF06FF9002579E72DE924
:105A3000F34106460F461446002514B902B0BDE8EE
:105A4000F081706803682246D3F80C80791901ABA5
:105A5000C047019B1D44E41A002BEED1B3681A78AD
:105A6000032AEAD0D3F854239206FBD5B3F8542383
:105A70006FF34512A3F85423DFE700000A4619B17B
:105A80000249006801F0F1BC704700BFE42F040038
:105A90002DE9F74F054617460E46002975D00C46EE
:105AA0003AF0F8F8A4EB060A14F8013B18444378DE
:105AB0001A07F5D41FFA87F905F110083046FFF7E9
:105AC000CBFDAB68DB8BA0EB0A00DB1B98424FF0F1
:105AD000000406EB0A0B15D901933AF0DBF81BF82A
:105AE0000420019B1044417811F0080F02D00A2ACB
:105AF0002FD02346A968C98B3A198A4228D201348B
:105B0000EAE70134A04218D01BF804300A2B0AEB54
:105B10000408F6D1286901F09DFC22462C4659461E
:105B20002846FFF784FF54F8100FFFF7AFFEB9B215
:105B3000204608F1010AFFF7A1FF286906EB0A01D8
:105B400001F093FC286903B0BDE8F04FFFF79EBE5B
:105B50001C46286901F07EFC224659462846FFF77C
:105B600066FF544434443AF095F8A4EB060A14F85E
:105B7000013B184443781B07F5D42869FFF786FEDC
:105B800049464046FFF77AFF98E703B0BDE8F08F3B
:105B90000A4619B10249006801F067BC704700BFAE
:105BA000DE2F04000A4619B10249006801F05DBC0D
:105BB000704700BFEA2F040070B50546FFF774FD7B
:105BC000037B0288818801339A42044601D101296E
:105BD00015D0012905F1100604D9013989B23046E2
:105BE000FFF7E0FF2388217B8B4209D9013B591A3B
:105BF00089B23046FFF7CCFFAB6800221A8570BD32
:105C0000C91A013189B23046FFF738FFF4E7F8B519
:105C10000546FFF749FD04468788C6882846FFF7F2
:105C200031FD78B12869FFF731FEB74205F1100563
:105C30000ED161882388C91A284689B2BDE8F84088
:105C4000FFF7A6BF2846FFF74FFD0028EAD1ECE793
:105C5000A388E188C91A89B22846FFF7A3FF2388E1
:105C600061888B42E7D9591A284689B2BDE8F840C5
:105C7000FFF704BF38B50546FFF716FD02884388D5
:105C80009A4204468388C28801D1934214D09A4232
:105C900005D9D21A92B20B49286901F0E6FB238894
:105CA00061888B4205F1100007D9591A89B2FFF7B4
:105CB0006FFFAB68DA8C1A8538BDC91A89B2FFF755
:105CC000DDFEF6E7D82F0400F8B51E46C3685B6812
:105CD000986004464068036817461D682E4A2346AC
:105CE000A847054600284DD1606901F0C0FF054670
:105CF000002847D1A368C3F84803A368C3F84C033E
:105D000001464FF45672A0683AF017F8A268DFF81F
:105D100098C0B2F8543343F02003A2F85433A36878
:105D2000B3F8542367F38202A3F85423A268B2F8AD
:105D3000543343F00803A2F85433A36801221A70C5
:105D4000A3685022DA83A36818229A83134A144B5B
:105D50009B1AD8082946814216D1072B04D9114B2A
:105D6000114804223AF0F0FA66B19DF81810E06884
:105D7000FCF7DEF90028A1BFE368DB6801225A7155
:105D8000B8BF04252846F8BD02EBC1077F683F680D
:105D90004CF821700131DEE721560000B47D04008B
:105DA000FC7D040051560000C8040020FFF73FBEF0
:105DB0000CB4F7B508AB02AD53F8046B45F8043DDD
:105DC0000F468168D1F854335B07044621D591F81A
:105DD0002230BB421DD002222231684639F089FFB1
:105DE00039462046FFF70AFD2A463146206901F070
:105DF000B9FB9DF800102046FFF700FD9DF801104B
:105E000011B12046FFF722FD03B0BDE8F04002B01B
:105E100070472A463146206901F0A4FBF4E70000F0
:105E20008168002281F82C2081680A858168CA84F3
:105E30000368024A0321FFF7BBBF00BF37310400EC
:105E400070B583681E78012E04461AD14068036835
:105E500000219B689847054688B908212046FFF72E
:105E6000CDFC31462046FFF7F1FC2069064901F0E0
:105E7000FCFAA36802221A702046FFF7D1FF2846D9
:105E800070BD0825FBE700BF3A310400F8B50446B1
:105E90008068C58CAB18B3F5C07F0F4616463BDA59
:105EA000002A39D0038DED1A03F12C0113442C3351
:105EB000ADB201446A1C184439F026FFA068038D76
:105EC0002C3332463946184439F01EFFA0682C3076
:105ED000FFF7C2FBA368D884A268138D2C33134448
:105EE00020460E4A0821FFF763FFA3681A8D32444B
:105EF0001A852046FFF7C6FB40B12069FFF7C6FCB4
:105F000055B12046BDE8F840FFF781BE2046FFF7B7
:105F1000EBFB0028F1D1F3E7F8BD00BF37310400F7
:105F20002DE9F04104468068D0F85433C28CC3F3A5
:105F30000008038D5FFA88F7D51A0E46ADB2002F20
:105F40003FD1B2F5BF7F41D83DB103F12C012D33D4
:105F500001442A46184439F0D7FEA3681A8D134429
:105F600083F82C60002F73D1A268D38C01339BB2CD
:105F7000D384134483F82C80002D73D02046FFF780
:105F800093FB8288C3889A4222D1A268138D2C3356
:105F9000134408212046354AFFF70AFFE91B89B25E
:105FA00004F11000FFF7F4FDA268138D013313858F
:105FB0002046FFF767FB20B32069BDE8F041FFF7FB
:105FC00065BCB2F5BF7FC8D9002DC6D1BDE8F08150
:105FD000274A2649206901F048FAA268138D2C331C
:105FE00013440821214A2046FFF7E2FE214A1F49B7
:105FF000206901F03AFA20490122206901F035FABE
:10600000D2E72046FFF770FB0028DFD02046FFF7DD
:106010004BFBC2888388013AD21A92B2054604F13A
:1060200010061AB11549206901F01FFA2069FFF71F
:106030002DFCE988AB88C91A304689B2FFF7B2FD5A
:1060400029880139304689B2BDE8F041FFF716BD15
:10605000002D93D1A268D38C01339BB2D384134417
:1060600083F82C5032460649C7E700BF3731040099
:10607000C22F0400C52F0400E42F0400D82F040011
:1060800058270400F0B585B0826800250446CDE9A4
:106090000155ADF80C50D2F850630F46002946D197
:1060A000002E3FD0FFF788FDA0683B460A22D0F8BB
:1060B000500301A901F040FEA368029AC3F85023DF
:1060C000A068D0F85033C58C002B50D100F5D670A5
:1060D000FFF7C2FAA36838B303F5D67103F12C00B9
:1060E0003AF06CFBA0682C30FFF7B6FAADF80C0064
:1060F000A268BDF80C301385A268AB42D38402D2EB
:106100002069FFF7C9FBA3682D4A20462C330821DC
:10611000FFF74EFE2046FFF7B5FA00284AD0206967
:10612000FFF7B4FB05B0F0BD83F82C00DAE7D2F836
:106130004C33B342F6D0D2F84833002BF2D0FFF7FD
:106140003BFDA368D3F8500340BB03F12C00FFF7DD
:1061500083FAA368D3F84823C3F8502385B2A06814
:10616000CDB100F12C0100F5D6703AF027FBA06804
:1061700001A900230A22D0F8500301F0DDFDA06838
:10618000BDF80C2000F12C010A230132D0F8500395
:1061900001F0D2FDACE780F8AC51E8E72B460A22CB
:1061A00001A901F0C9FDA368019ABDF80C50C3F81C
:1061B0005023DCE72046FFF797FA0028AFD1B1E77C
:1061C0003731040038B504468068038DC58CED1A5C
:1061D000ADB2002D40D003F12D012C3301442A46ED
:1061E000184439F091FDA268D38C013BD38420463A
:1061F000FFF75AFA8288C3889A4215D1A268138D94
:106200002C3313442046154A0821FFF7D1FD54F8DA
:10621000100F1249124A01F028F9691E204689B26E
:10622000BDE83840FFF7B4BC0E4A0C49206901F0C4
:106230001CF92069FFF730FBA268138D2C3313443F
:106240002046064A0821FFF7B3FD2069064A0349A4
:10625000BDE8384001F009B938BD00BF373104004E
:10626000CC2F0400C22F0400C52F0400F0B5C36872
:106270005B6891B004460D46002203A9186801F03E
:10628000C6FE002840F093809DB1039801F03AFDCE
:10629000A268D2F844330133C2F84433A368D3F878
:1062A000443303F00703012B03D00125284611B026
:1062B000F0BD2046FFF7F8F981880129064605D987
:1062C000013989B204F11000FFF76CFC3188012913
:1062D00005D9013989B204F11000FFF759FC206992
:1062E000FFF7DAFA2DB1334A02212046FFF760FDAD
:1062F000DCE70023082204A9039801F01DFD069B9A
:106300000793BDF81430ADF82030BDF81630ADF865
:10631000223001238DF825309DF8103003F0030260
:10632000012A25D1BDF81050049E0398C3F3C2037F
:10633000C5F383158DF82430AA0008230AA901F0BB
:10634000FBFCC6F39526236900932A4607AB0AA9EE
:106350003046FBF78FFF039801F0D4FCE3685B68DD
:10636000002203A9186801F052FE0028C1D09CE762
:10637000022AF0D1BDF81250C3F3C203AD098DF863
:1063800024300827082D2E4628BF08263B463246D3
:106390000AA9039801F0D0FCAD1B236907AA314676
:1063A0000AA83744FBF7CAFF002DEBD1D3E700253D
:1063B0007CE700BF902F0400436801219868FFF735
:1063C00055BFF7B547680191BC68A3681E78042ED5
:1063D0000ED001A9386801F020FD054650B901989A
:1063E00001F08CFC032E03D129462046FFF73EFF27
:1063F00003B0F0BDF11E18BF01212046FFF736FFA4
:10640000E7E700002DE9F04F04468068A5B01021B1
:1064100000F55570FFF71BF8A3681B78022B40F0BE
:10642000DC8000230B9303936068036801221D69DD
:106430000DF12B010BABA8470B9B002B00F0B48098
:106440009DF92B30002BEFDB01F09CFCA3685A7800
:10645000012A00F0DD854BD3022A40F05186039AD1
:106460005A70A368D3F85423110740F19D809DF81A
:106470002B20313A1B2AD7D801A151F822F000BFB6
:10648000CB700000D9700000FB700000BD700000F0
:1064900029640000296400002964000029640000C8
:1064A00029640000296400002964000029640000B8
:1064B00029640000296400002964000029640000A8
:1064C0001D700000297000002D7000007B7000001E
:1064D00029640000C170000029640000CF70000032
:1064E000296400002964000029640000DD700000B8
:1064F0009DF82B500D2D38D00A2D36D0B3F85423EB
:106500006FF38D12A3F85423092D00F0358300F2A8
:106510001383002D88D0082D00F0138539F0BAFBC5
:106520009DF82B100844437813F0970F3FF47CAF8D
:10653000A368D3F854231507C2F3C00000F15B84AD
:10654000DA8CB2F5BF7F3FF66FAF1A8D551C1D85F3
:10655000134483F82C10A3681A8D134483F82C007D
:10656000A268D38C0133D3845EE7D3F8542312F4AA
:106570007F5F3FD0D3F85423C2F387129542C3D133
:10658000B3F8541362F38D11A3F85413A368DA8C93
:1065900092BBC3F850232069FFF778F9A368022261
:1065A0001A702046FFF73CFC00212046FFF75EFEF4
:1065B00098B12368BC4A03212046FFF7F9FBA36882
:1065C000D3F85423120708D520462C33B64A0821A5
:1065D000FFF7EEFB2046FFF71AFB206900F03AFFB9
:1065E000A0686FF0100100F55570FEF746FF25B06A
:1065F000BDE8F08F2A46C3E793F82C30002B40F01B
:106600008880A0682C30FFF727F8A368002687B29F
:10661000C3F850632FB3A368D3F848033D4600285E
:1066200000F0BC8033460A2217A901F085FBBDF8B3
:106630006430BB4240F0B280A0680A2300F5D671F6
:106640007A1CD0F8480301F077FBA06800F5D671FA
:106650002C303AF0A9F8A368002840F09D8083F818
:10666000AC01A0684FF4C072002100F5D67039F07B
:1066700064FBA068C28C00F12C0100F5D67039F0E3
:1066800038FBA66806F5D6763046FEF7E5FF3EB144
:106690004FF0000885B2C3466B1E9845C0F2C78014
:1066A000A06800F5D670FEF7D7FFA36801305885C3
:1066B0002046FFF7DFFA2046FEF7E4FF10B9206915
:1066C000FFF7E4F8A26817A92C320CA8FFF7ECF842
:1066D0000C9A0346002A3FF45EAF002840F0EE809B
:1066E000724F734EF61BF6080546AE42179B40F0FC
:1066F000EB80704A009202216F4A2046FFF758FB58
:106700004CE70135B5F5803F04D1002283F82C20F9
:1067100077E7002539F0BEFAA3685A19AEB292F8AD
:106720002C20104442781207EBD476B1DA8C03F1B6
:106730002C000132521B411939F0E6FAA268D38CC1
:106740009B1BD384A368DA8C1A85A568EB8C2B334A
:106750001D442F46B84639F09DFA98F80030184489
:10676000EE1B437813F00802B6B207F1FF37F1D100
:10677000A368D98C01F12B00184480453FF441AF48
:10678000891B0B4483F82C20A268D38C9E1BD684D3
:10679000A368DA8C1A8534E783F8AC6108270B35D7
:1067A00004EB07082946606901F079FA06460028DB
:1067B00037D0A368D3F84803C8B9C3F84863A368BF
:1067C000C3F84C63CDE91700A368DB8CADF86430E7
:1067D00017A9304600230A2201F0A3FAA168CA8C47
:1067E0000A2301322C31304601F09BFA39E70023AD
:1067F0000A2217A901F0A0FAA068189600230A221D
:1068000017A9D0F8480301F08CFA00231893A36865
:10681000D3F848231792DA8CADF86420C3F84863A4
:10682000D6E74046FEF7B4FF013FBBD119E739F088
:1068300031FA16F80810084408F1010341789AB2B9
:106840000F07029204D45F46DDF80880BB4623E7B9
:10685000029A4FF00009B1181FFA89FC0BEB0C07E4
:106860009C441FFA8CFC6545BFB2EDD9CDE90331DC
:1068700039F010FA0499039B11F809C0604401EB48
:10688000090E90F801A01AF0080A09F10109E3D1F4
:10689000002FD9D0ED1BA5EB08027146F01839F096
:1068A00033FAADB25746CFE737310400B47D040068
:1068B000FC7D04004B3004006D7B0400A84A0221DB
:1068C0002046FFF775FA69E67A681846116839F0CC
:1068D0006BFFB846083718B10135AE42BFF405AFBB
:1068E000A0680021102204300D9139F026FAD8F862
:1068F0000430DA6822B10FCBA568043585E80F00B3
:10690000D8F804304FF000089B680393CDF810804E
:106910000125C3460C9BAB4210D924AB03EB850683
:10692000904956F8340C39F03FFF00282FD1A26867
:10693000B2F8543343F00203A2F85433B8F1000F15
:106940000FD0A068428D00F5D6712C3039F0D1F906
:10695000A3685A8DDA84A26817A92C320CA8FEF716
:10696000A3FFA3681B69002B00F0E480049A04983D
:1069700017A901EB82020C99091A20469847A368CF
:10698000B3F854236FF34102A3F8542306E6764983
:1069900056F8340C39F008FF0028C8D056F8340CEB
:1069A000FEF75EFE002800F08B8056F8343C029320
:1069B00024AB002643F8586DB146059309F1010355
:1069C000079313AB00934A46059B03982946FEF7AD
:1069D0009DFE0E9BDBB1002219680298FEF797FC22
:1069E000002867D10E9B1B6806931846FEF734FEFD
:1069F000A26883B21F460893538D01333B44B3F51D
:106A0000C07F37D9594A04212046FFF7D1F9002E1B
:106A100094D0A068029900F5D67039F006FF0746B9
:106A20000298FEF719FE07B3A36803F5D6739F42D9
:106A30001FFA80F909D917F8013C202B02BF09F190
:106A400001091FFA89F907F1FF373846FEF704FEFE
:106A5000A268538DA3EB09035385421CA2EB0902E4
:106A600007EB0901384639F04FF9B04401355F466C
:106A7000BB464FE7029902F5D67039F0D6FE824642
:106A80000028C4D0FEF7E8FD82B2781C01325146DE
:106A9000504439F039F93A460699504639F029F907
:106AA00020230AF80730A2680899538D013319444E
:106AB00051850136B9F1FF3FA9D0DDF81C907DE783
:106AC0000FAB0BF1010700935A460DAB2946039813
:106AD000FEF71CFE002F3FF431AF0D9B002B3FF45F
:106AE0002DAF196856F8340C39F05EFE0028BFD17E
:106AF0000D9EF368CBB1B8F1000F0FD02046FFF721
:106B0000B9F82046FEF7BEFD10B92069FEF7BEFEBB
:106B1000174A02212046FFF74BF930E796E80F00AD
:106B2000A7680495043787E80F00B368039301351D
:106B300000279DE70F4AECE71B2D0CD07F2D7FF43B
:106B4000EDACA368D3F854331E077FF56DAC204637
:106B5000FFF738FB68E4A36801225A7064E400BFC1
:106B6000373004005F3004006230040069300400F4
:106B7000B7300400E6300400A068D0F854331D0795
:106B80007FF552ACC38CC3F5BF7301331FFA83FA90
:106B9000BAF1000F3FF448AC00F12C01028D00F572
:106BA000D67039F0A6F8A3681A8D1344039A83F8B7
:106BB000AC2139F06FF8A3681A8D1A4492F82B2093
:106BC0001044427802F00801C2F3C0020792039A0F
:106BD000C3F85023A268089102F5D67217A90CA831
:106BE000FEF762FE1798FEF737FD0023CDE90D335F
:106BF00087B21E4604931D4602939B4605930C9B49
:106C00002BB1079A013B1344AB4200F2C580089BAD
:106C1000002B36D124AB03EB850353F8340CFEF77D
:106C20001BFD87B224AB03EB85034FF000090993EA
:106C300009F1010306930FAB00934A460DAB2946B9
:106C40003046FEF763FD0D9B002B59D01968099B58
:106C50003A4653F8340C39F0C1FD8046A8B9029B7E
:106C6000013302930D9B18680E9B8BB9FEF7F4FC61
:106C700083B2D81B8245049301DD1FFA80FACB460C
:106C800031E00027CEE7CDF81490DDF81890CFE77B
:106C9000FEF7E2FC049B80B2834238BF03460493B4
:106CA000BAF1000F1FD013AB009330460EAB059A1C
:106CB0002946FEF72BFD0D9B18680E9BD3F800C0EC
:106CC00007EB08021FFA88F1835C1BB98A4528BFCD
:106CD0008A4608E01CF802209A42F7D108F1010820
:106CE000B8F5803FECD10D9B0E93069B002BCAD1CB
:106CF000B54A04212046FFF75BF84FF0FF330593B8
:106D00004EB10D9B3BB10C9B079A0135ADB21344BC
:106D10009D42FFF474AF029B002B3FF485AB012B27
:106D200040F08C8033783BB10FAB0093059A0EABEB
:106D300029463046FEF7EAFC0E9B1868FEF78CFCED
:106D4000B84206D00E9B1968524639442046FFF7D8
:106D50009DF838F09FFFA368198D5A1892F82C20DF
:106D60001044427812F008024AD1D3F85413C907EC
:106D700040D5B3F8541362F30001A3F8541320462E
:106D80002021FFF7CDF8A268B2F8543343F0010395
:106D9000A2F85433FFF748BB24AB4FF0000803EBD5
:106DA00085090FAB009342460DAB29463046FEF7EE
:106DB000ADFCB8F1FF3F06D1834A04212046FEF71F
:106DC000F7FFFFF731BB0D9B002B3FF42DAB59F8BC
:106DD000340CFEF745FC002892D10D9B59F8340C79
:106DE000196839F0E1FC08F101080028D9D10D9BA0
:106DF0009E6885E720212046FFF792F8FFF714BB35
:106E0000DB8C8B427FF610AB2046FEF74DFCA26870
:106E10008588138D013313852046FEF745FC838852
:106E2000AB4206D169490122206900F01EFBFFF741
:106E3000FBBA2069FEF72AFDFFF7F6BAA368039AAA
:106E40009A8424AB03EB8503DFF8949107930BF14D
:106E5000010305930FAB00935A460DAB294630460C
:106E6000FEF754FC0D9B1968079B3A4653F8340C07
:106E700039F0B4FC30BB029B013B02930D9BD3F86D
:106E800000B0BBF1000F20D1A368A3F824B0029B8F
:106E9000C3B923684E4A20460321FEF789FFA36841
:106EA0004C4A2C3308212046FEF782FF2046FEF78D
:106EB000AEFE0E9B1968524639442046FEF7E6FFA7
:106EC000FFF7B2BADDF814B0C1E74846FEF7C4FBDD
:106ED000049BA268184483B24846B2F81E80069309
:106EE000FEF7BAFB08905846FEF7B6FB069B181A49
:106EF00082B2A0680692089A818CA8EB0208B8FBBF
:106F0000F3F39BB2B1FBF3F203FB121301F1010C9B
:106F10009BB2A0F824C06BB9CDF800B04B462E4A06
:106F200007212046FEF744FF069904F11000FEF702
:106F3000A5FDACE75B46274A07212046FEF738FF50
:106F4000F2E7A068D0F854331F077FF56DAAC68C0E
:106F5000002E3FF469AA038D002B3FF465AAF61AB0
:106F600003F12C01B6B22B33721C0144184438F0E3
:106F7000CBFEA268138D013B1385A268D38C013B25
:106F8000D384002E42D02A461449206900F06DFABD
:106F90002046FEF789FB8288C3889A4222D1A268E4
:106FA000138D29462C33254613442046094AFEF703
:106FB000FFFE55F8100FFEF76FFC31462846FEF72E
:106FC000E7FDFFF731BA00BF04310400E42F0400ED
:106FD00036310400373104003031040058270400F2
:106FE00015580400474A4849206900F03EFA2069D4
:106FF000FEF752FCA268138D2C3313442946424AF3
:107000002046FEF7D5FE414A3F490DE7404AFBE7DF
:107010009DF82B205B2A73D102229EE50121204698
:10702000FFF730F8FFF700BA0021F8E72046FEF737
:107030003BFB038842889A42054604D18188C28876
:1070400091423FF4F1A96A899A424FF001020FD1AF
:107050002646304956F8100F00F007FA6989304685
:10706000FEF796FDA268138D01331385FFF7DCB997
:107070002949206900F0F9F9F4E72046FEF714FBEE
:10708000037B028801339A42054603D18388012B92
:107090003FF4CAA9012A20690BD1204900F0E5F983
:1070A000698904F11000FEF7E9FCA268138D013B29
:1070B000DBE701221A4900F0D8F9F6E703225A70FB
:1070C0002046FEF7D7FDFFF7AFB903225A702046DE
:1070D000FEF772FDFFF7A8B903225A70A268D2F832
:1070E0005433B2F8541303F0010383F0010363F344
:1070F0000001A2F85413FFF797B903225A7020E554
:10710000039A2AE5C22F040037310400C52F04007A
:10711000D02F0400D82F0400E42F0400EA2F04002D
:10712000DE2F04002DE9F04F044689B07F48DFF8D8
:10713000209217460E4639F049FB05467C4839F047
:1071400045FBA368CDF800907A4A5B6808212D1AA8
:107150002046FEF72DFEA3685868FEF77DFA8046AC
:10716000484639F033FBA36808EB000292B29968F5
:107170002046FEF78DFC704A00212046ADB2FEF796
:1071800017FE3FB136B14FF00C09B04609FB076955
:10719000C14527D1664839F019FB02300544ADB22C
:1071A000624B009305F10308644A082120462B46F0
:1071B0001FFA88F8FEF7FCFD424661492046FEF7BB
:1071C00067FC36B10C23DFF8749103FB0767BE42FE
:1071D00022D1A368D3F80C90B9F1000F59D109B0AE
:1071E000BDE8F08FD8F80400FEF736FA8246D8F8EA
:1071F0000000FEF731FA5044A8420AD9D8F804003A
:10720000FEF72AFA0546D8F80000FEF725FA0544ED
:10721000ADB208F10C08BBE7D6E900238BB342B34B
:107220000192434A00920821464A2046FEF7C0FDDB
:107230007068FEF711FA83463068FEF70DFA824651
:107240003B4839F0C3FA0BEB0A01691A091A89B2F3
:1072500004F11000FEF712FC3A223B49206900F0CD
:1072600004F9B16889B142462046FEF711FC0C369C
:10727000ADE700932B464A4608212046FEF798FDCD
:10728000EFE7002AEDD00092F4E72069FEF7FEFA5E
:10729000EDE70DF12008002248F8142D164604AF42
:1072A000009743460121484602F1010AFEF72EFAF3
:1072B000039D5DB12868FEF7CFF9B04204D9039B66
:1072C0001868FEF7C9F986B25246E9E7BAF1010F2C
:1072D00085D01E4A29462046FEF76AFD06F1020ABD
:1072E0002A46164D1FFA8AFA43460097012148465E
:1072F00002F1010BFEF70AFA039B002B3FF46FAF7C
:107300001B680093082153462A462046FEF750FD8D
:10731000039B596831B1721D92B22046FEF7B8FB4B
:107320005A46E1E72069FEF7B1FAF9E7F02F0400C9
:107330004C31040031310400FB2F040005300400FF
:107340000D300400203004005827040029300400C8
:10735000D42F040041680A6042685360014B1860F2
:1073600000207047F410002000207047002914BF4F
:107370000620002070470000F8B5114C114F124D47
:107380000646204600F03CFE20B93B685B68D3E926
:107390000021904740220C490C48FDF74BF940B9B9
:1073A0003046FDF742F929460246204600F0BEFE6F
:1073B000E7E7922803D0BDE8F840FBF7C3BDF8BD6E
:1073C000607D0400F41000202410002050310400DF
:1073D00010B503481C4600F08BFD2060002010BD56
:1073E000607D040038B508481C461546FDF7FCF8DA
:1073F00030F0080302D12560184638BD112804BFBB
:1074000000202060F9E700BF5031040010B50446A9
:10741000032918D8DFE801F00B0212020A4B1B689F
:107420005B680120D3E90021BDE810401047FDF75B
:10743000FCF806490246064800F078FE2046BDE802
:107440001040FFF799BF10BDF41000202410002059
:10745000607D040010B5826804462AB14369016862
:10746000006998470023A36010BD0EB403B50399CB
:1074700029B102AA04AB42F8043D00F073F802B04F
:107480005DF804EB03B070470A2938B504460D4691
:1074900002D10D21FFF7F8FFA3682268591CA160F3
:1074A000D554D4E901329A4204D32046BDE838408D
:1074B000FFF7D0BF38BD00002DE9F84F9946DDE950
:1074C0000A431746824688460A460126BA420FD228
:1074D0004E4538BF4E4613F0010B01D164B900246C
:1074E0000125B9F1010F1AD909F1FF397D43F8E7F8
:1074F000B2FBF7F20136E9E79B070ED5B9F1000FB1
:107500000CBF30252025A642EAD2013C2946504630
:10751000FFF7BAFF002CF6D1E1E72025F3E7B8FB2F
:10752000F5F39F42E2D9DFF83890B8FBF5F3504607
:1075300019F8031005FB1388FFF7A6FFB5FBF7F555
:10754000002DF2D1BBF1000F02D00CB1A64201D345
:10755000BDE8F88F20215046013CFFF795FFF4E786
:10756000A23104002DE9F74F054690460E4600294A
:1075700000F03A8116F8011B002958D0252940F067
:10758000D180002702E047F001071646324612F884
:10759000013B2D2BF7D0302B04D02B2B05D147F0FE
:1075A0000407F2E747F00207EFE700242A2B06F171
:1075B00001021BD1D8F80030191DC8F800101B6853
:1075C00016461C4433782E2B1CD101364FF0000A8E
:1075D000314611F8012BA2F13000092814D80A23F2
:1075E00003FB0A23A3F1300A0E46F1E712F8013C2F
:1075F000A3F130010929E5D80A2101FB0434303C0C
:107600001646D3E74FF0000A324612F8011B01F08C
:10761000FB0068281646F8D0692916D054D8582996
:1076200070D00ED825297DD03378002BA2D12B7BAA
:10763000002B00F0D980284603B0BDE8F04FFFF7DB
:1076400009BF632968D06429EED1D8F80020111D44
:10765000C8F80010D2F8009089EAE972A2EBE9724A
:107660004FF0010B092A61DCD34538BFD3462CB15A
:10767000B9F1000F01DB790700D5013CBA0702D54B
:10768000BAF1000F04D0FB0702D4002C54D100241F
:10769000B9F1000F58DAC9F100092D212846FFF78A
:1076A000F3FE07F00302022A05D1BAF1000F02D15E
:1076B000002C4DD10024CDE9004753460A2249460B
:1076C0002846FFF7F9FEAFE7732954D016D8702982
:1076D000AAD1D8F800301A1DC8F800203021284659
:1076E0001C68FFF7D1FE78212846FFF7CDFE002267
:1076F0000823CDE9003221461022E1E775292FD079
:10770000782991D1D8F800100A1DC8F80020CDE9D9
:107710000047534610222CE0D8F800301A1DC8F854
:10772000002019782846FFF7AFFE7DE70A230BF10A
:10773000010B92FBF3F295E7A345A9D2202128463D
:10774000013CFFF7A1FEA0E77807AAD52B21A5E70A
:10775000A345B0D230212846013CFFF795FEA7E7AC
:10776000D8F80010CDE900470A1DC8F8002053469C
:107770000A220968A4E7D8F800301A1DC8F80020CA
:10778000F907D3F8009012D54F46A7EB090B17F86D
:10779000011B41B9A345BFF447AF20212846013C56
:1077A000FFF772FEF6E72846FFF76EFEEDE7B9F148
:1077B000000F17D0484639F009F80746BC4200D9F7
:1077C00054B909F1FF3919F8011F00293FF42CAF12
:1077D0002846FFF759FEF6E720212846013CFFF72F
:1077E00053FEEBE74F46E9E703B0BDE8F08F00003A
:1077F00007B50B46A0B9154B5B886BB1144B154808
:10780000154AC01A0E23C0080093144B00041449F3
:1078100040F00100FAF7FAFB0E2003B05DF804FB1C
:107820006BB90A4B5B88002BF6D0094B09480D4A0F
:10783000C01AC0080E2300930004084BE7E703605A
:107840001B68114603B05DF804EB18474C05002097
:107850000C7E0400CC7E04005F320400B2310400D0
:1078600064320400DB3204002DE9F3419646B0B9DE
:10787000504B5B88002B00F095804F4B4F48504A8F
:10788000C01AC0080E244F4B009400044E4940F02B
:107890000100FAF7BBFB204602B0BDE8F0816AB9EF
:1078A000444B5B88002B7DD0434B4448474AC01A69
:1078B000C0080E2400040094424BE7E7D0F800C053
:1078C000BCF1000F0DD13B4B5B88002B6CD03A4BC9
:1078D0003A483F4AC01AC008082400040094394BB3
:1078E000D4E76BB9334B5B88002B5FD0324B334806
:1078F000384AC01AC008092400040094314BC5E777
:107900004768D7F80480B3FBF8F708FB17376FB167
:10791000284B5B88002B49D0274B28482E4AC01A99
:10792000C008092400040094264BAFE78F070DD050
:10793000204B5B88002B3BD01F4B2048274AC01AA6
:10794000C0081024000400941E4B9FE712F0030FA0
:107950000CD0184B5B885BB3174B1848204AC01AF1
:10796000C008102400040094164B8FE7C768B94282
:107970000BD34C1E05691C44AC4206D8DCF80C4005
:10798000A44602B0BDE8F04160470A4B5B887BB17A
:10799000094B0A48134AC01AC00810240004009476
:1079A000084B73E70E2476E7082474E7092472E78E
:1079B000102470E74C0500200C7E0400CC7E0400EF
:1079C0005F320400C431040064320400E132040078
:1079D000D532040094320400E7320400113304006D
:1079E000293304004C330400F7B5A0B9374B5B884A
:1079F000002B63D0364B3748374AC01AC0080E24D4
:107A0000364B00940004364940F00100FAF7FEFAC4
:107A1000204603B0F0BDD0F800C0BCF1000F0DD17E
:107A20002A4B5B88002B4BD0294B2A482D4AC01A81
:107A3000C008082400040094284BE4E76AB9234BEB
:107A40005B88002B3ED0224B2248274AC01AC00830
:107A5000092400040094214BD5E74768D7F800E0DB
:107A60000EF1FF370F420CD0184B5B8863B3184BF5
:107A700018481E4AC01AC008102400040094174B6E
:107A8000C1E7C768B9420CD34C1E05690EFB02441E
:107A9000AC4206D8DCF81040A44603B0BDE8F04084
:107AA00060470A4B5B887BB1094B0A48104AC01AF1
:107AB000C008102400040094084BA4E70E24A7E794
:107AC0000824A5E70924A3E71024A1E74C0500201A
:107AD0000C7E0400CC7E04005F320400D731040029
:107AE00064320400D532040094320400EA31040008
:107AF00010320400014B43600020704780330400C3
:107B00000846704700207047024B1868003018BFC5
:107B1000012070478011002008B50248FDF7D7FC0E
:107B2000002008BD8011002008B510461A4638F024
:107B3000E0F8002008BD00002DE9F041804686B045
:107B400013480E4615461F46FDF7B8FC044630B1F3
:107B5000112018E006EB043000F006FD0134A542C8
:107B6000F8D10B48FDF7B3FCD8F8083000246BB10E
:107B7000022268468DF80020CDE90146CDE9034593
:107B800005979847204606B0BDE8F0811846FAE709
:107B9000801100202DE9F041804686B012480F4642
:107BA00016461D46FDF78AFC0446D8B9AA08314698
:107BB000384600F0F1FC0C48FDF789FCD8F8083095
:107BC00073B101228DF800200C9A05926846CDE928
:107BD0000147CDE903659847204606B0BDE8F0812E
:107BE0001846FAE71120F8E7801100202DE9F04748
:107BF000B0F806904479D2F800A09DF8208009FBE7
:107C000004F4043C06460AEB0300A0420F4688BF7A
:107C1000A4EB030A191DC2F800A0B1FBF9F509FB9A
:107C200015114DB9A9EB0104544528BF5446BAF1CA
:107C3000000F04D1BDE8F0873668013DF1E704315B
:107C40007B1970182246B8F1000F0ED00146184675
:107C5000AAEB040A38F04DF8D145254436684C4665
:107C60004FF0000128BF5446E1E71946F0E7FDF761
:107C700089BCF8B546790146721E05460023934239
:107C80002D6803D30024A64202D8F8BD0133F6E7DD
:107C90000F682846FDF7AFFC01343946F3E72DE9BC
:107CA000F843CD1C068B0746FDF783FC043E3544A4
:107CB0000446B5FBF6F5F0B14FF48073EDB2838066
:107CC000C680013D076081464FF00008A84512D2EA
:107CD0003846FDF76EFC064648B16379013363719F
:107CE00008F10108C9F8000007608146EEE7204668
:107CF000FFF7BFFF34462046BDE8F883012104307A
:107D0000FDF7C6BB10B5012104460430FDF7CBFBDF
:107D100010F0FF0F04D12046BDE81040FFF7A9BFC7
:107D200010BD1FB504AC44F8042D00220092224679
:107D3000FFF75CFF04B010BD1FB504AC44F8042D80
:107D4000012200922246FFF751FF04B010BD00004F
:107D500008B50020FDF746F8F1EE103A23F09F0336
:107D6000E1EE103ABFF35F8F054B4022C3F8842148
:107D70000020FDF739F820BF40BF20BF08BD00BF7D
:107D800000E100E07047026813685268934291BFB7
:107D9000D01A80680130801888BFC01A70472DE95A
:107DA000F04103681F681D685B689D4284BF83685B
:107DB0000133164688465D1BC2684168AE420446E0
:107DC00007FB02110CD87243404637F092FFA368BC
:107DD0003E449E4288BF002623681E60BDE8F081B5
:107DE00005FB02F73A46404637F083FFE2686168D8
:107DF000751B6A4308EB070037F07BFF23681D60A3
:107E0000ECE7036881681A685B688B4234BF013312
:107E10000023D31A584258417047F8B50446002051
:107E20000D46FCF7DFFF2046FFF7EBFF10B1237C88
:107E3000002B3DD12168A6684B684A68B24234BF26
:107E4000013200224A6038B12168A0680A68824283
:107E500034BF013200220A60E2686068511E0729BF
:107E600020D8DFE801F004101F141F1F1F182A7804
:107E7000C2542046FFF787FF23689A68824200D2E7
:107E80009860002415E02A8820F81320F1E72A687A
:107E900040F82320EDE7D5E9006700EBC300C0E917
:107EA0000067E6E7294602FB030037F022FFE0E720
:107EB00004240020FCF798FF2046F8BD70B5054665
:107EC0000E46144682B10020FCF78CFF2846FFF7CF
:107ED0005AFFA0420AD3224631462846FFF75FFFE9
:107EE00000240020FCF780FF204670BD0524F8E741
:107EF00070B505460E46144682B10020FCF772FFAD
:107F00002846FFF740FF844228BF04462246284601
:107F10003146FFF744FF0020FCF766FF204670BDA6
:107F200010B504460020FCF75DFF2046FFF72BFF4D
:107F300004460020FCF758FF204610BD2DE9F04F05
:107F40008368D3F854339B078BB0064606D50022CE
:107F500011460BB0BDE8F04FFFF7E4B8012906D990
:107F6000214A02210BB0BDE8F04FFDF721BF1F4CA5
:107F70001F4D204FDFF88080DFF880901C232D1BE1
:107F8000B5FBF3F503FB0545AC4202D10BB0BDE8F0
:107F9000F08FE36809932368D4F808A0D3F808B0F9
:107FA0002046FFF7BDFF94F810C0642303FB00F1E7
:107FB000BCF1000F0CBF3A46424603FB0BF3B3FB88
:107FC000FAF3CDE9043BB1FBFAF1099B0191CDE94C
:107FD00006A2CDE9020A00934A46636908213046A9
:107FE000FDF7E6FE1C34CFE7942E0400607D04000C
:107FF000B47D0400F0330400F933040005340400B8
:10800000036818685B68C31A58425841704770B5D6
:10801000054600200C461646FCF7E4FE2846FFF70E
:10802000EFFF002830D129680B682EB90A68A868CC
:10803000824238BF561C0E60EA686968501E0728E5
:108040001CD8DFE800F0040C1B101B1B1B14CB5CBE
:10805000237000240020FCF7C7FE204670BD31F8D5
:1080600013302380F5E751F823302360F1E701EB6B
:10807000C301D1E90023C4E90023EAE703FB0211AD
:10808000204637F036FEE4E70524E3E710B58468C0
:10809000FFF746FF201A10BD2DE9F84304461646A7
:1080A0008846FFF7F3FF23681A685D68AA429CBF01
:1080B000A2680132551B8146E26858686368AE4287
:1080C00002FB003017D87243414637F012FE226897
:1080D000A168536833448B4296BF53680026F61854
:1080E00056602046FFF74FFE23689A68824238BFE9
:1080F0009860BDE8F88305FB02F73A46414637F041
:10810000F8FDE2686068751B6A4308EB070137F009
:10811000F0FD2368B1455D60E3D22268A168536831
:108120008B4234BF013300231360DAE770B5054694
:108130000E46144682B10020FCF754FE2B7C6BB92E
:10814000AB689C4228BF1C46284622463146FFF7B2
:10815000A3FF0020FCF748FE204670BD2846FFF72D
:1081600095FF844228BF0446EEE7826800239360AF
:1081700082681361826853618268D3608268536049
:10818000826813607047F8B505460F4616461C46D0
:1081900083B9AB686868D3E9031300F1010CCA1A0C
:1081A00062450ED10027376014B3A868FDF78FF938
:1081B0000020F8BD8068FDF781F90028E9D0112082
:1081C000F7E701EA00021840824236BF6344ACEB95
:1081D00002035B1A3168994294BF316033602B68A7
:1081E00013443B60AA683168D3680B44D360DFE76F
:1081F0002046DEE738B5846843682569A268013304
:108200002B449B1A8B420CD30A44A26083689A6861
:10821000DA608068FDF758F900280CBF08200020BC
:1082200038BD0420FCE710B5826813699468E41A2D
:108230008C420AD30B44136183681A695A618068BF
:108240000430FDF744F9002010BD0420FCE770B5B0
:10825000446806460D46206818B1B3682946984719
:1082600018B923682B60256070BD2468F3E7436864
:10827000186808B102681A60704743681868704748
:108280004368186800B970478842026802D11A60D2
:108290000120704703461046F4E7000038B5084C4B
:1082A00004F108030546002818BF1C4623682BB1BB
:1082B0001A6822605B6828469847F7E738BD00BF18
:1082C0008C11002020B9054B01225A70FFF7E6BF40
:1082D000012802D1014A9070F8E77047841100200C
:1082E00038B5094C23786BB908486360A3602361F3
:1082F000E36000F07DF9054600F088F90123237062
:10830000284638BD8525FBE784110020C582000082
:1083100038B5134CA378054603F0FF0073B115B1CF
:108320006B68012098470020FCF75CFDE36801338F
:10833000E3600020BDE83840FCF756BDFCF752FD75
:1083400025B1226913463BB92A602561E368002BF9
:10835000ECD100F071F9E9E79D42F7D01B68F2E734
:108360008411002038B5134C6378054603F0FF00F4
:1083700073B115B16B68002098470020FCF732FDFF
:108380006368013363600020BDE83840FCF72CBD12
:10839000FCF728FD25B1A26813463BB92A60A56009
:1083A0006368002BECD100F059F9E9E79D42F7D062
:1083B0001B68F2E78411002038B5084C0020FCF758
:1083C00011FD6368013B6360656815B900F058F9F9
:1083D00065700020BDE83840FCF706BD8411002020
:1083E00010B5074C23784BB9064B002808BF184638
:1083F00000F0A0FA08B90123237010BD8520FCE726
:1084000098110020B134040008B500F0C6FABDE8A8
:10841000084000F0C9BA10B50446FFF7F5FF204642
:1084200000F0AAFA00F0B2FA002010BD07B502A9C8
:1084300001F8010D0548FFF7F0FC0448FFF7E1FCE7
:1084400008B100F055FB03B05DF804FB7C7D04002F
:1084500038B50C4D2B7893B90B4B0C49002808BF4D
:1084600018460388284620F8013F00F001FB044627
:1084700018B900F02BFB01232B70204638BD852452
:10848000FBE700BFE8110020B23404002D84000097
:1084900010B504460248FFF743FD207010BD00BF31
:1084A0007C7D040010B50A4601460448FFF706FD2E
:1084B000044600F00BFB204610BD00BF7C7D04008D
:1084C000074A084B1360084A03F110011160074A7C
:1084D00003F120011160064A0120C2F804357047FB
:1084E00024120020F4110020F0110020EC110020D3
:1084F00000E0004010B5114B04461868884202D0D5
:10850000102237F0F6FB0E4B0022C3F800210122A7
:108510001A604FF08070D3F8002162B10022C3F8D6
:108520000021084B1968A14203D01022204637F0E1
:10853000E0FB012001E00138EDD110BDF011002079
:1085400000E00040EC110020024B014610221868A8
:1085500037F0CFBB24120020024AD2F80034002B9F
:10856000FBD0704700E001400A4908B50223C1F87A
:108570000435BFF36F8FBFF34F8FC1F80805FFF7C6
:10858000EBFF0023C1F80435BFF36F8FBFF34F8FAC
:1085900008BD00BF00E001400E4B10B50124C3F838
:1085A0000445BFF36F8FBFF34F8F01EB8204401A76
:1085B000A14208D1074B0022C3F80425BFF36F8FF7
:1085C000BFF34F8F10BD431851F8042B1A60FFF70B
:1085D000C3FFEDE700E0014050E8002F02EA01038D
:1085E00040E8003C9CF0000FF6D1104670470000B8
:1085F000054A13792BB90121106011715371184686
:1086000070478520704700BF28120020084B1A6869
:10861000D2075FBFC02283F8002301221A604FF007
:1086200080420123C2F81835024A1370704700BF18
:1086300000E100E069870020074B00221A6082B049
:108640001B680193019B4FF080430222C3F804236F
:1086500001229A6002B0704704010040074B0022DB
:108660001A6082B01B680193019B4FF08043012286
:10867000C3F804231A6002B0704700BF0001004035
:10868000074B01221A604FF08042D2F80C3403F0FD
:108690000113B3F1011FF8D0024B00225A71704749
:1086A000040000402812002007B5154B1A687AB163
:1086B00000221A601B680093009B4FF08043012248
:1086C000C3F808230F4B587910B95A711B689847A3
:1086D0000D4B1A6882B100221A601B680193019B3E
:1086E0004FF080430222C3F80823064B1B68012089
:1086F00003B05DF804EB184703B05DF804FB00BF5E
:1087000000010040281200200401004000F18040D8
:1087100000F5C040002382B0036003680193019B11
:1087200002B0704703681F2B83BF03F01F03036071
:1087300001484FF0A04070470003005007B502AB5E
:1087400043F8040D1846FFF7EDFF019B00EB830093
:10875000D0F8003723F44033C0F80037D0F80037A2
:1087600043EA0141C0F8001703B05DF804FB0000C4
:108770002DE9F04F002489B0CDE902445F4A604EF4
:10878000604D01211368A2F5C040012B80B206D1D3
:10879000D6F804330B4202D0FFF7B8FF0C43043283
:1087A000AA424FEA4101EDD1574B1B68012B0ED174
:1087B0004FF4BE70FFF7AAFF4FF0A04344F000440F
:1087C000D3F810350293514BD3F81035039314F0BE
:1087D000FF0F1AD04E4F00250126344210D0AB00B7
:1087E00003F1804303F5C043D3F81005D3F8101507
:1087F00057F82530C0F30520C1F3014103B1984774
:108800000135082D4FEA4606E7D1002C72DA04AE96
:108810000023049373604FF0FF33CDE906333C4FE0
:108820004FF0010800252C467B1993F96020531C5A
:1088300047D0D2B222F0C00908A84FEAD90300EB12
:10884000030B02F007011BF8080C08FA01F10842BB
:1088500037D007EB0900920990F9300057F820A0B3
:10886000BAF1000F05D1032A2BD1F05C0843F05474
:1088700001E0032AF9D001A8CDF80490FFF752FFD8
:10888000019B03F5E07350F823301BF8180C0842E5
:10889000C3F3014305D0022B13D1032A0BD1114698
:1088A00004E0032B0DD1032A05D102214846FFF72E
:1088B00045FF0134E4B2BAF1000F02D01146484638
:1088C000D0470135042DAFD1A4B14FF0A043029998
:1088D000D3F8102503F540739142D3F8103502D137
:1088E0000399994206D002920393049A059B06923B
:1088F000079397E709B0BDE8F08F00BF0061004023
:1089000000600040206100407C6100400003005096
:108910003012002000F1804382B01A68002A14BF90
:108920000120002004D000221A601B680193019BE3
:1089300002B070470E4B1A78C2B902784FF08041EE
:10894000C2F34002C1F88025027802F00102C1F8AA
:108950007825084A1168C9075FBFC02182F8001353
:108960000121116001221A70002070478520704794
:108970006A87002000E100E0034B00221A600268D1
:1089800002B11A60704700BFA41200204FF080436C
:108990004FF46072C3F8042370474FF080434FF4E4
:1089A0006072C3F808237047014B00221A607047B9
:1089B000A412002010B54FF08043D3F8044362079F
:1089C00007D54FF48470FFF7A5FF10B11E4B1B684D
:1089D0009847A30608D54FF48A70FFF79BFF18B19C
:1089E0001A4B00201B689847600608D54FF48C701E
:1089F000FFF790FF18B1154B01201B68984721061F
:108A000008D54FF48E70FFF785FF18B1104B00208A
:108A10001B689847E20508D54FF49070FFF77AFF7E
:108A200018B10B4B01201B689847A3050AD54FF4DA
:108A30009270FFF76FFF28B1054B02201B68BDE85D
:108A40001040184710BD00BF9C120020A01200204B
:108A5000A412002008B5FFF7ADFFBDE80840FFF7FE
:108A600023BE0000014B1B68184700BFA81200205E
:108A700010B5124C2278FAB9114B1960037813F033
:108A8000010F104B1EBFD3F8042542F00102C3F8BA
:108A90000425D3F8002222F00102C3F80022437813
:108AA000094A5B01DBB282F80D334FF400531360C7
:108AB00001232370002010BD8520FCE7B4120020A4
:108AC000B012002000D0004000E100E0064B002280
:108AD0001A6082B01B680193019B044B0122C3F80A
:108AE00004231A6002B0704700D1004000D000405B
:108AF000024A0123C2F808335360704700D0004097
:108B0000074B00221A6082B01B680193019B054B42
:108B1000D3F80805044B1B68C0B202B0184700BF69
:108B200000D1004000D00040B0120020044A9168FB
:108B30009368CB1A23F07F438342F9D3704700BF79
:108B400010E000E0034B044A1B68B3FBF2F3584308
:108B5000FFF7ECBF3401002040420F00F7B5057964
:108B6000314C0C266E43A7193B7A002B5AD1A251E7
:108B70004A687A609C46467902685F1CDBB29E4276
:108B800046D8120B53B2CE78284F002BAEBF03F15C
:108B9000604302F00F02264B4FEA4616F6B2AABF18
:108BA00003F561439E5483F8006303681B0B5EB2B8
:108BB0007609012203F01F0302FA03F347F8263077
:108BC00007684B78D7F8046503F0030326F0030623
:108BD0003343C7F8043507688B78D7F8086503F086
:108BE000030326F003063343C7F8083506680B78FD
:108BF000D6F8100503F00F0320F00F010B43C6F861
:108C000010350C2303FB05440020227203B0F0BD95
:108C10009B0003F5A07342F803C0D3580193019B56
:108C20003B46A8E70820F1E7B812002000E100E089
:108C300014ED00E0036801221A600379034A0C2155
:108C400001FB032302221A72704700BFB8120020F2
:108C50000368044901221A6103790C2000FB031305
:108C60001A727047B812002038B503681B0B5AB24D
:108C70000121520903F01F0301FA03F320320C49CA
:108C800041F8223003680025D3F80022C3F80052CF
:108C900003684FF0FF320446C3F80823FFF7D8FFFC
:108CA0002379044A0C2101FB03231D7238BD00BF48
:108CB00000E100E0B81200200379044A0C2101FB16
:108CC0000323187A831E584258417047B812002077
:108CD00010B58B0040330268DBB20124D45001F59B
:108CE000A871036853F8210010BD73B54FF48034A8
:108CF0008C4005688BB18B0003F5A0730026EE5005
:108D0000EB580193019B0368C3F80443036801F522
:108D1000A87143F8212002B070BDC5F80843F5E7FB
:108D2000F0B407689DF810C0D7F8004240F2011572
:108D30008D4024EA0504C7F800420568D5F80042D2
:108D40002343C5F80032F0BC6346FFF7CEBF0000F6
:108D5000F7B5104E104F114D0024A3199B001A684F
:108D600092B1D7F804134FF48032A2400A420BD0DC
:108D700000221A601B68019304F150008000019BDF
:108D800080B2D5E9003198470134062CE5D103B013
:108D9000F0BD00BF5068001000A00140B8120020D4
:108DA00000F1804000F51C3001230360BFF36F8F9A
:108DB000BFF34F8F70470000064A10F0800F00F09D
:108DC0000F0314BFD2F81005D2F81405D84000F0F4
:108DD0000100704700700240054B1B68082B01BF63
:108DE000044B1868B0FA80F0400918BF00207047A3
:108DF000300100103401001030B54C68A34209D98D
:108E0000002545600968016093420CD1201C18BF01
:108E1000012030BD43600D6805600868E41A1844FD
:108E20004C600860F0E70020F3E74B689A4228BFE7
:108E30001A460B68C0E9003248680B68801A48601F
:108E40001A4400300A6018BF012070474B689A42EC
:108E500028BF1A4662B10B68C0E900324B689B1A02
:108E60004B600B68101C13440B6018BF0120704747
:108E70001346F1E7054B10F0800FA3F1900208BFF5
:108E8000134600F00F0003EB001070476013002042
:108E900010F0800F14BF0023102300F00F001844BF
:108EA00070470000054B1B68082B02BF044B0022D3
:108EB0001A60044B00221A70704700BF3001001086
:108EC0001C7C0240C512002007B5084A002313701D
:108ED000074A019302A81370012300F8043D054BD3
:108EE0001B68984703B05DF804FB00BFC412002064
:108EF000F4130020F013002070470000F8B54D680F
:108F00000B4F954228BF15460C4606462A4609686F
:108F1000384636F0EEFEC6E9007560682368401BEF
:108F200060601D440030256018BF0120F8BD00BFFF
:108F3000FC130020F8B54C68944228BF144606463E
:108F40000D468CB1094F09682246384636F0D1FEED
:108F5000376074606B681B1B6B602B68201C23449C
:108F60002B6018BF0120F8BD0460F2E7FC1300205D
:108F700007B500238DF804300B4BD3F82025ADF84E
:108F80000620D3F8C034094A002B13680CBF4FF4F5
:108F900080714FF001210B431360054B01A81B6842
:108FA000984703B05DF804FB00700240CC1200202B
:108FB000F013002008B50146FFF774FFFFF75AFFD2
:108FC000837B032B0AD10846FFF762FF0121814012
:108FD000C9430448BDE80840FFF7FEBA0368002B08
:108FE000F1D008BDC81200208720FFF7E3BF86201C
:108FF000FFF7E0BF8520FFF7DDBF8420FFF7DABF72
:109000008320FFF7D7BF8220FFF7D4BF8120FFF76F
:10901000D1BF000013B5FFF745FF114B93F81E2198
:10902000032A06D16FF480710E48FFF7D5FA02B01B
:1090300010BDD3F81041002CF9D16FF480710948AC
:10904000FFF7CAFA06238DF8043088238DF806301E
:10905000054B8DF807401B6801A89847E7E700BF5C
:10906000D0120020C8120020F013002008B5FFF72E
:1090700019FF084B93F89E20032A06D16FF00101D7
:109080000548BDE80840FFF7A7BAD3F89030002B99
:10909000F4D008BDD0120020C812002073B5012200
:1090A00002FA01F51E491F4E0B6810F0800F43EACB
:1090B000050304460B6027D000F00F021A4B33F86B
:1090C000123003F1804303F51C331A684AB10022C1
:1090D0001A60BFF36F8FBFF34F8F802811D0FFF757
:1090E00069FF316829400AD106238DF804308DF8D4
:1090F00006408DF807100D4B01A81B68984702B079
:1091000070BDFFF7B3FFECE733681D42F7D10623CC
:109110008DF804308DF806008DF80720EBE700BFCE
:10912000CC120020C8120020FA340400F0130020F2
:1091300008B5054B1A781046FFF7AAFEBDE80840AF
:1091400001461046FFF7AABFF4130020FFF78EBFB9
:1091500013B5FFF7A7FE0D4B93F88E20032A13D00B
:10916000D3F8804084B96FF080710948FFF734FA72
:1091700006238DF8043008238DF80630054B8DF852
:1091800007401B6801A8984702B010BDD01200200C
:10919000C8120020F013002013B5204BD3F8004470
:1091A000C3F80044BFF36F8FBFF34F8FBFF36F8FD0
:1091B000BFF34F8FE1050BD5194B01221A7002A89E
:1091C00000230193022300F8043D164B1B689847C7
:1091D000A2050AD5124A002302A8019313700323A3
:1091E00000F8043D0F4B1B689847630513D50C4BE3
:1091F0001A7882B100221A70084B0121C3F80815B1
:109200005820FFF7CDFD02A80423019200F8043D89
:10921000044B1B68984702B010BD00BF00700240AD
:10922000C4120020F0130020064B1868082802D151
:1092300004331B6823B9A0F10D035842584170470D
:1092400001207047300100102DE9F04F764B87B0B8
:109250001A780193002A40F08680DFF8D4B1734B6E
:109260001968734B1C6821407DD011F001247DD01A
:1092700094FAA4F4B4FA84F40F2C86BFA4F1100875
:109280005FFA88F844F080084046FFF7F3FD4FFA94
:1092900088FABAF1000F064608F00F0582896ADAEB
:1092A000D0E9003104A8984700B93060614B1B68D1
:1092B000082B02BF604B82221A60019B059A04981A
:1092C00001211970A140B368DBF80040134424EA7F
:1092D0000101BAF1000FB360CBF80010574B78DAF8
:1092E000072D9BBF142101FB0533C3F8A006C3F86B
:1092F00000068CBFC3F8A426C3F80426FFF76CFD54
:10930000AB002DB26E004E4A4E49002872D0BAF121
:10931000000FB5BF92468A4604242824B2444A4D21
:109320004A4E1C4400272F60BFF36F8FBFF34F8F4F
:109330002046FFF735FD0220FFF704FC2B68002BC9
:10934000F1D01E20FFF7FEFB33689B0650D50120AD
:10935000FFF7F8FBBAF8003003F1804303F51C3344
:109360001B68002BDFD007B0BDE8F08F91FAA1F1A8
:10937000B1FA81F480E7072D304B25D9D3F8C0949A
:1093800019F4803F18BF4FF000094B4671683768E9
:1093900004A8B847049B002B86D0059B4B4583D27D
:1093A00001210225A140B573C9432048FFF714F9F4
:1093B00006238DF80C30264B8DF80E808DF80F505B
:1093C0001B6803A898474AE705F5947153F8219064
:1093D000DBE7072D9BBF142101FB0533C3F8A00772
:1093E000C3F800078CBFC3F8A427C3F8042785E798
:1093F0000220A7E7BAF1000FACBF282004201844D0
:10940000FFF7CEFC12EA2A0A38BF8A4611493AF819
:10941000153003F1804303F51C331A68002AA2D1EA
:109420000A68002AF9D09EE7C5120020C812002061
:10943000CC120020300100101C7C02400070024061
:10944000FA340400163504000471024074740240BA
:10945000F01300200071024038B5174BD3F86C446C
:10946000C3F86C44BFF36F8FBFF34F8FFFF7B4FCAB
:1094700038B1124A136823F0011103F001130C43B1
:10948000136001251CB9BDE83840FFF7DDBE94FA32
:10949000A4F3B3FA83F30F2BD9B2C8BFA1F1100024
:1094A00005FA03F3CCBFC0B241F0800024EA030404
:1094B000FFF7F4FDE6E700BF00700240F81300205C
:1094C00037B50446FFF7EEFCFFF7D4FC837B032B94
:1094D0000CD12046FFF7DCFC01218140C9430F4835
:1094E000FFF77AF8FFF7B0FE03B030BD0568002D36
:1094F000F8D12046FFF7CCFC01218140C943074841
:10950000FFF76AF806238DF80430054B8DF8064006
:109510008DF807501B6801A89847E3E7C8120020A0
:10952000F01300200720FFF7CBBF0620FFF7C8BFCE
:109530000520FFF7C5BF0420FFF7C2BF0320FFF7D8
:10954000BFBF0220FFF7BCBF0120FFF7B9BF00007B
:10955000024A00231360024A13707047F013002080
:10956000C61200204D4B4FF4006210B5C3F8002422
:10957000BFF36F8FBFF34F8FFFF756FE80B1002010
:10958000FBF730FC464B474A1868032100287AD184
:1095900049F275301860116018600020FBF724FC58
:1095A000414B1B68082B10D10020FBF71BFC3C4BE8
:1095B0003E4A1868C021002867D149F2753018600A
:1095C000116018600020FBF70FFC344B0122C3F838
:1095D0000025BFF36F8FBFF34F8FD3F80024120520
:1095E000FBD54FF40062C3F80024BFF36F8FBFF3C5
:1095F0004F8F2D4B1B68082B0FD10020FBF7F2FB80
:10960000274B2A4A1868002841D149F27531196060
:10961000106019600020FBF7E7FB234B1B68082B49
:1096200009D1234B40F2E3721A6040225A60BFF323
:109630006F8FBFF34F8F194B00248022C3F81C2576
:10964000C3F830451B4B40F2FF121A601A4B1C60E6
:10965000FFF728FC194B1C70194B02221A70FFF7F8
:10966000E3FDC8B12046FBF7BDFB0D4B0D4A186862
:1096700080B949F275311960106019600020BDE8A9
:109680001040FBF7B1BB116087E711609AE7002338
:109690001360BFE71460F1E710BD00BF0070024027
:1096A00000EC064014ED06403001001014EC0640BA
:1096B00000780240CC120020C8120020F4130020D1
:1096C000C612002008B50F4B00221A70C0B9FFF770
:1096D00083FB0D4B0D4A002814BF184610460C4B57
:1096E0000C4AC3F80403C02182F82713802151607B
:1096F0000122C3F80425BFF36F8FBFF34F8F08BD5E
:109700000148ECE7C41200200714E0010714C0016F
:109710000070024000E100E0024B1878003018BFF2
:1097200001207047C6120020034B1878012894BF0F
:1097300000200120704700BFC6120020044B1B7898
:10974000012B83BF034B5868C0F3C0100020704743
:10975000C612002000E100E010B50020FBF742FB3C
:10976000124B1B7803F0FF04BBB1114AD2F82C3521
:10977000D3B10023C2F82C350E4B1B68082B0CD13B
:109780000D4B186802F58F2202F21442C02148B92D
:1097900049F275301860116018600020FBF724FB57
:1097A000204610BD1160F8E71C46F6E7C412002001
:1097B000007002403001001000EC0640024B034AEA
:1097C000C3F80823704700BF0070024004148001F2
:1097D000024B034AC3F80423704700BF00700240E5
:1097E00004148001014B00221A707047C41200203B
:1097F00008B5FFF73FFB818108BD000070B51B4B2A
:109800001C7884BB1A4A106001221A70264664F044
:109810007F05082CEDB20CBF4FF4007140212846A3
:10982000FFF7E6FF2846FFF725FB0134092C867376
:1098300006608660EBD10024402125462046FFF7D4
:10984000D7FF2046FFF716FB0134E4B2092C8573DD
:109850000560856001D1002070BD082C0CBF4FF45D
:1098600000714021EAE70820F6E700BFC612002099
:10987000F013002008B5FFF7FDFA808908BDFFF757
:109880009BBA00002DE9F0410C460746FFF700FBAC
:1098900005460020FBF7A6FA17F00F0103D1274B6E
:1098A0001B78BB4245D1012303FA05F5244B1A6806
:1098B000244BD243186892B202432A4298463AD1C6
:1098C0003846FFF7D7FA0C233A06064603FB01F3A6
:1098D0002BD51D4A2168134401F06041A268B1F103
:1098E000005F02F001021BD1C2B9184A326094E84D
:1098F000070083E807007360D8F800301D43144B5D
:10990000C8F8005000248022B460B473C3F8042166
:109910000020FBF769FA2046BDE8F0810D4AE5E733
:109920000AB90D4AE2E70D4AE0E70D4A13440D4A31
:10993000DCE71024ECE71124EAE700BFF413002071
:10994000CC120020C81200206C8700202B8E000053
:1099500000E100E04D8E0000FD8E0000358F00001C
:10996000D8870020F98D00002DE9F0410746884690
:10997000FFF78EFA04460020FBF734FA3B0703D1C9
:10998000154B1B78BB4223D1144B154E1B68326814
:10999000DB4301259BB2A540134313EA050419D10B
:1099A0003846FFF767FA8460D8F800300360D8F8CB
:1099B00004304360336884731D430A4B3560802252
:1099C000C3F804210020FBF70FFA2046BDE8F08120
:1099D0001024F7E71124F5E7F4130020CC1200203F
:1099E000C812002000E100E000487047FC1300208E
:1099F000044B40F48070C3F81805BFF36F8FBFF3BA
:109A00004F8F70470070024000F00F03072B11D8F2
:109A100010F0800F084A0BBF03F5887303F58473B9
:109A200002EB830352F8230008BF5868431E5842D4
:109A3000584170470020704700700240064BC3F841
:109A40000C05BFF34F8F40F48070C3F80C05BFF3D3
:109A50006F8FBFF34F8F70470070024010B5082220
:109A60000021044636F069F90E4BD3F880242270A9
:109A7000D3F884246270D3F88824D3F88C1442EA93
:109A800001226280D3F89024D3F8941442EA012290
:109A9000A280D3F89824D3F89C3442EA0323E380CD
:109AA00010BD00BF0070024008B5FFF795F958B12E
:109AB000EFF3108272B64C20FFF772F94C20FFF7DB
:109AC0006FF982F3108808BD4C20BDE80840FFF70D
:109AD00067B9000013B5FFF7E5F9104B9A7B032A2D
:109AE00006D16FF480310E48FEF776FD02B010BD4E
:109AF0001C6884B96FF480310948FEF76DFD0623B8
:109B00008DF80430074B8DF806408DF807401B6830
:109B100001A89847EAE7FFF7C7FFE7E7D012002060
:109B2000C8120020F01300205020FFF739B954204C
:109B3000FFF736B9014B1878704700BFF4130020C7
:109B4000F8B50246FFF748F90746104602F00F0441
:109B5000FFF79EF901258540ED43144E97B1002093
:109B6000FBF740F93068124B28406400306004F283
:109B7000C57400201C60586004331B68BDE8F840C1
:109B8000FBF732B93846FBF72DF93068072C00EAAD
:109B90000500306008D804F59474064B43F824702F
:109BA000BFF36F8FBFF34F8F0020E7E7CC12002089
:109BB0000078024000700240F7B504460020FBF731
:109BC00011F92046FFF756F905462046FFF760F9E0
:109BD000012314F0800F03FA00F0294917D10B6814
:109BE00030EA030309D02046FFF7AAFF0323AB7333
:109BF0000020FBF7F9F803B0F0BD2B600A68C04302
:109C000002400A601F4A136803401360EEE704F045
:109C10000F02072A0FD8802C1B4E1C4B27D002F2B4
:109C2000DA32520032601A681E68D2B242F0020282
:109C300032431A601B68134E0A68336862EA0307EE
:109C40000742D5D022EA0002184300230A602B60A5
:109C50000323AB738DF807300D4B306006228DF86F
:109C600004208DF806401B6801A89847C0E740F221
:109C7000B47232601A681E68D2B242F00402D7E7AA
:109C8000C8120020CC120020007802400478024064
:109C9000F0130020FFF790BFF7B5174B174CD3F820
:109CA00080542368164EDA43164B37781B6892B2FD
:109CB00038461A43FFF7ECF8012303FA00F010428C
:109CC00002D03846FFF778FF6FF0011105F08005EC
:109CD0000C483570FEF780FC236843F001032360D5
:109CE00002A800230193052300F8043D064B1B68DE
:109CF000984703B0F0BD00BF00700240CC120020B6
:109D0000F4130020C8120020F01300202DE9F041C8
:109D1000544BD3F804530022294616460124002947
:109D20007CD1FFF759F8002869D04F4B1B78002BE6
:109D300065D1960263D54D494C4E40F2A9730B6034
:109D40004B4B1C6814F0FF041CBF1868044040F221
:109D5000AA700860186810F0FF001CBF196808405E
:109D600040F2AB713160196811F0FF01B4461CBFBD
:109D70001E68314040F2AC76CCF800601E6834407A
:109D80003C4E08D037682743376040F2A977CCF8BB
:109D900000701C601C68354F40F2AD743C601C685C
:109DA000204008D0346844EA0044346040F2AA7489
:109DB0003C60186018682D4840F2AE740460186862
:109DC00001400DD0CC0748BF42F40002C806274826
:109DD00040F2AB74046019601B6848BF42F0010296
:109DE000336833F001111CBF05F08070024313F09B
:109DF000011F04D06B0544BF316042F480621E4FE6
:109E000002F4000622F400044FF00108E4B9FFF761
:109E10001BFA2EB3BDE8F041FFF73EBF91FAA1F364
:109E20001648B3FA83F39F00384407683FB10660D1
:109E3000BFF36F8FBFF34F8F04FA03F0024304FAAE
:109E400003F321EA03016AE794FAA4F5B5FA85F56C
:109E500057F8253008FA05F5984724EA0504D5E7B0
:109E6000BDE8F08100700240C51200200078024079
:109E700004780240F81300202835040000710240E5
:109E8000F8B5114E114A34681268240C24041443A6
:109E900001271CB940F2FF133360F8BD94FAA4F512
:109EA000B5FA85F5E8B20F2DC6BF1038C0B240F044
:109EB000800000F00F03072B01D8FFF77DFE07FAA3
:109EC00005F524EA0504E4E7CC120020C8120020BE
:109ED00038B50C4C8025C4F8845163681B060FD537
:109EE000FFF7CEFF084B0022C3F80425BFF36F8FA6
:109EF000BFF34F8F4FF0FF32C4F88450C3F80823EC
:109F000038BD00BF00E100E00070024008B5FFF777
:109F1000DFFF094BD3F80423C3F808230022C3F85A
:109F20000025BFF36F8FBFF34F8FFEF7BBFF034BCF
:109F300001221A7008BD00BF00700240C612002046
:109F400010B50020FAF74EFF0E4B1B7803F0FF040C
:109F50002BB900240020FAF747FF204610BDFFF779
:109F60008FFF094AD2F8003413F40073F1D10121B4
:109F7000C2F82C15D2F80014890544BFC2F82C355C
:109F80001C46E7E7C41200200070024010B50446EA
:109F9000FFF712FE134A04F00F0064B2002C4FF0DA
:109FA0000103B4BFD2F81015D2F8141503FA00F368
:109FB0006FEA0303B5BF0B400B40C2F81035C2F87F
:109FC0001435BFF36F8FBFF34F8F074B074A33EA48
:109FD000240428BF14460123225C9340014AC2F89E
:109FE000083310BD007002400C350400F03404004A
:109FF000F8B5214A214B224D47B233EA270328BF47
:10A00000134600F00F0401211B5D01FA03F3C5F8AC
:10A0100004330646FEF7D0FE68BB002FB4BFD5F868
:10A020001035D5F8143501FA04F1B5BF19431943B9
:10A03000C5F81015C5F81415BFF36F8FBFF34F8F18
:10A04000013C062C17D8002F15DB0020FAF7CAFEBA
:10A050003046FFF775FD3046FEF71AFF094A012327
:10A0600003FA00F0136823EA000313600020BDE840
:10A07000F840FAF7B9BEF8BDF03404000C3504001E
:10A0800000700240C8120020030610B504460AD42E
:10A0900000F00F03072B06D89B00074AD358012B6B
:10A0A00001D1FFF74DFD054BC3F81845BFF36F8F86
:10A0B000BFF34F8F10BD00BF4474024000700240D8
:10A0C0000369C1688B429DBF8268D21802F1FF32DA
:10A0D00003F1FF3394BF501A581A70472DE9F0412D
:10A0E000D0E902670446F61B40689642884615464A
:10A0F000384405D935F0FDFD3D44E560BDE8F0810B
:10A100003246AD1B35F0F5FD2A4608EB06016068C6
:10A1100035F0EFFDF1E72DE9F843C56806468946BD
:10A1200017464FF000083469B3687068A54228BF2D
:10A13000E418013C621B5C1BBC4228BF3C469442B5
:10A1400028BF144649462844224635F0D2FDB3685C
:10A150002544AB4208BF00253F1BA044A144F56045
:10A16000E1D14046BDE8F88310B5114C114AA26117
:10A170000223C4E90433104BE361A2644FF400737B
:10A180000E4A2362E264002310220D49A362E01DFF
:10A190006362E362A3656365E365226536F00EFBE7
:10A1A0000849204636F00AFB2023A37110BD00BFEA
:10A1B00044880020DF3504004C1400203C140020AB
:10A1C000E8350400EC350400F8B5184C182300FB02
:10A1D000033503FB00402544C46A012C0F46164694
:10A1E00011D003D3022C1BD000240AE02846FFF72D
:10A1F00067FF864205D8324639462846FFF76EFF8C
:10A2000034462046F8BD2846FFF75AFF86423446BA
:10A2100028BF0446224639462846FFF75FFFF0E78D
:10A220002846BDE8F840FFF776BF00BF448800200D
:10A23000FFF79ABFF0B585B004A9002341F8043DAB
:10A24000054616F009FF064628460BF07FFD022161
:10A250000446284604F0A4FD032E25D1264B5B8836
:10A26000B4B9022B0BD9254B25482649C01A039BAC
:10A27000C00800041A7940F00300F7F7B3FE00208D
:10A2800008F026FF15B128460BF000FB05B0F0BD25
:10A29000002BF4D01A48194B1B49C01AC0080004FF
:10A2A000224640F00100E8E7284604F0F3F9464270
:10A2B0000746002EE6D0104B5B8893B13046F8F786
:10A2C00047F90F4C0D4B1149E41AE4089723240475
:10A2D00001930F4B00933246034644F00100F7F719
:10A2E000A1FEF7F7EFFC0028FBD1C7F59C4020301A
:10A2F000F8F728FEC6E700BF0C0500200C7E04001E
:10A300004C7E0400F3350400113604003636040098
:10A310004D36040007B50120F8F7A6F8F8F794F8D1
:10A320004FF480410020F7F789FA08B1F8F70AFEE8
:10A33000F7F780F8FDF7D4FF08B1F8F703FE002027
:10A34000FDF7E6FFF8F790FE08B1F8F7FBFD4020B7
:10A3500000F044F9164A00231370164A1380164A77
:10A3600013700CF019FA0CF019FA6846F8F76CF94A
:10A37000684610F001FF4FF4803010F0C7FE012056
:10A3800004F07AF80D4804F02BFE402011F0D0F9CB
:10A390000B4BC0F8033000F061F901F03FFC08B14D
:10A3A00010F03CFFF7F78EFC00F076F9F5E700BF00
:10A3B000910100209201002094010020A0000020C3
:10A3C000EDE10000054B1B68082B01BF044B18682A
:10A3D000B0FA80F0400918BF00207047300100102B
:10A3E0003401001008B54FF080430022C3F80C215F
:10A3F000C3F81021C3F838254FF0805203F54043CD
:10A40000D2F80414C3F82015D2F80814C3F82415A0
:10A41000D2F80C14C3F82815D2F81014C3F82C1570
:10A42000D2F81414C3F83015D2F81814C3F8341540
:10A43000D2F81C14C3F84015D2F82014C3F8441500
:10A44000D2F82414C3F84815D2F82814C3F84C15D0
:10A45000D2F82C14C3F85015D2F83014C3F85415A0
:10A46000D2F83414C3F86015D2F83814C3F8641560
:10A47000D2F83C14C3F86815D2F84014C3F86C1530
:10A48000D2F84424C3F87025FFF79CFF10B1384B75
:10A49000384A1A60FFF796FF18B1374BFB22C3F812
:10A4A0001825FFF78FFF48B13449354B0A681B6800
:10A4B00022F00F0203F00F0313430B60FFF782FF3C
:10A4C00018B1304B4FF400721A604FF08043D3F84C
:10A4D0000024D20744BF6FF00102C3F800242A4AC7
:10A4E000D2F8883043F47003C2F88830BFF34F8F3E
:10A4F000BFF36F8F4FF01023D3F80022002A03DB45
:10A50000D3F80432002B2FDA204B0122C3F80425A4
:10A51000D3F80024002AFBD04FF010221221C2F8F9
:10A520000012D3F80024002AFBD04FF0102312228F
:10A53000C3F80422154B1A46D3F800140029FBD0A7
:10A540000021C3F80415D2F80034002BFBD0BFF370
:10A550004F8F0D490E4BCA6802F4E0621343CB6083
:10A56000BFF34F8F00BFFDE70A4B0B4A1A6008BDCF
:10A570008C5600404881030000F00040E40E00408B
:10A58000580200104096024000ED00E000E001405B
:10A590000400FA05340100200090D0037047083809
:10A5A00008B5062818D8DFE800F0080F13171717AA
:10A5B0000400BDE80840F9F703B8FFF7B5F858B94B
:10A5C000BDE80840F8F7FABFBDE80840F9F70AB857
:10A5D000BDE80840F8F7F6BF08BD0000184B07B506
:10A5E0001870184A18480121F8F770FD08B1F8F7FB
:10A5F000A9FC00224FF480411448F8F772FD08B11D
:10A60000F8F7A0FC0021012300911A461048FBF73F
:10A610005BFB08B1F8F796FCFAF778FB0D48F8F702
:10A6200045FF08B1F8F78EFC0B48F8F7E5FF20B1BD
:10A6300003B05DF804EBF8F785BC03B05DF804FBEC
:10A64000F37600209DA500008836040068010020F4
:10A6500068360400103704005031040038B5F8F7AC
:10A6600097FF08B1F8F76EFC094D4FF47A7445F086
:10A6700001054FF47A40A847013CFAD10548FBF7A1
:10A68000DFFB18B1BDE83840F8F75CBC38BD00BF4F
:10A6900060360400683604000148FBF7B3BE00BF13
:10A6A00068360400014B1878704700BFF37600202D
:10A6B00013B58368D3F854339907044606D50022AE
:10A6C000114602B0BDE81040FCF72CBD0A4A082133
:10A6D000FBF76EFB03230422CDE900322046074A34
:10A6E0000821FBF765FB064A0821204602B0BDE8B9
:10A6F0001040FBF75DBB00BF1C3704003837040077
:10A700003A45040038B58368D3F854339B0705D520
:10A7100000221146BDE83840FCF704BD0E4DF8F7A5
:10A7200061FF4FF47A7445F00105013C0FD1FFF74A
:10A7300005F860B9BFF34F8F0849094BCA6802F4A6
:10A74000E0621343CB60BFF34F8F00BFFDE74FF4D0
:10A750007A40A847E9E700BF5037040000ED00E069
:10A760000400FA0508B10BF091B8704737B50D46F3
:10A77000044636F02BF801230093C1B202232A4687
:10A78000204603F0F2FE03B030BD000010B40B46CB
:10A79000054C0649002A14BF22460A4602215DF8EC
:10A7A000044BFBF705BB00BF0F3A0400113A04004D
:10A7B000132808D8044BC0EB00103C22002103EB07
:10A7C000800035F0BABA7047047C00202DE9F04FC4
:10A7D00087B0CDB20746DFF8A88011F0A9FD4FF091
:10A7E0003C0909FB05840378637040F28A222946FC
:10A7F000204810F067F9824668B100221E49A06B1C
:10A80000FFF7C4FF2846FFF7D3FF384607B0BDE87F
:10A81000F04F0BF03BB838460BF022F994F8353086
:10A82000DB000370064611F083FD03785A1C0270AA
:10A83000737086F802A0618AF01C0FF0CCFC94F8CB
:10A840000BA094F80CB00646FFF72CFF0B4B0493BB
:10A85000238A0393E389CDF800B009FB0582CDE993
:10A860000103033253463146384611F0CBFC07B0A2
:10A87000BDE8F08F85A800001D3A040065A7000020
:10A88000047C002010B5074A07493C2303FB002342
:10A8900004460122986BFFF779FF2046BDE810407F
:10A8A000FFF786BF047C0020FD3904002DE9F04746
:10A8B00086B0CCB20746DFF8BC8011F039FD3C25EC
:10A8C00005FB048503786B7040F28A2221462648F6
:10A8D00010F0F8F868B100222449A86BFFF756FF82
:10A8E0002046FFF765FF384606B0BDE8F0470AF09E
:10A8F000CDBF38460BF0B4F895F83530DB00037067
:10A90000064611F015FD03785A1C0270737002237D
:10A91000B370698AF01C0FF05EFCC4EB04142B7D4D
:10A9200000F8013BA40004F115024244297D10F017
:10A9300043FE95F80B9095F80CA00646FFF7B2FE83
:10A940000B4B04932B8A0393EB89CDF800A00334BF
:10A95000CDE9010308EB04024B463146384611F0BD
:10A9600051FC06B0BDE8F08785A800001D3A040040
:10A9700065A70000047C00202DE9F0431B218DB069
:10A9800004460BF062F9754B417D804600273C2060
:10A99000994600FB07F5EA5C012A59D15A19567805
:10A9A0008E4255D1D17A032959D1E81C18440AF0B6
:10A9B0009DFC3C2606FB0796B8F80F20338A9A4286
:10A9C00049D1B8F81120F3899A4244D198F80B2064
:10A9D000337B9A423FD198F80030002B3BD1B8F836
:10A9E0000130834237D198F813200B2A33D840F630
:10A9F0001203D340DB4313F001082CD10B2A31D1D1
:10AA000020460AF0A9FF0228054640F09C80204617
:10AA10000AF098FF8046524AB06B2946FBF7C8F906
:10AA200098F8012098F80030009229464D4AB06B02
:10AA3000FBF7BEF9FFB2002239464B4810F062F82E
:10AA40003846FFF7B5FE20460AF020FF012003E05C
:10AA50000137142F9DD100200DB0BDE8F083B2F86E
:10AA60000300A6E7B3784D442046002B44D10AF0FA
:10AA700073FF02286FD920460AF064FF06460028BB
:10AA800069D083782BBB011DC07810F0EBFC04303B
:10AA90005FFA80F820460AF05FFF20460AF05CFF6C
:10AAA000804558D8414620460BF017F8B378002B64
:10AAB0003DD10DF10808331DF2782821404603F0FE
:10AAC000ADFB002808DA29490122A86BFFF75EFEDA
:10AAD000B0E74FF00308E0E73388CDF80480F27860
:10AAE00000920821224AA86BFBF762F9214AA86B61
:10AAF0000821FBF75DF99DE70AF02EFF00B3204621
:10AB00000AF020FF0646D8B10378B3B120460AF018
:10AB100023FF4FF0030820460AF01EFF80450FD8A0
:10AB2000414620460AF0D9FF3378002BDED0124A86
:10AB3000A86B0821FBF73CF97CE74FF00108EAE736
:10AB400001220E49C1E7064AB06B0221FBF730F93A
:10AB500098F80030FFDE00239B78FBE7047C0020A0
:10AB60008F370400B437040085A80000CD370400F7
:10AB7000ED3704003A4504000B3804002038040087
:10AB8000544B2DE9F0479246804600243C229946DA
:10AB900002FB04F0C05CE8B964B2D8F80830D3F81E
:10ABA0005463C6F34006DEB1002211464046FCF76E
:10ABB000B9FA4046484A0821FBF7FAF84046474AA6
:10ABC0000821FBF7F5F84046454A0821BDE8F04763
:10ABD000FBF7EEB80134142CDAD14FF0FF34DCE788
:10ABE000072972D13F49DAF8100035F0DDFD30B1A8
:10ABF0003D4900224046BDE8F047FFF7C7BD0126AA
:10AC0000631C02D100223949F4E7C4EB0415AD00FE
:10AC1000E91C01224944DAF8040003F0F9FC3C275E
:10AC200007FB04970246F87208B93149E2E705F1DB
:10AC30000C014944DAF8080003F06EFB05F110013D
:10AC40004944DAF80C00FFF791FD024608B929499A
:10AC5000D0E77EB1012387F835300AF1100A05F1FB
:10AC60000E014944DAF80400FFF780FD024630B9CE
:10AC70002149BFE70AF10C0A87F83560EFE705F1D3
:10AC800012014944DAF80800FFF770FD024608B9DE
:10AC90001A49AFE73C23634309EB03020025012176
:10ACA000957009F80310C2F83880A1B22A461448FA
:10ACB0000AF0D9FD60B140462A461249FFF766FD09
:10ACC000E0B2BDE8F047FFF773BD062998D08FE7E3
:10ACD000BDE8F087047C002040380400913804006F
:10ACE000C2380400DC380400DF380400F9380400FE
:10ACF00019390400293904003C3904004F39040093
:10AD0000CDA700001D3A0400714B2DE9F34716460C
:10AD1000044600253C22984602FB05F0C05C10BBAF
:10AD20006DB2A368D3F85433C3F340030BB30022CE
:10AD300011462046FCF7F6F92046664A0821FBF743
:10AD400037F82046644A0821FBF732F82046634A68
:10AD50000821FBF72DF8624A0821204602B0BDE821
:10AD6000F047FBF725B80135142DD5D14FF0FF354D
:10AD7000D7E7092940F0A3805A49306935F014FD1E
:10AD800038B159490022204602B0BDE8F047FFF72C
:10AD9000FDBC4FF001096B1C02D100225349F2E7C0
:10ADA000C5EB0517BF00F91C01224144706803F090
:10ADB0002FFC4FF03C0A0AFB058A02468AF80B007A
:10ADC00008B94B49DFE707F10C014144B06803F0D3
:10ADD000A3FA07F110014144F068FFF7C7FC0246EF
:10ADE00008B94449CFE7B9F1000F0DD001238AF823
:10ADF0003530103607F10E0141447068FFF7B6FC9C
:10AE0000024628B93C49BEE70C368AF83590F1E78E
:10AE100007F112014144B068FFF7A8FC024608B9E7
:10AE20003649B0E7D6F80CA0504635F0CFFC4FF0CD
:10AE3000010907F114024244C1B2CDF800904B461B
:10AE4000504603F092FB024608B92D499BE7306952
:10AE500035F0BCFC3C2303FB058315371A7D422AE1
:10AE6000C1B247441FD159751F223169781C35F092
:10AE7000C7FC3C236B4308EB03020121917008F8E7
:10AE800003109463A9B200221E480AF0ECFCD8B16A
:10AE9000204600221C49FFF779FCE8B202B0BDE869
:10AEA000F047FFF785BCCDF800903A462023306983
:10AEB00003F05BFB02460028DBD1144963E7082955
:10AEC0007FF45FAF994666E702B0BDE8F08700BF48
:10AED000047C0020403804006439040096390400E2
:10AEE000BD390400DC380400DF380400F938040000
:10AEF00019390400293904003C3904004F39040091
:10AF0000CE390400ADA800001D3A0400E539040064
:10AF100037B50D46044635F059FC01230093C1B204
:10AF200002232A46204603F020FB03B030BD000078
:10AF300070B50D4E002406EBC4056B7983B12B79F7
:10AF400083420DD1094B0A4A56F834000221FAF720
:10AF50002FFF0023FF2246F834306B712A7170BD39
:10AF60000134032CE7D1FAE7B4800020FD39040056
:10AF70000F3A04002DE9F04F1B21C9B004460AF036
:10AF800064FEC37C0A2B074640F0B1800378B34EC1
:10AF900073B97388022B1ED9B148B7F80120B149A3
:10AFA000301A8008000440F00300F7F71BF812E0A5
:10AFB000421CFF2108A803F0BBFA002873886EDA50
:10AFC000022B08D9A648A849301A8008000440F08E
:10AFD0000300F7F703F820460AF0BEFC032840F20E
:10AFE000AB8020460AF0AEFC0546002800F0A480A5
:10AFF000C11C807810F036FA03305FFA80F82046E2
:10B000000AF0AAFC20460AF0A7FC804500F29480D2
:10B01000414620460AF061FD914B944ADFF88CB21C
:10B02000F31A9B081B0443F0030A914B9B1ADB089D
:10B030001B0443F001094FF00008C8F1FF0108A804
:10B040004044EB1CAA7889B203F0E8F8B0F100089C
:10B0500033DA884B5B881BB159464846F6F7BEFF8A
:10B0600020460AF079FC032866D920460AF06AFCDB
:10B070000546002860D0C11C807810F0F3F9C11C8F
:10B08000C9B2204605910AF067FC20460AF064FC2C
:10B090000599814250D820460AF01FFDCDE7022BCA
:10B0A00099D908A8F6F7D2FD6D4B7349F31A9B089E
:10B0B0001B04024643F0030077E77388022BCFD9C5
:10B0C000B7F811200792B7F80F302988069308A81F
:10B0D0000591AD78F6F7BAFD05990091CDE90150DB
:10B0E000DDE9063265495046F6F7AAFFB8E7072BB7
:10B0F0002CD1634E427D002537464FEAC50806EB4A
:10B1000008035979F9B11B7993421CD10022FF2120
:10B110005C480FF0F7FCD8B15B4B5C4A56F8350041
:10B120000221FAF745FEB8440023FF2247F83530E4
:10B1300088F8053088F8042020460AF0A7FB012093
:10B1400049B0BDE8F08F0135032DD6D10020F7E7D7
:10B1500020460AF001FC032820460CD80AF0F2FB36
:10B16000037833B94A4A56F835000821FAF720FE29
:10B17000D9E7484AD2E70AF0EFFBA0B320460AF02D
:10B18000E1FB064678B303785A0629D020460AF038
:10B19000E3FB4FF0040920460AF0DEFB814522D88C
:10B1A000494620460AF099FC3B4A57F83500DFF83B
:10B1B00000A1DFF800B10821FAF7FAFD4FF000090D
:10B1C000327857F835007388A2BB72788AB1012AA9
:10B1D0002ED05A460221FAF7EBFD4FF001090CE0A0
:10B1E0004FF00109D7E72D4B284A57F835000221C7
:10B1F00097E752460821FAF7DBFD20460AF0ACFB40
:10B2000000B320460AF09EFB0646D8B103785B06E1
:10B2100016D020460AF0A0FB0421204605910AF032
:10B220009BFB059981420DD820460AF056FCC7E7E2
:10B230001B4ADFE7009202211A4AFAF7B9FDCCE770
:10B240000121EAE757F83500B9F1000F03D0164B9A
:10B250000E4A022165E70E4A082187E7780500209B
:10B26000EC040020383A04006B3A04000C7E040021
:10B270004C7E04000C050020A93A0400063B0400A3
:10B28000B480002031AF0000503B04000F3A0400AE
:10B290003A4504006F3B0400322F0400A43B040035
:10B2A000023C0400843C0400C43C0400DA3A04007C
:10B2B000D13B0400413C04002DE9F04F0E468FB015
:10B2C000044684491068154635F06EFA012E07468B
:10B2D00004D0A368D3F854339B0715D50022114638
:10B2E00020462D68FBF71EFF7B4A08212046FAF70F
:10B2F0005FFD7A4B00937A4A2B4608212046FAF7E5
:10B3000057FD0FB0BDE8F08FF31F022B02D8072EB8
:10B3100007D030B1734B744A02212046FAF748FD3A
:10B32000EFE701220BA9686803F072F98DF8340089
:10B3300008B96E4BEFE70DF13501A86802F0ECFF9C
:10B3400008B96B4BE7E70DF12201E868FFF7E0FD74
:10B3500008B9684BDFE708A92869FFF7D9FD08B9E4
:10B36000654BD8E709A96869FFF7D2FD08B9634BB7
:10B37000D1E70DF12601A86902F0CEFF08B9604BB4
:10B38000C9E75FB95F4B0A93072E14D00AAA5E493A
:10B39000E86935F08DF918B95C4BBCE75C4BF2E716
:10B3A000092E08D10DF12A025749286A35F080F993
:10B3B00008B9584BAFE70AF012FA814600287AD054
:10B3C000554D6E7936B16B7B002B76D06B7D002BA3
:10B3D00075D10226F70005EB0708012388F8053030
:10B3E00045F8364010F0A4FF037888F8043048464A
:10B3F0000AF036FB4FF0000B80F800B0804610F0EA
:10B4000097FF03785A1C027088F80130062388F8E9
:10B41000023088F803B0BDF8241008F104000EF0E3
:10B42000DAFE9DF8263000F8013BBDF828100EF03A
:10B43000D2FEBDF82A100EF0CEFE82469DF8260000
:10B4400010F064F930B150465A469DF8261010F0BD
:10B45000B3F882469DF835309DF834B00793FFF776
:10B4600021F9BDF822200392BDF82020079B00930C
:10B470004FF000082F44CDE9010251460BAACDF848
:10B4800010805B46484610F0BDFE40F24512397907
:10B4900022480FF017FB00283FF433AF204B124A2D
:10B4A00002212046FAF784FCFF2387F805803B71D0
:10B4B00045F8368025E71B4B2DE701268AE7204615
:10B4C000194B094A0221FAF773FC48460AF0DEF9E3
:10B4D00017E700BF8C370400063D04001A3D040046
:10B4E0000F3D04008E3D0400113A0400AC3D040001
:10B4F000C33D0400DD3D0400F23D0400073E0400AE
:10B500001E3E040001003C00373E04003B3E0400A8
:10B510000F00FFFF563E0400B480002031AF000052
:10B52000C43E0400713E04009E3E0400034A044BE6
:10B53000002908BF1A460821FAF73ABC384504002A
:10B540003A45040073B51646002204460D461146DE
:10B55000FBF7E8FD2046064A0821FAF729FC009689
:10B560002B46044A08212046FAF722FC02B070BD9F
:10B57000063D04000F3D040038B513468268D2F83A
:10B580005443C4F3400405462CB11968064ABDE88B
:10B590003840FFF7D7BF20460FF084FD21462846EC
:10B5A000BDE83840FFF7C2BF194104000B46024A0C
:10B5B0000221FAF7FDBB00BF113A040038B58368D9
:10B5C000D3F854339B070446154605D5002211468F
:10B5D000BDE83840FBF7A6BD012919D10FF010FED8
:10B5E000032804BF1B4B187850B91B4A082120467A
:10B5F000FAF7DEFB20460121BDE83840FFF796BF91
:10B60000012801D1154AF1E70228F3D1144AEDE7E8
:10B6100002291DD1134B1B7823B11349BDE83840D3
:10B62000FFF7C4BF0C49506835F0BEF818B9094B94
:10B630000E4A1870DAE70949686835F0B5F820B99C
:10B64000044B01221A700A4AD0E70A492046E5E76E
:10B650000949E3E7900100206343040066430400C6
:10B660008D610400CD800020694304007F43040005
:10B670008F4304009F430400DF38040001297FB595
:10B6800004460D460DD104F0F3FB08214388144A0B
:10B690002046FAF78DFB29462046FFF747FF04B006
:10B6A00070BD022919D15668304635F08FF8012354
:10B6B0000093C1B22B460DF10E02304602F055FF49
:10B6C00030B104F0D5FBBDF80E3043800021E3E734
:10B6D00004492046FFF76AFFE1E70349FAE700BFA4
:10B6E0001E430400224304003943040038B51346C6
:10B6F0008268D2F854239207044605D51968194A7E
:10B70000BDE83840FFF71EBF174D2A7812BB0FF077
:10B7100003FD164B1B789BB1012B15D10FF06CFD6F
:10B72000134A08212046FAF743FB0FF075FDB0B924
:10B7300001232B7020460021BDE83840FFF7F6BEFC
:10B740000FF04EFD0B4AECE70B492046BDE83840B0
:10B75000FFF72CBF022018F0B3F80028E8D1074902
:10B76000F3E700BFB0430400CD800020900100202B
:10B77000D6430400E74304009F430400FD43040054
:10B780002DE9FF478368D3F85453C5F340050446B9
:10B79000164635B13E4A3168FFF7D4FE04B0BDE825
:10B7A000F087012930D10FF0B7FC02900FF0C6FCF2
:10B7B000DFF81091374BDFF81081039002AF4A4653
:10B7C00008212046FAF7F4FA0B264FF0010A3A68EE
:10B7D0000AFA06F3134205D03346424608212046B2
:10B7E000FAF7E6FA01361B2EF1D12B4A0821204642
:10B7F000FAF7DEFA0437294B25B100212046FFF77E
:10B8000095FECBE70125DAE702293ED1244B1D78CE
:10B810001DB12449FFF7CAFEC0E76A462249706895
:10B8200034F046FF009AA2F10B030F2B11D901AAA5
:10B830001E497068009534F03BFF019B1C4A1A407A
:10B8400022B123F0FF6323F4FF232BB119492046D3
:10B85000E0E70123934001930FF05EFC019B9842C7
:10B86000CBD0009A7AB11346134A08212046FAF742
:10B870009FFA01980FF04AFC01980FF059FC0198CB
:10B880000FF078FCB9E70D4AEFE70D49C2E700BFBA
:10B89000D13F0400C93F0400322F0400754004006A
:10B8A000CD800020694304007F40040083400400F1
:10B8B00000F8FF078740040097400400AF400400F1
:10B8C000DF38040066400400524C04002DE9F041CA
:10B8D0008368D3F854339B078AB005460E46144656
:10B8E00001D4012907D13A4A21682846FFF72AFEE8
:10B8F0000AB0BDE8F08102291ED13649106834F043
:10B9000053FF0646002853D16468204634F05EFF9A
:10B910000096C1B2122305AA204602F026FE002896
:10B9200040D005A9032003F08BFE00283CD1002164
:10B930002846FFF7FBFDDBE7032904D0264928460C
:10B94000FFF734FED4E72549106834F02DFF804618
:10B950000028F3D1224B1B780BB92249EFE7676827
:10B96000384634F033FFCDF80080C1B2122305AA67
:10B97000384602F0FAFDA8B1324603A9A06802F0E9
:10B9800047FE98B105AA314603A80DF055F90028E5
:10B99000CDD01549D3E71549606834F005FF00287C
:10B9A000CCD112E01249CAE71249C8E71249C6E7EA
:10B9B0001249206834F0F8FE0028BFD110496068B1
:10B9C00034F0F2FE0028E6D1012003F00DFEAEE7D0
:10B9D000974104002E460400744104007E42040096
:10B9E000CD8000208242040063410400ED45040044
:10B9F0003F410400524104008141040068460400B4
:10BA00001422040038B58368D3F854339B070446E6
:10BA1000154605D529681F4ABDE83840FFF792BD95
:10BA20001D4B1B7823B91D49BDE83840FFF7BEBD4B
:10BA3000012910D11A4B1B4A19781B4B002908BF4A
:10BA400013461A4A0821FAF7B3F920460021BDE847
:10BA50003840FFF76BBD022919D11549506834F001
:10BA6000A3FE30B901200FF06FFB0D4B01221A70BD
:10BA7000EBE768680F4934F097FE054620B90FF0F0
:10BA800063FB074B1D70E0E70B492046CCE70B49F1
:10BA9000CAE700BF98420400CD8000208242040023
:10BAA000CC800020944204008C370400C52404009C
:10BAB00014220400ED450400EE420400DF380400C7
:10BAC00070B513468268D2F85423920786B00546B3
:10BAD00005D5144A1968FFF735FD06B070BD124A46
:10BAE00014781CB11149FFF761FDF6E7022917D15F
:10BAF0005E68304634F06AFE0094C1B2102302AA98
:10BB0000304602F032FD40B1214602A81CF092FA04
:10BB100021462846FFF70AFDDFE705492846E2E708
:10BB20000449E0E702430400CD800020694304009B
:10BB30000A4304007441040013B513464FF0FF326A
:10BB400001928268D2F854239207044605D5154A1B
:10BB50001968FFF7F7FC02B010BD02291FD1124A85
:10BB600012781AB11149FFF721FDF4E701AA104933
:10BB7000586834F09DFD0198202802D90D492046CF
:10BB8000F1E7C0B20FF042FB2046019B0A4A0821B0
:10BB9000FAF70EF901212046FFF7C8FCDBE7074959
:10BBA000E1E700BFF33E0400CD80002069430400BC
:10BBB0007F400400803F0400AD3F0400DF380400F4
:10BBC000012937B5134604460D460ED168460FF0DD
:10BBD000E9FA69462B460822204602F0AFFB2946C7
:10BBE0002046FFF7A3FC03B030BD02290FD103228A
:10BBF0006946586802F00CFD20B168460FF0CAFA99
:10BC00000021EDE703492046FFF7D0FCEBE70249AE
:10BC1000FAE700BFCF400400E8400400014B187869
:10BC2000704700BFCD80002037B50D46044634F084
:10BC3000CDFD01230093C1B202232A46204602F023
:10BC400094FC03B030BD0000132806D8034B342207
:10BC5000002100FB023034F070B87047BC8800202F
:10BC600010B5084B084A0446342000FB043002217A
:10BC7000006B064BFAF79CF82046BDE81040FFF732
:10BC8000E3BF00BFBC8800200F3A0400FD39040068
:10BC90002DE9F04F0D462F4C34266E4304EB060978
:10BCA00087B0074610F044FB99F82C10037889F808
:10BCB00001300901002241F0010199F82A30009277
:10BCC00001F0F101384610F015FBA24680464C46C3
:10BCD000A8EB000394F82920DBB29A422CD894F800
:10BCE000029094F80BB0FEF7DDFC00230493E38987
:10BCF0000393A389CDF800B0F21CCDE901035244AF
:10BD00004B464146384610F07DFA94F82C30EDB29F
:10BD1000BBB940F28A2229460F480EF0D3FEB0B1DB
:10BD20000E4B0F4A206B0221FAF742F8284607B063
:10BD3000BDE8F04FFFF788BF23441B7C08F8013BA8
:10BD4000C6E7084A206B0821FAF732F8EEE707B099
:10BD5000BDE8F08FBC88002061BC00008148040071
:10BD6000113A04003A4504002DE9F3471B21064629
:10BD700009F06BFF0746417D584800253424804672
:10BD800004FB05F31A1813F800C0BCF1010F40F0D2
:10BD9000908092F801C08C4540F08B809178032907
:10BDA00040F08F800333184409F0A0FA342404FBD8
:10BDB0000584B7F80F20E3899A427ED1B7F81120A5
:10BDC000A3899A4279D1FA7AE37A9A4275D197F89F
:10BDD0000090B9F1000F70D1B7F8013083426CD1F7
:10BDE000FB7C0B2B69D1304609F0B6FD0228824658
:10BDF00070D1304609F0A6FD4378394A0746002B3A
:10BE000014BF02210321206BF9F7D2FF7A783B7827
:10BE10000092002A14BF02210321324A206BF9F755
:10BE2000C7FF7B78304A206B002B14BF022103210F
:10BE3000F9F7BEFF7B78002B46D02C4B2C4A206BA9
:10BE40005146F9F7B5FF3423EFB203FB058595F8AA
:10BE50002C2032BB394627480EF054FE454280461E
:10BE6000FDB1254B5B889BB12846F6F771FB234C4F
:10BE7000234B2449E41AE4084FF424732404019367
:10BE8000214B00932A46034644F00100F6F7CAF816
:10BE9000F5F718FF0028FBD1C8F59C402030F7F7D4
:10BEA00051F83846FFF7D0FE304609F0EFFC01208C
:10BEB00004E00135142D7FF463AF002002B0BDE82B
:10BEC000F087B2F8030071E7104A206B0821F9F7F8
:10BED0006FFFB8E799F80130FFDE00BFBC88002093
:10BEE0006F4604008D460400322F0400A54604006E
:10BEF0000F3A040061BC00000C0500204C7E0400D9
:10BF00000C7E040036360400BC4604003A450400AA
:10BF100001292DE9F7430546144614D1146800227F
:10BF20001146FBF7FFF86F4A08212846F9F740FF52
:10BF30006D4B009323466D4A08212846F9F738FFD8
:10BF400003B0BDE8F0838368D3F85463C6F34006BA
:10BF500066B103226649FBF7E5F8624A08212846E4
:10BF6000F9F726FF634B00932368E4E7624B342024
:10BF7000984600FB06F2D718D25CA2BB0539012314
:10BF800005293B703BD887F82C304FF4827387F833
:10BF90002920BB815949606834F006FC00283AD05A
:10BFA0000434342202FB06F7F91C012241442068C4
:10BFB00002F02EFB08EB070989F8020050B950493E
:10BFC000206834F0F1FB50BB89F8020089F80300C7
:10BFD00089F8040007F10B014144606802F09CF904
:10BFE000F8B9484B0CE00136142EC2D1464B474AF3
:10BFF0000221284603B0BDE8F043F9F7D9BE444B0F
:10C00000424A28460221F9F7D3FEF0B203B0BDE858
:10C01000F043FFF719BE87F82C000834C1E73D4B09
:10C02000EEE707F10E014144A068FFF7FDFD08B9F6
:10C03000394BE5E73949E06834F0B6FB48B10C34D8
:10C0400007F12A0141442068FFF7EEFD60B9344B47
:10C05000D6E707F10C0141442069FFF7E5FD08B977
:10C06000304BCDE71434EBE72F49606834F09CFB8C
:10C0700048BBA06834F0AAFB322881460CD91923AA
:10C080002A4A04212846F9F793FE4FF0320919F0A5
:10C09000010F03D0264BB3E70028F8D1002300930B
:10C0A00007F11002192342445FFA89F1A06802F0F7
:10C0B0005CFA08B91F4BA3E7342303FB06834FEA5E
:10C0C000590983F82990342303FB06880022C8F815
:10C0D0003050B1B2184809F0C6FB00283FF430AF29
:10C0E000164B8DE7063D0400074704000F3D040092
:10C0F0009048040055470400BC880020A64704006F
:10C10000D4690400BE47040066480400113A0400E4
:10C11000DF380400A9470400CE470400DF470400CD
:10C12000F3470400E2470400004804000348040009
:10C130003D4804005848040091BC00001D3A04002A
:10C1400008B109F0A3BB704770B50546F6F786FC49
:10C150000221FCF7BDFD04460EF018FFAE696A69C6
:10C16000064B811A994288BF121A4FF4705394BF3C
:10C170004B435343A01B184470BD00BFFEFFFF7F1D
:10C1800010B5144606282BD8DFE800F00F1104265E
:10C19000212A27001A4A4FF47A73B1FBF3F3E069BE
:10C1A0000221BDE81040F9F703BE137BA3B94FF499
:10C1B0007A73144AB1FBF3F3E0690821F9F7F8FD4B
:10C1C000E069114A0821BDE81040F9F7F1BD137B81
:10C1D00013B9D37A002BF3D010BD0C4B0C4ADEE719
:10C1E0000C4B5A88002AF7D00B4A0C499B1A9B0823
:10C1F0001B040246BDE8104043F00100F5F7F2BE13
:10C20000D94B0400044C04003A4504001A4C0400C5
:10C210000F3A040074050020EC040020364C0400A2
:10C2200010B508480023242101FB03F2145C1CB95B
:10C2300001238354104410BD01330A2BF4D1002094
:10C24000F9E700BF4881002018B12422002133F013
:10C2500074BD704770B50B4E00EBC00406EB840450
:10C2600005462046FFF770FF242303FB05650146C2
:10C270002B6A13B12246022098472046BDE8704041
:10C28000FFF7E2BF488100202DE9F74F054600285F
:10C290007ED0102109F0D9FC4279074652BBB0F894
:10C2A0000690DFF810A14FF000084FF0240B0AF1C0
:10C2B00001030BFB08F616F80A20012A08D10AEB45
:10C2C0000604627A022A2ED1B4F801204A454BD0E6
:10C2D00008F10108B8F10A0FEBD12F484388012B70
:10C2E0001BD92E4B3A682E49C01A8008000440F032
:10C2F000020010E0032A04D1063008F0F7FF81465F
:10C30000CFE72548438843B1244B2649C01A80080B
:10C31000000440F00100F5F765FE284603B0BDE8D3
:10C32000F04F09F0B3BA9819019308F0DFFF019BB1
:10C330008145CCE7236A23B1E27A92B922460420F0
:10C340009847227B002AE8D117491848B610714354
:10C35000C9B20EF0D7FB0028DFD12046FFF774FFEB
:10C36000DBE722463846EBE72046FFF7EDFE3F6865
:10C370000146002FDED0084B5A88002ACDD007484E
:10C380000B491B1A9B081B043A4643F00100C2E705
:10C3900003B0BDE8F08F00BF74050020EC0400205E
:10C3A000A44B0400364B0400398EE33855C200001C
:10C3B0007D4B04004881002018B10C22002133F08D
:10C3C000BCBC70472DE9F04F1B2193B0054609F026
:10C3D0003CFCB0F80F204BF6EF639A42044603D0C2
:10C3E000002013B0BDE8F08FB0F81130B3F5827FB4
:10C3F000F6D11B212846B84F09F027FC3A680646BB
:10C40000002A3BD0242200210DEB020033F095FCE2
:10C41000F37C022B4FD0032B05D07BBB01238DF87F
:10C4200030308DF82F3001238DF824302846737D6D
:10C430008DF82E3009F090FAADF832000EF0A6FD1E
:10C440008046F6F70BFB0221FCF742FCCDE90780A2
:10C4500007AA92E803000EAB83E80300337873B3B6
:10C460009E4B5B88022B09D99D489E4B9E49C01A62
:10C47000C008000440F00300F5F7B0FDE27C012A9B
:10C4800040F08680994B627D002624219A4601FB6C
:10C4900006F818F80300012821D103EB0807B87A41
:10C4A00090421CD17A7A022A1DD008F1010018446A
:10C4B00008F01CFF19E001238DF83030B3E70223A8
:10C4C0008DF82D300E99B6F80130ADF825304FF4C7
:10C4D000705041433B6809AA05209847CEE70136D2
:10C4E0000A2ED4D17CE7B7F8010094F800B0BBF174
:10C4F000000F7FF475AFB4F8013083427FF470AF62
:10C500003846FFF721FE7A494FEAA80801FB08F1F7
:10C510005A468146C9B277480EF0F4FAC0F1000BD2
:10C520008046BBF1000F1FD06C4B5B889BB1584617
:10C53000F6F70EF86A4C6B4B6F49E41AE4084FF4B7
:10C540002E73240401936D4B00935A46034644F026
:10C550000100F5F767FDF5F7B5FB0028FBD1C8F53D
:10C560009C402030F6F7EEFC242303FB06A6336A3A
:10C570001BB13A46494601209847B8F1000F02D155
:10C580003846FFF761FE284609F080F9012028E7C8
:10C5900012F0FD0640F0C280284609F0DDF9584A45
:10C5A00033460C2606FB03F7B95C49BBD6194FF09E
:10C5B000010802F807807071627D3271E27C002A06
:10C5C00008BF4146B1712278002A7AD14C4BB4F8A9
:10C5D0000120DC196280FEF765F8824609F0FFF859
:10C5E0008146F8B947484388012B63D9464B4749F0
:10C5F000C01A8008000440F00200F5F7EFFC59E093
:10C6000001330A2BCED13F484388012B7FF6E8AE99
:10C610003D4B3F49C01A8008000440F00200F5F786
:10C62000DDFCDDE609F01CFA11220270227942706D
:10C6300080F8028000F1030B6279CD21584633F077
:10C640007CFB2F4B33486179A479CDF800A00237E9
:10C65000DA194BF6EF63CDE903304FF48273CDE97D
:10C6600001A359440223484644B30FF0CBFD47428F
:10C670008046FFB1194B5B889BB13846F5F768FFE0
:10C68000174C184B1C49E41AE4084FF40F732404A8
:10C6900001931A4B00933A46034644F00100F5F724
:10C6A000C1FCF5F70FFB0028FBD1C8F59C402030FA
:10C6B000F6F748FC3046FFF77FFE64E7F6F7FDFB30
:10C6C000F8E710484388012BF4D90F4B1249C01AE0
:10C6D000800800048FE700BFB48200200C05002012
:10C6E0004C7E04000C7E0400274904004881002091
:10C6F000398EE33855C200003636040088490400FC
:10C70000D080002074050020EC040020FC490400C7
:10C71000CC49040041C10000304A0400032A3FF420
:10C7200032AF07484388012B7FF62DAF054B0649F2
:10C73000C01A8008000440F00200F5F753FC22E71D
:10C7400074050020EC040020604A04002DE9F0414B
:10C75000044688B0FDF7A6FFE3894F2B07460AD9A8
:10C76000236A002B00F08C8022460021062008B0AE
:10C77000BDE8F041184709F032F880460028EFD0B4
:10C7800009F06EF9554E1123037033784370237B03
:10C79000C51C002B79D0E37A002B74D00023837062
:10C7A000E289AB21284633F0C8FAE3891D44337887
:10C7B000A372013333700EF0E9FB0646F6F74EF92B
:10C7C0000221FCF785FACDE9066008AA12E9030008
:10C7D00004F1140383E803004148E67A637A009782
:10C7E0004BF6EF61CDE903104FF48271CDE9017191
:10C7F000621C29464046002E49D00FF003FD4642F8
:10C800000746FEB1374B5B889BB13046F5F7A0FE7B
:10C81000354D364B3649ED1AED084FF401732D04B2
:10C820000193344B00933246034645F00100F5F77F
:10C83000F9FBF5F747FA0028FBD1C7F59C402030FB
:10C84000F6F780FB236A3BB12046FFF77DFC236AA5
:10C8500001462246032098472749228A2748641A1E
:10C860002749A4104FF47A7361435343C9B24FF47C
:10C870007052B3FBF2F20EF025F9454206464DB96F
:10C8800008B0BDE8F081022389E7032387E7F6F7C4
:10C8900014FBD7E7134B5B889BB12846F5F758FE8E
:10C8A000114C124B1249E41AE40840F217232404F5
:10C8B0000193104B00932A46034644F00100F5F71C
:10C8C000B1FBF5F7FFF90028FBD1C6F59C402030FD
:10C8D00008B0BDE8F041F6F735BB00BFB0820020DC
:10C8E00089C200000C0500204C7E04000C7E040070
:10C8F00036360400884904004881002055C20000F3
:10C90000398EE3382DE9F74F8368D3F85433C3F3F6
:10C9100040079B0705460E46904601D4012916D1D3
:10C92000002211462846D8F80040FAF7FBFB2846BB
:10C930003C4A0821F9F73CFA3B4B00933B4A23461B
:10C9400008212846F9F734FA03B0BDE8F08FCB1E72
:10C95000022B07D9364B374A022103B0BDE8F04F0E
:10C96000F9F726BAFFF75CFC044620B9324B314A8E
:10C9700002212846F1E7314B0362C77242F210737D
:10C980000127DFF8CCA0DFF8CCB007730382A6F153
:10C990000209B94517D806F18046023E0122A118C6
:10C9A00058F8260001F034FEB7006072F0B9244B4D
:10C9B000204A28460221F9F7FBF9204603B0BDE8DA
:10C9C000F04FFFF741BC514658F8270033F0ECFE1A
:10C9D00018B90123E3720137DBE7594658F82700FD
:10C9E00033F0E2FE0028F6D12073F4E7B84404F1F6
:10C9F0000E021449D8F8040033F05AFE08B9124B5D
:10CA0000D6E7E3894F2B06D9104A08212846F9F7C3
:10CA1000CFF94F23E3812046E56103B0BDE8F04F35
:10CA2000FFF794BE063D04008F4A04000F3D04004A
:10CA3000DF380400113A0400F938040081C1000015
:10CA4000A9470400C03C0400D54A0400F14A040090
:10CA5000C14A0400CB4A040010B504462EF0C3FBC3
:10CA6000064A034608212046F9F7A2F92046044A5F
:10CA70000821BDE81040F9F79BB900BF624C0400E3
:10CA80003845040037B58368D3F854339B07044610
:10CA90000D4605D500221146FAF744FB03B030BD20
:10CAA00002291CD10DF10701506801F035FC30B9A5
:10CAB0000D4B0E4A29462046F9F77AF9EEE79DF824
:10CAC0000700A0F10B030F2B01D9094BF1E72EF062
:10CAD0007BFB084A08212046F9F76AF9DEE7064B96
:10CAE000024A0221E8E700BF804C0400113A04002A
:10CAF000904C040038450400DF38040030B58368EA
:10CB0000D3F854339B078BB004460D4605D500225D
:10CB10001146FAF707FB0BB030BD012905D0174BC2
:10CB2000174A0221F9F744F9F5E701A831F0F6F9BF
:10CB300020B1144B124A02212046F3E79DF8183029
:10CB40002BB99DF81C3013B99DF820300BB10E4B5A
:10CB5000F0E78DF818508DF81C508DF82050F6F73E
:10CB60002DF801A831F088F908B1084BE2E7084A2E
:10CB700008212046F9F71CF9CDE700BFDF38040093
:10CB8000113A0400BA4C0400E34C0400F74C0400D2
:10CB90003A450400F0B51E468368D3F854339B072A
:10CBA0008BB004460F4605D500221146FAF7BAFAB3
:10CBB0000BB0F0BD022A05D02B4B2C4A0221F9F70D
:10CBC000F7F8F5E701A831F0A9F920B1284B274A79
:10CBD00002212046F3E79DF8183013B99DF81C3068
:10CBE0000BB1244BF3E72449384633F0DDFD58B14F
:10CBF0002249384633F0D8FD78B12149384633F020
:10CC0000D3FD60B11F4BE2E706AD0DF10301706883
:10CC100001F082FB28B91C4BD9E707ADF5E708AD59
:10CC2000F3E71A49306833F0BFFD40B99DF803308F
:10CC3000AB7001A831F020F978B1154BC7E7154961
:10CC4000306833F0B1FD30B99DF80330003318BFC0
:10CC500001236B70EDE7104BB9E7104A082120461D
:10CC6000F9F7A6F8A4E700BFDF380400113A040082
:10CC7000BA4C04001A4D04004F4D0400524D0400FC
:10CC8000564D04005A4D0400704D0400CB4F040073
:10CC9000F74C04001F500400804D04003A45040086
:10CCA00013460A460149FFF775BF00BF564D040001
:10CCB00013460A460149FFF76DBF00BF524D0400FD
:10CCC00013460A460149FFF765BF00BF4F4D0400F8
:10CCD00010B50849002201EB02135C7A24B11C7ADA
:10CCE000844201D1184610BD0132032AF3D100203D
:10CCF000F9E700BFB88200200848437A2BB1437E91
:10CD000043B190F829303BB9022300EB0310012313
:10CD1000437270470123F8E700207047B882002073
:10CD20000023FF2243720272C0E90033837270470E
:10CD300073B51646002204460D461146FAF7F2F97D
:10CD40002046064A0821F9F733F800962B46044A94
:10CD500008212046F9F72CF802B070BD063D04000A
:10CD60000F3D040037B50D46044633F02FFD012377
:10CD70000093C1B202232A46204601F0F6FB03B01D
:10CD800030BD2DE9F0410746904600240D46A6B27D
:10CD9000B54208EB440106D957F82400FFF7E2FF3B
:10CDA00001340028F3D1AB1B58425841BDE8F08153
:10CDB00010B40B46054C0649002A14BF22460A4609
:10CDC00002215DF8044BF8F7F3BF00BF0F3A0400EF
:10CDD000113A040010B5FFF77BFF044648B1006824
:10CDE00004490122FFF7E4FF2046BDE81040FFF7A9
:10CDF00097BF10BD9453040010B5FFF769FF0446B8
:10CE000048B1006804490122FFF7D2FF2046BDE87F
:10CE10001040FFF785BF10BD8F5A040010B5FFF713
:10CE200057FF044648B1006804490122FFF7C0FFDC
:10CE30002046BDE81040FFF773BF10BD6A540400E0
:10CE400010B5FFF745FF044648B1006804490122C8
:10CE5000FFF7AEFF2046BDE81040FFF761BF10BDF1
:10CE6000AE5904002DE9F0410E4604464C491068C5
:10CE7000154633F099FC012E804605D0A368D3F8FF
:10CE80005423C2F3400232B12968464A2046BDE825
:10CE9000F041FFF74DBF072E05D043492046BDE8BE
:10CEA000F041FFF785BF08F09AFC074610B902462B
:10CEB0003E49F3E7182108F0C8FE03220146064662
:10CEC000686801F0A5FB024640B939492046FFF7E2
:10CED0006FFF3846BDE8F04108F0D8BC06F1080104
:10CEE000A86801F019FA024608B93249EEE70122B2
:10CEF00006F10D01E86801F08BFB0246307308B9BA
:10CF00002D49E3E706F11501286901F005FA02460B
:10CF100008B92A49DAE706F10A016869FFF722FF32
:10CF2000024608B92649D1E7022206F11601A8698E
:10CF300001F06EFB10B900222249C7E7FFF7DCFEC3
:10CF4000054610B902462049C0E704601F4938462B
:10CF5000B8F1000F0ED115F067F92872297AFF2970
:10CF60000BD1204600221A49FFF722FF2846FFF77F
:10CF7000D7FEAEE715F05BF9EFE740F24512154832
:10CF80000DF0A0FD48B1204600221349FFF710FF25
:10CF90002846BDE8F041FFF7C3BEBDE8F08100BF01
:10CFA0008C370400055204008E3D0400713E0400DD
:10CFB000795204009F520400B9520400DE5204006A
:10CFC000DD3D0400FD52040033530400A1DB0000EA
:10CFD0004D530400D5CD0000C43E040001292DE9C5
:10CFE000F3410446904605D08368D3F85453C5F303
:10CFF000400545B12C4AD8F800102046FFF798FEAE
:10D0000002B0BDE8F081022904D028492A46FFF782
:10D01000CFFEF5E708F0E3FB074618B902462449BE
:10D020002046F4E7062108F010FE858006460DF143
:10D030000601D8F80400FFF795FE024638B91D49ED
:10D040002046FFF7B5FE384608F020FCD8E7BDF8CB
:10D05000063073803380FFF74FFE064610B9024654
:10D060001549EDE704601549384617F079FFFF28A8
:10D070000146307208D120462A461149FFF798FE32
:10D080003046FFF74DFEDEE740F245120D480DF049
:10D0900019FD0028B4D020462A460B49FFF788FE28
:10D0A0003046FFF73DFEABE7D15304008E3D040050
:10D0B000713E0400E35304003353040089D8000098
:10D0C0004D5304001DCE0000C43E04002DE9F7437B
:10D0D00005230129044689461646ADF8043005D0DB
:10D0E0008368D3F85453C5F340053DB1804A316895
:10D0F0002046FFF71DFE03B0BDE8F0837D49506870
:10D1000033F052FB28B97C4900222046FFF750FE3D
:10D11000F1E77A49706833F047FB0028F3D0B9F1A2
:10D12000050F02D82A467649EFE708F058FB8046FB
:10D1300010B902467349E8E70A2108F055FC0DF1E1
:10D14000060105467068FFF70DFE024638B96E49C4
:10D150002046FFF72DFE404608F098FBCBE7BDF8D0
:10D1600006302B800DF10601B068FFF7FBFD02468B
:10D1700008B96649ECE7BDF806306B800DF1060191
:10D18000F068FFF7EFFD024608B96149E0E7BDF836
:10D190000630AB80A91D306901F0BEF810B900223D
:10D1A0005C49D5E7AB79022793B16FF0010107FB2A
:10D1B0000311404608F0B5FC05F10802A97906F113
:10D1C0001400FFF7DEFD024608B95349C0E7002707
:10D1D000AB790533E91D56F8230001F09DF80246AE
:10D1E00008B94E49B4E7E97999B1C7EB4101404626
:10D1F00008F097FCAB79E979981D05F1080202EB7C
:10D20000430206EB8000FFF7BCFD024608B9444923
:10D210009EE7AF79EB7906371F44BB1C4B4507D01F
:10D220000027FFF769FD064658BB02463D498FE7D8
:10D23000304956F827004FEA870933F0B5FAC0B9EC
:10D240004E4401AA3849706833F032FA012807D0F9
:10D250000523364AADF8043004212046F8F7A8FD2E
:10D26000BDF80430324A08212046F8F7A1FD012715
:10D27000D7E7224956F8270033F096FA0028DFD086
:10D28000CEE704602A884FF6F7739A42294A8CBF8A
:10D290000123002383724FF00801274B204688BFEB
:10D2A0001346264AF8F784FD2549404617F044FF07
:10D2B000FF280146307202D10022224948E71FB9F7
:10D2C000B37A002B7FF417AFBDF804201E4802EBA1
:10D2D00082120DF0F7FB00283FF40DAF204600222C
:10D2E0001A49FFF765FD3046FFF71AFD03E700BF57
:10D2F0009B5404009255040095550400CB5504003E
:10D300008E3D0400713E0400E3530400D555040033
:10D31000F3550400085604002B5604004E56040032
:10D320007256040033530400C03C040096560400B7
:10D33000CD5604008954040093540400E2560400BE
:10D3400009D80000F8560400FDDB0000C43E0400CC
:10D3500003292DE9F34104460D46904605D1836823
:10D36000D3F85463C6F3400646B1234AD8F80010F8
:10D370002046FFF7DDFC02B0BDE8F08108F02FFA8F
:10D38000074628B902461D492046FFF711FDF2E77E
:10D39000294608F029FB0DF106010546D8F80400DE
:10D3A000FFF7E0FC024638B915492046FFF700FDBB
:10D3B000384608F06BFADEE72946BDF8063021F85A
:10D3C000023BD8F8080000F0A7FF024608B90D4953
:10D3D000EBE7FFF791FC054610B902460A49E4E77E
:10D3E00004600A49384617F077FEFF282872C2D138
:10D3F00032460749D9E700BFD25A0400713E040003
:10D40000005B0400185B0400335304003DDA0000A5
:10D41000F856040001292DE9F34104460E469046D2
:10D4200005D08368D3F85453C5F3400545B1204A6D
:10D43000D8F800102046FFF77BFC02B0BDE8F08171
:10D44000022904D01B492A46FFF7B2FCF5E708F091
:10D45000C6F9074618B9024617492046F4E731468F
:10D4600008F0C2FA0DF106010646D8F80400FFF7ED
:10D4700079FC024638B911492046FFF799FC384635
:10D4800008F004FAD9E7BDF806303380FFF734FC22
:10D49000064610B902460A49EEE7046009493846D3
:10D4A00017F032FEFF283072C7D12A460649E3E75B
:10D4B000B25104008E3D0400713E0400E3530400A9
:10D4C00033530400A9D90000F856040038B50546C6
:10D4D000FFF7FEFB044678B90D4B5B88BBB10D4BE3
:10D4E0000D480E49C01AC00800042A4640F0010049
:10D4F000BDE83840F4F776BD2B460068084A0221A3
:10D50000F8F756FC2046BDE83840FFF709BC38BDA7
:10D510000C0500200C7E04004C7E0400A75B040078
:10D52000D15B0400014A0821F8F742BC38450400E9
:10D5300073B58368D3F85453C5F3400504462DB141
:10D5400000221146F9F7EEFD02B070BD012904D0AA
:10D5500012492A46FFF72CFCF6E768460DF014FE48
:10D56000684607F0C3FE4FF6FF739842064610D098
:10D57000C0F307230A4A20460821F8F719FC204681
:10D58000F3B2074A0821F8F713FC2046FFF7CAFF59
:10D59000DAE72A4603492046DCE700BF8E3D040057
:10D5A00051270400B15A04002DE9F04F8DB0074611
:10D5B00008F0C8F906460078FFF78AFB0446002801
:10D5C00000F0A28073780068002B40F09880F27819
:10D5D000237B9A4203D1504A0821F8F7E9FB96F8D9
:10D5E00003A03379D4F80080DFF858B15344059391
:10D5F000751D059B534525D8F5783279B3781544C8
:10D60000AB4273D9002A71D0384608F029FA0421B8
:10D61000384608F01AFBE389438005703F493846D5
:10D6200018F082FCFF28207209D101223C492068B1
:10D63000FFF7BEFB002F69D12046FFF771FB0DB04D
:10D64000BDE8F08F0DF11C092A461121484600F073
:10D650006FFF002803DC5946484633F0AFF800233B
:10D660008DF82C30B5F8093002932B7A2D4ACDE98C
:10D670000093082153464046F8F79AFBEB7A2A4A72
:10D6800008214046F8F794FBEB7A012B07D0032BD7
:10D6900014D0264A08214046F8F78AFB05E0AB89FA
:10D6A000234A08214046F8F783FB224A08214046D6
:10D6B000F8F77EFB0AF1010A15359AE705F10C022D
:10D6C0001121484600F034FF002803DC5946484643
:10D6D00033F074F800238DF82C302B7D0093164A1C
:10D6E0004B4608214046F8F763FBDEE72068134A03
:10D6F0000821F8F75DFB2068FFF714FF9AE7104A4E
:10D700000221F8F755FB95E7002F98D0384608F02E
:10D71000BDF8002C93D08FE7B0570400A9D50000C6
:10D720004D53040018580400355804006A5804008A
:10D7300045580400322F04005E580400835804004A
:10D74000AB58040007580400F7B5054608F0FAF88E
:10D75000077806463846FFF7BBFA044698B9224BCD
:10D760005B8853B12148224B2249C01AC0080004EB
:10D770003A4640F00100F4F735FC284603B0BDE816
:10D78000F04008F083B8002239461B480DF0BAF982
:10D7900063684BB9727820683378BAB1009202217D
:10D7A000164AF8F705FB18E0294620469847002856
:10D7B000F0D140F24512217A0F480DF083F980B183
:10D7C00001220F492068FFF7F3FA06E00D4A08210D
:10D7D000F8F7EEFA2068FFF7A5FE2046FFF7A0FA5B
:10D7E000CBE703B0F0BD00BF0C0500204C7E040069
:10D7F0000C7E0400A25F0400CDD40000E05F0400B2
:10D8000010600400C45F04002DE9F743064608F0E9
:10D8100099F819210546304608F017FA804628780D
:10D82000FFF756FA044620B36B7803BB144A00682E
:10D83000DFF850900821F8F7BBFA6F1D2B7943B938
:10D84000A37AB3B92068FFF76DFE2046FFF768FAA8
:10D850000FE017F8012BB8F80130009208214A4672
:10D860002068F8F7A5FA2B79013B2B71E6E7852BA9
:10D87000E8D0304603B0BDE8F04308F007B800BF79
:10D88000322F0400205704007FB5064608F05AF8EE
:10D8900005460078FFF71CFA044620B9304607F029
:10D8A000F5FF04B070BD0022FF211B480DF02AF9DE
:10D8B00020B1012219492068FFF77AFA6B7843BB3F
:10D8C000A91C02A80CF010FD022205F10A010DF1BD
:10D8D000060032F00EFA0DF105030122BDF8061024
:10D8E00002A807F01FFD034668B90822206801233B
:10D8F0000DEB020100F022FD2068FFF713FE204629
:10D90000FFF70EFACAE7064A20680221F8F750FA34
:10D91000F5E7044AF8E700BF1DCE0000503B0400C5
:10D92000FD5304003454040073B5064608F00AF8A9
:10D9300005460078FFF7CCF9044620B9304607F0D9
:10D94000A5FF02B070BD0022FF2113480DF0DAF8E8
:10D9500020B1012211492068FFF72AFA6B78A3B998
:10D96000022205F10A010DF1060032F0C2F9206829
:10D97000BDF806300A4A0821F8F71AFA2068FFF7BE
:10D98000D1FD2046FFF7CCF9D8E7064A20680221EE
:10D99000F8F70EFAF5E700BFF9CD0000503B0400A0
:10D9A0004B5A0400515A04002DE9F041074607F094
:10D9B000C9FF05460078FFF78BF9044620B93846C1
:10D9C000BDE8F04107F062BF6B78006833BB6B883D
:10D9D000154ADFF864800821F8F7EAF9134A20684D
:10D9E0000821F8F7E5F96E1D2A792068131D2B44EC
:10D9F000B3420CD822B11B780D4A0821F8F7D8F9A8
:10DA00002068FFF78FFD2046FFF78AF9D7E716F861
:10DA1000013B42460821F8F7CBF9E5E70122054929
:10DA2000FFF7C6F9EFE700BFD3510400E45104004B
:10DA3000C9370400EC510400E85104002DE9F04F0F
:10DA400087B0824607F07EFF06460078FFF740F970
:10DA5000054628B9504607B0BDE8F04F07F016BF9D
:10DA600073780068002B5CD1B27A7388F47A96F8E8
:10DA70000CB002F00F02039232890292F2880192F6
:10DA80007279009204F10048284A082108F1FF3811
:10DA9000F8F78EF906F10D07254A286808214FEAA4
:10DAA0004806F8F785F9BB190593B946059B286820
:10DAB0004B4528D82CB137F818301E4A0821F8F702
:10DAC00077F91D4A2868DFF8749008215C4404F156
:10DAD0000044F8F76DF90236013C3E4407EB440878
:10DAE000B045286816D8BBF1000F05D037F81430C0
:10DAF000104A0821F8F75CF92868FFF713FD28465B
:10DB0000FFF70EF9A6E739F8023B0C4A0821F8F7AF
:10DB10004FF9CBE736F8023B4A460821F8F748F9B7
:10DB2000DEE701220649FFF743F9E8E7295B040035
:10DB30007A5B0400905B0400995B0400875B04003F
:10DB4000EC510400F8B5074607F0FCFE06780546E0
:10DB50003046FFF7BDF8044690B1002231460D482B
:10DB60000CF0D0FF20B101220B492068FFF720F90B
:10DB70006B7820684BB9FFF7D5FC2046FFF7D0F84B
:10DB80003846BDE8F84007F081BE044A0221F8F7A4
:10DB90000FF9F2E741CE0000503B04007F5904002A
:10DBA00070B5054607F0CEFE06460078FFF790F800
:10DBB000044620B92846BDE8704007F067BE002241
:10DBC000FF210B480CF09EFF20B10122094920687B
:10DBD000FFF7EEF8737820682BB9FFF7A3FC204617
:10DBE000FFF79EF8E6E7044A0221F8F7E1F8F6E7C6
:10DBF000D5CD0000503B04006453040010B5FFF77E
:10DC000067F8044638B10068FFF78CFC2046BDE891
:10DC10001040FFF785B810BD2DE9F04F044685B0E0
:10DC200008460F4607F08EFE437806461BB10120DA
:10DC300005B0BDE8F08FC278237B9A4204D12B4A0D
:10DC400020680821F8F7B4F8DFF8A890DFF8A8A05A
:10DC5000DFF8A8B0751D00223179F37802F10108D0
:10DC6000D2B2914219D85D18B378AB42DFD90029FE
:10DC7000DDD0384607F0F4FE0421384607F0E5FF12
:10DC80000570E38943801A49384618F036F9A0F147
:10DC9000FF03207258425841CAE7134408214A46FC
:10DCA0002068F8F785F8012329460822206800F04B
:10DCB00045FB524608212068F8F77AF80822A9188F
:10DCC0000123206800F03AFB6A7D2B8A03922A7DAB
:10DCD0000292EA7C0192AA7C009208215A462068AE
:10DCE000F8F766F816354246B6E700BF1B5F04003A
:10DCF00049D700006E5F040016580400755F0400E9
:10DD000013B513468268D2F85423C2F34002044686
:10DD10002AB100221146F9F705FA02B010BD022916
:10DD200003D91149FFF744F8F7E718D103226946F0
:10DD3000586800F06DFC024660B168460DF01CFAB0
:10DD4000204601230822694600F0F8FA2046FFF732
:10DD5000E9FBE2E705492046FFF72AF8F0E76846C5
:10DD60000DF012FAECE700BF8E3D0400B253040040
:10DD700001292DE9F0410446164605D08368D3F801
:10DD80005453C5F3400535B131682D4A2046BDE8EE
:10DD9000F041FEF7CDBF022905D02A492A46BDE849
:10DDA000F041FFF705B807F01AFD074618B902461B
:10DDB00025492046F3E70C2107F047FF0322811C89
:10DDC0008046706800F024FC024640B91F49204696
:10DDD000FEF7EEFF3846BDE8F04107F057BDFEF70D
:10DDE0008BFF064610B902461949F0E74FF6FF735C
:10DDF000A8F80030A8F80A5016490460384616F012
:10DE00008FFFFF280146307208D120462A4612496A
:10DE1000FEF7CEFF3046FEF783FFDBE740F2451208
:10DE20000E480CF04FFE48B120462A460C49FEF73A
:10DE3000BFFF3046BDE8F041FEF772BFBDE8F0819C
:10DE4000415A04008E3D0400713E0400B2530400A8
:10DE50003353040029D900004D530400F9CD0000CC
:10DE6000C43E040001292DE9F04705468946904645
:10DE700006D08368D3F85433C3F3400A9B0707D511
:10DE8000D8F800102E4A2846BDE8F047FEF750BFEC
:10DE900007F0A5FC064630B902462A492846BDE8E7
:10DEA000F047FEF785BF042107F0CFFE022281185C
:10DEB0000746D8F8040000F0ABFB044650B92249ED
:10DEC00002462846FEF774FF304607F0DFFC8CBBA5
:10DED000BDE8F087B9F1020F09D93946D8F8080032
:10DEE00000F01AFA044620B902461849E9E787F813
:10DEF00000A0FEF701FF044610B902461449E0E70E
:10DF0000144B056043601449304617F0F6FFFF28B4
:10DF10000146207202D100221049D2E740F2451298
:10DF20000F480CF0CFFD0028D2D000220D49284622
:10DF3000FEF73EFF2046BDE8F047FEF7F1BE00BF0A
:10DF4000CB590400E5590400075A04002B5A040079
:10DF50003353040019DC000049D700004D5304007E
:10DF6000CDD400001060040001292DE9F8430546D6
:10DF70000E46914609D08368D3F85473C7F340071F
:10DF80005FFA87F8B8F1000F07D0D9F80010304ACF
:10DF90002846BDE8F843FEF7CBBEFEF7ADFE0446CB
:10DFA00030B902462B492846BDE8F843FEF700BFCA
:10DFB000012905601DD9022200F10E01D9F80400E3
:10DFC00000F026FB024640B923492846FEF7F0FE42
:10DFD0002046BDE8F843FEF7A3BE022E0CD004F1A4
:10DFE0000C01D9F8080000F097F9024660B91B4906
:10DFF000EBE742461A49E8E7277307F0F0FB0646CD
:10E0000038B902461749E0E7032EF6D042461649D2
:10E01000DBE7042107F019FE04220746002131F056
:10E020008CFE237B3B70E3897B801049304617F0E0
:10E030007BFFFF28207208D1284600220C49FEF7FA
:10E04000B7FE304607F022FCC2E7BDE8F88300BF08
:10E050003657040033530400505704007E57040021
:10E0600063570400713E040094570400A9D50000D2
:10E070004D5304002DE9F04F012985B005460E46A9
:10E08000174605D08368D3F85443C4F340043CB129
:10E09000494A39682846FEF74BFE05B0BDE8F08FC7
:10E0A00007F09DFB804628B9024644492846FEF702
:10E0B0007FFEF2E70B2107F0C8FD0B2221468146C7
:10E0C00031F03BFE012E0AD83D4922462846FEF794
:10E0D0006FFE404607F0DAFB002C69D1DDE70DF159
:10E0E0000E017868FEF73EFE044610B90246354937
:10E0F000ECE7BDF80E30A9F80830022E07D1FEF784
:10E10000FBFD044600283AD102462F49DEE7B868F5
:10E1100003782D2B1DD00322494600F079FA0446DE
:10E12000C8B10324DFF8BCA0DFF8BCB0A642E6D932
:10E1300057F8243001931846514632F035FB019BC5
:10E1400060B999F80A3043F0400389F80A30013485
:10E15000ECE70224E6E702461C49B7E759461846B1
:10E1600032F022FB20B999F80A3043F08003ECE743
:10E17000002217492846FEF71BFE0024A9E7056088
:10E180001449404617F074FFFF280146207202D15F
:10E19000002211499AE740F2451210480CF092FC17
:10E1A00000283FF47AAF00220D492846FEF700FE12
:10E1B0002046FEF7B5FD70E7DE580400713E04000E
:10E1C0002459040050570400335304003F590400FD
:10E1D0006C59040045DB00004D53040041CE0000A3
:10E1E000C43E04005859040063590400F8B5094EB0
:10E1F000094CA41B0746A4080025AC4201D100200D
:10E20000F8BD56F82530384698470128F8D0013532
:10E21000F3E700BFFC7D04000C7E040073B50E46DE
:10E220001C460546002863D0002B61D0212A46D029
:10E2300014D8102A2ED008D8092A40D00B2A16D07C
:10E24000082A33D013462C4A32E0192A37D001D895
:10E25000182AF6E71B2A0AD0202AF2E72B2A33D005
:10E2600008D8282A27D0292A2BD0232AEAD12368A4
:10E27000224A1DE0312A22D001D8302AE1E7422A81
:10E2800025D0F02ADED1012300932246082300F096
:10E2900025F926E01C781A4A1A4B002C18BF1346A1
:10E2A000194A02B0BDE8704032F0CEB92378174A5F
:10E2B00031462846F5E793F90030154AF1E72388FF
:10E2C000F5E7B3F90030F8E71B68124AE9E7187878
:10E2D00088420DD26A1E191B884204DC00232B548D
:10E2E000013002B070BD13F8011F02F8011FF2E700
:10E2F0004FF0FF30F5E700BF57600400A858040056
:10E300004C6004005160040037310400373E0400C3
:10E31000C03C0400534C040013B50C4601AA064946
:10E3200032F0C6F928B1019BFF2B9ABF2370012060
:10E33000002002B010BD00BFA85804002DE9F04F26
:10E340004FF00208012418FB024483B09146E21DFD
:10E350009B46D2086B46A3EBC20302AF9D4602ADBB
:10E3600006468A4622460021284631F0E6FC4B4606
:10E3700052462146CDF800B0284600F0AFF80028FC
:10E38000BBBF074B074A074A4146A4BF2B4608219B
:10E390003046F7F70DFD0437BD46BDE8F08F00BFEE
:10E3A0003460040037310400022015F089BA0000FF
:10E3B00010B50F4C2378D3B10022FF210D480CF08B
:10E3C000A1FB0D4B88B918700C4B20705B88022B99
:10E3D0000DD90B480B4B0C49C01AC008000440F083
:10E3E0000300BDE81040F3F7F9BD01221A7010BD1B
:10E3F000E9820020A9E30000EA8200200C05002049
:10E400004C7E04000C7E04009560040008B512F0F8
:10E41000DBFBE8B90F4B1B78D3B10F4B0F4A1870D9
:10E420001378ABB9012111700D4A13700D4A1370A6
:10E430000D4B5B88022B0BD90C4B0D480D49C01AB4
:10E44000C008000440F00300BDE80840F3F7C6BD73
:10E4500008BD00BFEC820020E8820020E982002095
:10E46000EA820020EB8200200C0500200C7E0400D4
:10E470004C7E04007360040007B500BB124B0C22F5
:10E48000C3F818270A22D3F81015013AC1F38011F6
:10E490000191F8D1019B73B90C4B5B88022B09D910
:10E4A0000B480C4B0C49C01AC008000440F0030094
:10E4B000F3F794FD0120044B0222C3F8182703B0A0
:10E4C0005DF804EB0CF074BE000300500C05002056
:10E4D0004C7E04000C7E0400426604002DE9F84FD7
:10E4E0001C469DF8283080468946924663B1661ED8
:10E4F000002BDFF838B014BF4FF0FF37012700259D
:10E5000024B92846BDE8F88F1E46F1E71AF8063010
:10E510005A46A9EB050108EB050032F095F80028F2
:10E52000F0DB013C05443E44E4B2E9E75127040036
:10E5300007B5012300930823FFF7D0FF03B05DF870
:10E5400004FB03463038C0B209280DD9A3F161029B
:10E55000052A02D8573BD8B27047A3F14102052AD9
:10E5600001D8373BF7E7FF2070472DE9F843022930
:10E5700005460C46164699469DF8207013D9037837
:10E58000302B10D190F8018031F084FB404441469B
:10E59000407800F00300012808BF2031782902BF2D
:10E5A000023CE4B20235B7B1631E1D444FF0FF38A0
:10E5B000B4EB490F2ADC4A460021304631F0BDFB5E
:10E5C0004FF000095FFA89F18C4207D8631A58426C
:10E5D0005841BDE8F8834FF00108E9E72878FFF7D4
:10E5E000B0FF0F28F2D8CA070BD596F9003007B153
:10E5F000000140B2184306F8010B454409F1010936
:10E60000E0E70FB90001C0B23070F6E70020E0E7A4
:10E610002DE9F34104468846164632F0D7F8054600
:10E6200024B90026304602B0BDE8F081B8F1000FF1
:10E63000F7D0204632F0CAF80028F2D02378302BE9
:10E640000ED1677831F026FB38443B46427802F021
:10E650000302012A08BF2033782B04BF0234023D95
:10E66000102D05D106F0FD06012EDAD1032605E0B6
:10E67000042DD6D1013E012ED3D8022601230093CA
:10E680004246C5F34703E9B22046FFF76EFF002874
:10E69000C8D1C6E72DE9F0438BB00AA9002341F8A1
:10E6A000203D074612F0D8FC8046384607F04EFB66
:10E6B00005460CF0A5FDA14E0446B8F1140F00F27A
:10E6C0000383DFE818F01C007A005C02F701010305
:10E6D0009000CD006501B601A30201031C001102E8
:10E6E000010301030103150095026A023302D502FA
:10E6F000934CB4F8028075B1B8F1020F01D801252E
:10E700006FE09048904B9149C01AC00800042A4617
:10E7100040F00300A1E01122294605A8029F31F034
:10E720000CFBB8F1020F09D98648874B8849C01AFB
:10E73000C008000440F00300F3F750FC07F110029A
:10E74000112105A8FFF7F4FE002803DA814905A886
:10E7500032F034F86388022B0DD905A8F3F776FA66
:10E76000794A784B7C499B1ADB081B04024643F02C
:10E770000300F3F737FCF8680CF0C8FCF8680CF0FD
:10E78000D7FC6388022B0AD96E486F4BFA6873492D
:10E79000C01AC008000440F00300F3F723FC6388AC
:10E7A000022BACD96748684B6D49C01AC0080004F9
:10E7B00040F00300F3F712FCA1E701233370604B34
:10E7C0005B88022B09D95F485F4B6649C01AC008B5
:10E7D000000440F00300F3F701FC002015F070F88E
:10E7E0000546002484E0564F7A88022A09D9554804
:10E7F000554B5D49C01AC008000440F00300F3F710
:10E80000EDFB7B88EDB974B1022B09D94D484E4B15
:10E810005649C01AC008000440F00300F3F7DEFBBD
:10E82000FFF7F4FD6BE7022B09D94648464B5049E8
:10E83000C01AC008000440F00300F3F7CFFB042027
:10E84000CCE7002B3FF45BAF3E483F4B4949C01A31
:10E85000C00800042A4640F00100F3F7C3FB4EE76E
:10E86000374F5DBB1122294605A831F066FA03A88F
:10E870000CF098FC03AA112105A8FFF759FE002807
:10E8800003DA344905A831F099FFFFF791FD7B8841
:10E89000022B7FF634AF05A8F3F7D8F9294C0546CB
:10E8A00001F0E6FA284B3449E41AE40843882404CA
:10E8B0002A4644F00300F3F79FFB20E77B8840B132
:10E8C000022BADD91F48204B2C49C01AC0080004A8
:10E8D000A2E7002B3FF413AF1A481B4B2849C01A7C
:10E8E000C00800042A4640F00100F3F77BFB012535
:10E8F0003378C3B123490B78ABB1234B1A78002A84
:10E9000000F0F28100221A700D4B0A705B88022B16
:10E9100009D90C480C4B1D49C01AC008000440F02E
:10E920000300F3F75BFB24B915F1FF3418BF4FF078
:10E93000FF3420460BB0BDE8F08300BFEC8200201E
:10E940000C0500204C7E04000C7E0400B76004001F
:10E95000F76004001D6104002561040037610400B4
:10E960004B6104007861040091610400B36104000C
:10E97000CA610400E26104001162040065620400DF
:10E9800098620400E9820020EA8200209560040079
:10E99000A54F75BB1122294605A831F0CEF903A871
:10E9A0000CF000FC03AA112105A8FFF7C1FD002807
:10E9B00003DA9E4905A831F001FF7B88022B11D9AB
:10E9C00005A8F3F743F99A4D074601F051FA994B20
:10E9D0009949ED1AED082D0443883A4645F00300A5
:10E9E000F3F70AFB0CB1FFF7E3FC002004F070FB27
:10E9F00085E67B8878B1022B0AD98D488D4B8F49EB
:10EA0000C01AC00800042A4640F00300F3F7EAFAEF
:10EA1000FFF7FCFCE9E7022BE7D98548854B8849DD
:10EA2000C01AC00800042A4640F00300F3F7DAFADF
:10EA3000DBE77D4C4DBB1122294605A831F07DF95D
:10EA400003A80CF0AFFB03AA112105A8FFF770FD86
:10EA5000002803DA754905A831F0B0FE6388022B5F
:10EA600011D905A8F3F7F2F8714C054601F000FA48
:10EA7000704B7449E41AE408240443882A4644F09D
:10EA80000300F3F7B9FA0220A8E66388022B0AD93B
:10EA90006748684B6C49C01AC00800042A4640F019
:10EAA0000300F3F79FFA4122042168480CF00AF8AA
:10EAB00004461CE75C4B5B8855B9022BA8D95D4B1B
:10EAC0005B486349C01A029BC00800041A799BE79F
:10EAD000002B8AD05648574B5E49C01AC008000424
:10EAE0002A4640F00100A1E7029D1122002105A85D
:10EAF00031F023F92A1D112105A8FFF719FD00287F
:10EB000003DA4A4905A831F059FE474B5B88022BCE
:10EB10007FF6F5AD05A8F3F799F8454C454B4E49FE
:10EB2000E41AE40824042B7B0246C2E6029D11226B
:10EB3000002105A831F001F92A1D112105A8FFF7D0
:10EB4000F7FC002803DA394905A831F037FE364BC7
:10EB50005B88022B7FF6D3AD05A8AF89344CF3F761
:10EB600075F8344B3D49E41AE408AB7B0093240468
:10EB700003463A4644F00300F3F748FABFE52A4B50
:10EB80005B88022B7FF6BBAD2A4B29483449C01A5B
:10EB9000029BC00800049A88BAE5029D1122002158
:10EBA00005A831F0CAF82A1D112105A8FFF7C0FCFD
:10EBB000002803DA1D4905A831F000FE1A4B5B88D6
:10EBC000022B7FF69CAD05A8AF89194CF3F73EF8F0
:10EBD000184B2449E41AEB7B0193E408AB7B0093C8
:10EBE000240403463A4644F00300F3F71BFA86E593
:10EBF0000D4B5B88012B7FF682AD0D480D4B1A49FA
:10EC0000C01AC008000440F00200D3E5064B5B8840
:10EC1000022B7FF674AD0648064B1449C01AC00893
:10EC200000042A4674E500BF0C0500201D610400A5
:10EC30004C7E04000C7E0400D86204001B630400B8
:10EC40004C63040087630400E2630400C1380200DF
:10EC5000F335040011360400096404003C64040028
:10EC60007A640400AF640400206504003665040083
:10EC70003F4D6A88022A09D93E483F4B3F49C01A96
:10EC8000C008000440F00300F3F7A8F906F0A7FD60
:10EC9000044650B1394606F076FE0421204606F0BF
:10ECA0001CFF204604F05AFA29E56B88002B3FF43C
:10ECB00026AD314B2F483249C01AC008000440F03D
:10ECC0000100F3F78BF912E6294B5B88022B7FF6E4
:10ECD00016AD294B27482B49C01AC00800042B4603
:10ECE000424640F00300E6E5274F3B78002B7FF4D7
:10ECF0001AAE264926480B7801229A40B2F5617F68
:10ED0000DCBF01330B70234BC8BF4FF461725A4311
:10ED100000214FF47053B2FBF3F20BF0D3FEC0F1BD
:10ED200000098046B9F1000F1FD0114B5B889BB1E1
:10ED30004846F3F70DFC0F4E0F4B1749F61AF6082D
:10ED40004FF43B7336040193144B00934A46034639
:10ED500046F00100F3F766F9F2F7B4FF0028FBD1A3
:10ED6000C8F59C402030F4F7EDF801233B70DAE55C
:10ED70000C0500204C7E04000C7E0400616504003C
:10ED800091650400D2650400E8820020EB82002037
:10ED9000A9E3000040420F0036360400006604007C
:10EDA00073B50D4602A9002341F8043D064612F052
:10EDB00053F90446304606F0C9FF032C09D006D3A8
:10EDC000063C012C03D820B92846F3F715FB02B006
:10EDD00070BD2846F3F724FBF9E700002DE9F8435E
:10EDE0001E4C074691461E46884602F0EBFDB4F8DD
:10EDF00062583423F201022F25F0070542EA880207
:10EE000084F865384FF0120334BF4FF0020E4FF014
:10EE1000000E3D4342EAC90284F86638002F4FF0E5
:10EE20006C034EEA020205F0E70584F8673842F603
:10EE3000414318BF4FF4305345EAC02084F864289A
:10EE4000A4F86A387F220023A4F86208A4F868288E
:10EE5000A4F86C2884F86E38BDE8F883CC8C0020C8
:10EE600030B40B4DB5F86F4824F00F04204320F068
:10EE7000F00040EA011020F4706040EA0220C0F384
:10EE80000B0040EA0330A5F86F0830BC10F0D6BB89
:10EE9000CC8C002070B583798B4205460C46164613
:10EEA00004D8BA214FF4496007F0C2FA043425F8B7
:10EEB000146070BD70B5C3798B4205460C4616468A
:10EEC00004D8C8214FF4496007F0B2FAAB791C446A
:10EED000043425F8146070BD70B51C4D1C4E95F8B7
:10EEE00076280023082102F0F00285F8771863F3F2
:10EEF0000712092185F87138A5F87238A5F8743819
:10EF000085F8781885F8762885F8B4381C4605F613
:10EF1000710536F81420E1B228460134FFF7BAFF34
:10EF2000082CF6D10B4E0C4D0024325DE1B2284680
:10EF30000134FFF7BFFF092CF7D10C23032207216F
:10EF40000020BDE87040FFF78BBF00BFCC8C0020D5
:10EF500078660400886604003D950020031C4FF08D
:10EF6000010218BF01231146FFF738BF08B50A4B4D
:10EF700093F8D521003218BF012211460123022047
:10EF8000FFF72CFF01220C2311460020FFF768FF3A
:10EF9000BDE80840FFF7A0BFCC8C002007B50F4BA1
:10EFA00093F8B428052A0AD8511C83F8B41803EB47
:10EFB0008203C3F89C08002003B05DF804FB04231F
:10EFC000019200934FF0FF3040F239134FF4496241
:10EFD00001210BF071FF6FF01C00EDE7CC8C0020DD
:10EFE0002DE9F7430CF0AAF90DF0A2F943681B785C
:10EFF0000193042300934FF4496240F24713012127
:10F000004FF0FF300BF058FF00260DF091F94368E8
:10F010001B78F4B2A3420CD80CF0B4F900286CD1E0
:10F0200040F261114FF4496003B0BDE8F04307F0CE
:10F03000FFB90DF07DF94368D3F8013053F824305F
:10F04000D3F81500FFF7AAFF0DF072F9D0F8AC3035
:10F05000A50063B10DF06CF9D0F8AC700DF068F953
:10F060004368D3F8013053F824301878B8470027A4
:10F070000DF05EF94368D3F801305B591B7CFCB29C
:10F08000A34201D80136C0E70DF052F94368D3F826
:10F0900001305B59D3F81130C4EB04142344D3F886
:10F0A0000B305BB10DF044F94368D3F801305B5984
:10F0B000D3F811302344D3F80B3098470DF038F9CA
:10F0C0004368D3F801305B5993F800800DF030F9B4
:10F0D0004368D3F801305B59B3F801900DF028F97B
:10F0E0004368D3F801305B59D3F8112049462244D4
:10F0F00040460FF0E1FD0137BAE703B0BDE8F08309
:10F1000073B5044606F01EFC43780BB9458845B13B
:10F1100000231D4800931A4621460BF06FFA02B0F7
:10F1200070BD8389194EB3F5285F0BD214230E20CE
:10F1300086F8F83309F02AFA204602B0BDE870409C
:10F1400014F024B81B0A0E2086F8F83309F01EFAD2
:10F1500096F8402412F0010311D096F868340C4858
:10F1600065F3030340F24512294686F868340BF034
:10F17000DBFA00952B461A4621460648CDE7D20613
:10F18000DAD50093F7E700BF99F10000CC8C00209E
:10F1900039F30000817D0200064B93F869246FF378
:10F1A000861283F8692401460A220C2083F84B2436
:10F1B00014F06CBBCC8C0020F0B528218DB0054636
:10F1C00006F043FD02AA034600F12807144618681A
:10F1D0005968164603C60833BB423246F7D120466B
:10F1E00003F002F99DF823600EB9012824D1102103
:10F1F000284606F02AFD08220746DEB109A930F0AC
:10F2000078FD08222146B81830F073FD00230093E2
:10F210001A46294612480BF0F1F9124B83F86C5448
:10F22000204612F045FE01221146204612F018FE3B
:10F230000DB0F0BD2146E2E70A21284606F005FDA3
:10F2400021460746082230F054FD01233B727E72AE
:10F25000334600963246294603480BF0CFF9DFE7E4
:10F2600069150300CC8C0020D126010010B50C4696
:10F27000282106F0EAFC0822214630F02BFDB0FAE6
:10F2800080F0400910BD000038B5054620B90D4892
:10F29000BDE8384006F0CBBA0B4A92F8693443F027
:10F2A000400382F86934022106F09EFB00240470BA
:10F2B00044700649284615F08FFE2046BDE83840C8
:10F2C00017F012BF89F20000CC8C002001F1000081
:10F2D00013B5044628B9144802B0BDE8104006F042
:10F2E000A6BA124991F868345A1C02F00F0262F370
:10F2F000030381F86834C3F303139A4208DD002343
:10F3000001460B4800931A460BF078F902B010BD85
:10F3100040F24512002104480BF006FA0023009346
:10F320001A4621460348EFE7D1F20000CC8C0020BA
:10F3300099F10000057C020013B5044628B9144871
:10F3400002B0BDE8104006F072BA124991F8683474
:10F350005A1C02F00F0262F3030381F86834C3F30E
:10F3600003139A4208DD002301460B4800931A4616
:10F370000BF044F902B010BD40F2451200210448E0
:10F380000BF0D2F9002300931A4621460348EFE719
:10F3900039F30000CC8C002099F10000817D02003F
:10F3A00010B51D4C30220021204630F0C6FCA4F5DB
:10F3B0008860627890F84034012143F0220361F3C1
:10F3C000010261F38713D2B242F0040203F0FE039C
:10F3D00062706FF3C3034FF6FF7280F840342281EE
:10F3E0004FF474730E22A2726362B4220B4BE2617B
:10F3F00063610522236194F8283084F820200322D9
:10F4000062F3071384F8283094F8293043F030036E
:10F4100084F8293010BD00BF0C91002000F8FF07D0
:10F42000064A92F84034D80707D592F86914C907FC
:10F430005CBF43F0100382F840347047CC8C00204E
:10F44000FFF7EEBF13B50E4B93F868246FF303027A
:10F4500083F868240022044611460A480BF052FB48
:10F4600040F24512002108480BF05EF9002300939A
:10F470001A46214605480BF0C1F802B010BD00BF86
:10F48000CC8C002039F30000D1F20000057C020092
:10F4900007B5002101AA04480BF0BAFBB0FA80F0CE
:10F4A000400903B05DF804FBD1F20000002210B562
:10F4B000114604460B480BF025FB002211460A4872
:10F4C0000BF020FB094B93F869246FF386120020A0
:10F4D00083F8692417F04CFE21460D20BDE810404A
:10F4E00014F0D4B939F30000D1F20000CC8C002024
:10F4F00037B5CCB22146054606F045FA0023009305
:10F500001A46214606480BF079F8064B0648D3F810
:10F510006424294603B0BDE830400BF005B900BFB4
:10F520009D430100CC8C0020B9F1000037B50446A2
:10F5300068460D4605F028FB6A46064920460BF052
:10F5400085FB00220446294603480BF0DBFA2046DF
:10F5500003B030BD6DF200007507020030B589B010
:10F56000054606F0EFF906AC411C0822204630F0B3
:10F57000C0FB002211460DF11303204605F084FE66
:10F580000146D0B905AA9DF8130002F047FB9DF88B
:10F59000132018BB059B5B7803F00C03042B1DD1D3
:10F5A0000121104611F0EEF80E4B002283F86C2476
:10F5B000284606F06BF909B030BD94E8030001ABB2
:10F5C00083E803000823009340F69D124FF4EB7389
:10F5D00001214FF0FF300BF06FFCE9E7104600F01F
:10F5E0007FFDE1E7CC8C0020034B93F8402460F3CF
:10F5F000C30283F840247047CC8C0020032898BFB6
:10F600000E4B73B594BF1D5C03250E462A464FF67C
:10F61000FF7130460AF00AFE0222044671190DF10C
:10F62000060030F066FBE443BDF80600A4B2001B00
:10F6300018BF4FF0FF3002B070BD00BF91660400EC
:10F6400073B505460E46FFF7D9FF044680B9032D72
:10F6500098BF0E4B0E4896BF5A5D052202323146C6
:10F6600030F047FB0B4B83F83A54204602B070BD94
:10F670000023009340F2D712A22301214FF0FF3064
:10F680000BF01AFC6FF03104EFE700BF9166040045
:10F69000F4900020CC8C0020094991F83A34037092
:10F6A00000231A468818013290F82804002808BF61
:10F6B0000133122AF6D1122B024808BF00207047EE
:10F6C000CC8C0020F4900020F0B5374C95B000238E
:10F6D0008DF81B3094F8BD339B0607460D460AD5BE
:10F6E00007AA0DF11B0108F09BF9013032D16FF030
:10F6F0001B0015B0F0BD0146082204F5737030F010
:10F70000E9FAF0B90DF11B00FFF7C6FF0646002825
:10F71000EDD031469DF81B00FFF770FF01ACD8B16A
:10F7200038687968234603C3082300934FF0FF30FD
:10F73000832340F2D71201210BF0BEFB6FF02B00A8
:10F74000D7E70822194904F5737030F0C3FA00288E
:10F75000D8D0CCE707AEDCE79DF81B30032B9BBF6E
:10F76000134AD15C052102310CAA304604F0F1FBAA
:10F77000102228460CA930F0BCFA2A462346103540
:10F78000106851681C4603C40832AA422346F7D1C8
:10F79000102300934FF0FF305C2340F2D712012179
:10F7A0000BF08AFB0020A4E7CC8C0020A1660400AB
:10F7B0009166040008B5F3F73DFA024B012283F885
:10F7C000282108BD00A00020034B93F828310BB975
:10F7D000FFF7F0BF704700BF00A00020024B0122DE
:10F7E0009A75F3F75FBA00BF00A000200148F3F755
:10F7F00043BA00BFFD9D0020034B9A7D012AFCD037
:10F8000093F817310370704700A0002010B50B4B20
:10F81000044693F84600F3F763FA64B9F2F7DAFEA8
:10F82000074B9C68F2F7D4FE14F0FF0005D1BDE849
:10F830001040F3F75ABA0120F9E710BDC49D00202B
:10F8400000A00020F7B5124C012506460F46F2F73E
:10F85000C1FEA560F2F7BCFE0E4B304693F8373080
:10F8600004F117023946F3F753FA064668B90090D7
:10F870004FF4937346F67A6229464FF0FF300BF04F
:10F880001BFBE56025602575A66003B0F0BD00BFD9
:10F8900000A00020C49D00202DE9F0411E4D074628
:10F8A0000E46F2F797FEAC68F2F792FE14F0FF04F2
:10F8B000A84605D00123EB602B602B75BDE8F081D5
:10F8C000032E85F818410DD11621384606F0BDF9F2
:10F8D0000468837C002C08BF0426DB075CBF03237D
:10F8E00085F81831384606F037F80230C0B288F88B
:10F8F0001700384606F026F80546384606F02CF87C
:10F9000029460246054830F0F4F921463046BDE864
:10F91000F041FFF797BF00BF00A0002018A0002013
:10F92000044B9A7D012A02BF00229A7583F81701C1
:10F93000704700BF00A000202DE9F041194C1A4D7E
:10F940004FF00008012607462E60C4F80C80F2F73D
:10F9500045FEC4F81C01C4F8088094F818216AB167
:10F9600094F81831013BDBB24146042084F8183189
:10F97000FFF768FF00232B60BDE8F0812660267545
:10F98000002FF7D07A78D20644BF0322C4F8302182
:10F9900038464FF0000258BFC4F83061E260F3F718
:10F9A000E3F9E7E700A000209899002073B504234D
:10F9B00001240E4D019006460093214640F27D132E
:10F9C00046F67A624FF0FF302C600BF075FA084B68
:10F9D00000219960D3F8242129602244C3F824210E
:10F9E000DE601C601C7502B070BD00BF98990020DD
:10F9F00000A000202DE9F74F2B4D2C4C99460123F8
:10FA00002B60E36D042B06468A46934644D8A36DCB
:10FA100004F16007DF423FD090F80080A8F10902AE
:10FA2000762A07D94FF4CC7146F67A60019306F036
:10FA3000FFFC019BDF5D4146384605F0D5FF42469D
:10FA4000711C30F056F9384605F08DFF00F802BC05
:10FA5000384605F088FF042100F801AC384606F06E
:10FA6000F4F8EB21C0F80090384606F077F9A36D62
:10FA7000E16D01330522B3FBF2F202EB82029B1A25
:10FA80000131A3650A4BE165012204295A601A7508
:10FA900002D90020F3F71FF93046F3F765F9002388
:10FAA0002B6003B0BDE8F08F98990020C49D002022
:10FAB00000A0002008B5F3F7EDF900280CBFE720FF
:10FAC000002008BD034A92F8ED3243F0020382F8A9
:10FAD000ED327047CC8C0020F0B585B004AE4FF607
:10FAE000FE730D2126F8023D074605F07DFF002537
:10FAF00053230222044603704570827031460B3056
:10FB000030F0F7F8054BC4F803302A4600952B4631
:10FB1000394603480AF072FD05B0F0BD25FB000030
:10FB20005D4E030013B50C21044605F05DFF46232E
:10FB300003700122002343708270C372C37003718B
:10FB4000437183711A460093214602480AF056FD1C
:10FB500002B010BD5D4E0300F0B5192189B0054615
:10FB600006F073F801AA034600F118071646186854
:10FB70005968144603C40833BB422246F7D11B78A8
:10FB800023701621284606F063F831460822044601
:10FB900030F0AFF803AB03CBA060E160BDF81430E8
:10FBA00023829DF81A30A27C104803F00F0363F300
:10FBB0000402A2749DF81A30D2B2C3F3011363F3A6
:10FBC0004612A2749DF81A30E27C9B0963F3461238
:10FBD000E2749DF81B3023759DF81C306375032279
:10FBE00029460AF0A1FD09B0F0BD00BF814803001D
:10FBF000F7B50F4609211446054606F026F8FF2CF6
:10FC000006460DD10822002130F097F80023377204
:10FC10001A460093294604480AF0F0FC03B0F0BDF0
:10FC2000214604F0B1FFF1E79D1A020073B50E46BC
:10FC3000044628B940F26A6140F2471006F0F8FB2A
:10FC4000F6B231462046002505F09DFE20461021E3
:10FC500006F03FF82B462A463146009508480AF040
:10FC6000CDFC0721204605F0F0FFFF2383712A46D3
:10FC700000952B46214603480AF0C0FC02B070BD37
:10FC800071150100750E010010B5064C94F81C2387
:10FC900094F81D13FFF7ACFF94F81C03BDE8104067
:10FCA00005F088B8CC8C0020F7B5124C1746B4F894
:10FCB000C8314A889A4206460D4616D1072105F0FA
:10FCC000C4FFAB88038013238370B4F8C831A0F855
:10FCD0000330FF238371002347711A460093314696
:10FCE00005480AF08BFC03B0F0BD03B0BDE8F0405E
:10FCF00005F0CCBDCC8C0020152B010030B504469E
:10FD000085B0104600220D460DF10F03114605F097
:10FD1000E3F990B99DF80F1041EA052144B1009034
:10FD20000B460122214608480AF068FC05B030BDA8
:10FD30002246054805F097FDF8E7002CF6D020464E
:10FD400005F0A4FDF2E700BFF9FE0000F8B5384C5D
:10FD500043F60953A4F8D430022384F8D73094F83A
:10FD60008E310F22002584F83A2184F88C2103F08B
:10FD7000EF03032243F00B0384F88D210746FF268F
:10FD80001022294604F23F1084F88E3184F88461F1
:10FD900084F8855184F88651C4F888512FF0CDFF3E
:10FDA00094F88F3184F84F5165F3C71384F88F317D
:10FDB0004FF6FF7384F82252A4F83431A4F8C83106
:10FDC000A4F8CA310FB184F8D53194F88E3184F893
:10FDD000D4616FF3820384F88E314FB10123082080
:10FDE00084F8AE3109F0F0FE09F0FAFE09F0F2FEF7
:10FDF0001C2200210F482FF0A0FF94F8ED220023D1
:10FE000063F3410284F8ED2294F8382384F8AF318B
:10FE1000A4F87C3184F8E13063F3C712FF2384F83F
:10FE2000382384F8D931BDE8F84001F0A9BD00BFFE
:10FE3000CC8C00205E8E002008B50120FFF786FFE5
:10FE400001F0FEFD27F01CFE074B084893F838230D
:10FE50006FF3000283F83823002140F24922BDE805
:10FE600008400AF061BC00BFCC8C0020C5FA00003D
:10FE700000487047948E0020F0B5104B104AD3F81C
:10FE80008051167800210E2707FB01F2B14205EBE5
:10FE9000020400D3F0BDAA5C12F0010F03D0B4F845
:10FEA00002E0864501D00131EEE76FF300022270D7
:10FEB00093F88421013A83F88421F0BDCC8C002092
:10FEC000F000002010B50C46511C05F02AFE00F889
:10FED000014B10BDE9280DD004D8DA2808D0E1285C
:10FEE00008D07047A0F1F003012B98BF062070479F
:10FEF000D3207047092070477FB50D460421064680
:10FF000005F0A3FE0446280AFFF7E4FFE9B22070DB
:10FF10000DF10E0004F07AFEBDF80E30A4F80130A9
:10FF2000002300931A46314602480AF067FB04B0EA
:10FF300070BD00BFCD18020013B50E4B93F84C24D2
:10FF4000D207044603D493F8D831072B0CD10020F4
:10FF500017F0A2F80123009300231A462146064811
:10FF60000AF04CFB02B010BD02B0BDE8104005F035
:10FF70008DBC00BFCC8C0020290D010037B50028B6
:10FF800038D01D4B93F8E822824233D1002283F807
:10FF9000E822D3F8E422916861B310681044013973
:10FFA000047B9160D3F8E452144A29681268013145
:10FFB0005208B1FBF2F002FB10122A6083F8E8420B
:10FFC00004230093019440F2AF6340F247120121F1
:10FFD0004FF0FF300AF070FF2CB94FF4D66140F2B9
:10FFE000471006F025FA002300931A4621460448DC
:10FFF0000AF004FB03B030BDCC8C0020F4000020DC
:020000021000EC
:1000000079010300044A92F8E83223B9034B1B68D4
:10001000013382F8E8327047CC8C0020F4000020D5
:10002000024B18680130C0B2FFF7A8BFF4000020EF
:1000300073B500230193044680884FF6F773984206
:100040000E461ED86378C3F30012EAB11B074CBFFB
:1000500004F1100504F1080501460DF10303002227
:10006000284605F05FF960B90A4B93F8D53143B1E2
:10007000A388B34205D101AA01219DF8030001F034
:10008000CDFD019802B070BD0DF10303012105F013
:1000900023F8E8E7CC8C0020F0B5104B93F86822E9
:1000A000DAB10026314680B201F1880503EB8505FF
:1000B000EC7AE7070BD503EB8107B7F82872874284
:1000C00005D16FF30004013AEC72D2B2012601317E
:1000D0001029E9D10EB183F86822F0BDCC8C002044
:1000E00037B5014605460DF1060004F08FFDBDF859
:1000F00006204FF6FF739A422DD01F4C94F8DF2252
:100100007AB194F8DD32AB420BD1013AD2B284F825
:10011000DF2232B1920004F2DF2104F2DB202FF063
:10012000F3FDB4F8C821BDF806309A4215D14FF658
:10013000FF731248A4F8C83105F079FB1DF07AFB73
:1001400094F84C34DB0702D5284604F0D1FDBDF805
:10015000060027F0A7FC03B030BD284618F0DCFCF1
:1001600028461DF0B7F9284601F034FDBDF8060019
:10017000FFF782FEEBE700BFCC8C0020D9FA00002D
:10018000F0B587B008230025654C029101900093DB
:1001900040F2471240F69A5306460F464FF0FF30A2
:1001A00001210AF089FE2A46FE215E4884F8AF51FB
:1001B0000AF0A8FC2A46FE215B480AF0A3FC2A4666
:1001C000FE215A480AF09EFC94F8EC3284F81E5343
:1001D00065F3041384F8EC3226F046FA4FF6FF700C
:1001E00084F8DF521FF0D2FA94F84C34DA070CD5B9
:1001F0000DF117032A46294604F5E67005F044F888
:1002000018B99DF8170004F0D5FD002F5DD194F8C2
:100210000436B4F8C80167F3000384F804363A469C
:100220000DF11703394604F057FF18B99DF8170070
:10023000FFF756FF082200213D482FF07EFD0822DF
:100240003C493D482FF046FD10B313F0C9F8024673
:10025000F0B901460DF11703374805F015F890B9CC
:100260003649082201F500702FF034FD58B19DF891
:10027000170004F09FFD9DF8170094F8D9318342D0
:1002800001D0FFF72DFF082200212B482FF055FD4C
:1002900094F8D901FF2801D0FFF722FF304611F072
:1002A000CFFB37E0012B25D100EBC00300EB43006F
:1002B000D4F8F83218440222437862F3840343707E
:1002C00094F8D90104F076FD14E094F84C34DB077F
:1002D00013D594F8D901FF280FD094F8E030022B01
:1002E000E0D101F077FC28B140F6B65140F247105A
:1002F00006F09EF8FF2384F8D93194F84C34104866
:100300006FF3000384F84C34002300931A463146FF
:100310000AF074F9FF2384F8D93107B0F0BD00BFAB
:10032000CC8C002099A2030091A403006D980100D9
:10033000A48D0020A166040098900020988E0020D3
:100340006D33020070B51021064605F07EFC1A4D93
:100350000446102200212FF0F0FC08221749204605
:100360002FF0C7FC95F8E030012B02BF237B43F050
:100370000E03237395F8D5311BB1237B43F00C0397
:100380002373237B0E4963F07F032373022363737C
:1003900004F1080005F019FE0523A37395F8A437AE
:1003A000084843F0010385F8A43731460A22BDE826
:1003B00070400AF0B9B900BFCC8C0020A48D002099
:1003C0008C90002005A003004378C3F3C000C3F362
:1003D000001318440130C0007047427812F0100F2B
:1003E0000CBF08231023110748BF0833510742BF31
:1003F000991CC35C01EB4303920748BF0E33D8B28C
:1004000070470000F7B50E4614210446174605F064
:100410001FFC0546D6B10E4B9B1BC5F80F3067B1CC
:10042000204605F08FFA43882B800223AB73FFF739
:10043000D4FF0146204605F050FB002300931A46E6
:10044000214604480AF0DAF803B0F0BD3346E4E789
:1004500000FDFFFFFD03030010B505F073FA04462D
:10046000FFF7BBFF205C10BD2DE9F04F89B00446BB
:1004700005F068FA00230778049305460721204613
:1004800005F0E3FB0722014606A82FF032FCAB790A
:1004900043B107F00307012F04D8A8884FF6F77679
:1004A000B04205D9204605F0F1F916F0EFFEE7E17C
:1004B0000FF0B2FB6B88B34209D99F4BA988B3F800
:1004C000C821914203D193F8ED329A07EAD595F805
:1004D00001A0CAF3401ABAF1000F14D0964B93F85A
:1004E000E030012BDED804A9A88801F015FEB0BBCE
:1004F000049BA3B393F800A00AF00C0ABAF1080A0F
:1005000018BF4FF0010A204605F01CFA437803F0AB
:100510001203122B06461AD10721204605F095FB3F
:1005200080463046FFF759FFB8F80230B2883044B1
:100530009A42A0F10900737814D11B074CBF06F151
:10054000100106F1080108222FF0C4FBA8B92046CB
:1005500025F012FC00287DD14FF001080FE04FF08C
:10056000010AD0E719074CBF06F1100106F1080196
:1005700008222FF0AFFB0028E9D14FF000086B886C
:10058000DFF8B4914FF6F77293422AD94FF6FF7213
:10059000934210D04FF6FD72934202D199F8D521C3
:1005A0004AB999F8E020012A3FF67CAF05339BB2A7
:1005B000012B3FF677AF012F13D02946BDF81A0063
:1005C00026F03CF899F8D5315BB1284625F01EFF9E
:1005D00000287FF467AF284625F0E2FE00283FF4AC
:1005E00061AF6878C0F34002002A42D099F804361F
:1005F000DA077FF557AF204602F060FF00287FF44E
:1006000054AF204605F09EF912210546204605F01C
:1006100060FB0721204605F018FB072206A92FF0F2
:1006200068FBB8F1000F07D0204605F08BF9BDF844
:100630001A100546FFF7FCFCBAF1000F67D0012F36
:1006400060D000223D48AB8800922146012209F08B
:10065000D5FF2AE7BDF81A3001930423009340F236
:10066000471240F6EB0301214FF0FF300AF024FC63
:1006700018E72046039205F065F90378834603F0F6
:100680000306FFF7AAFE012E0146039A1FD103902D
:100690002046FFF7E1FE039999F88F215307C0D058
:1006A00099F84C2412F0010F99F8042611D0D207C2
:1006B00017D5012E7FF4F6AE06287FF4F3AEBBF813
:1006C0000220B9F8C8319A427FF4ECAEA9E710468F
:1006D000E2E7D3073FF5E6AE012E7FF4E3AE07284D
:1006E000F2E7002E7FF4DEAE204605F046F90378EF
:1006F00003F00302012A7FF4D5AE990691D48378E2
:10070000052BE1E72046FFF7A7FE042899D1AB7936
:10071000012F03F1FF33AB7140F0B5802046FFF7A6
:100720009BFE431EDBB20C2B824609D902462946AA
:100730002046FFF7B9FAB8E6CC8C00200D1901006D
:1007400001280AD06A884FF6F7739A4205D92846DD
:1007500025F05CFE00287FF4A5AE99F8E0306E88A5
:10076000012B00F2C5804FF6F7739E4240F298804D
:10077000AB79002B40F08A80002701266B785B075D
:1007800002D5A88803F004FA04A9BDF81A0001F004
:10079000C3FCC0B904989DF81C3003719DF91D304D
:1007A00043719DF91D1001F0E5FD049B5A7812F08C
:1007B0001C0F08D193F9050010F1640FB4BF00209D
:1007C00001200EF0E1FEB8F1000F3BD0204605F00D
:1007D000B9F807210546204605F037FA6B788046C0
:1007E000D80640F1948019074CBF05F1100005F1BF
:1007F000080005A901F0A4FC20BB059B5A7812F063
:100800001C0F1FD01B7803F00C03082B1AD1A888EB
:10081000B8F80230834215D0B8F800304FF6F072C5
:1008200023F00F0393420DD060B16B78DA0673D5D5
:100830001B074CBF05F1100005F1080001F088FE10
:1008400009F01CFA002F7DD0002E68D0002221462E
:100850003E4805F008F898B104230093019440F64F
:10086000B72340F2471201214FF0FF300AF024FB7A
:100870000123009300231A462146354809F0BEFEA5
:1008800009B0BDE8F08F4FF0000A66E72FB1AAF17A
:100890000902D2B2012A3FF66FAF01273E466DE74B
:1008A000B9F8C831B3423FF467AF2046FFF7D4FD33
:1008B00005283FF461AFAF79002FEFD004A9688815
:1008C00001F02AFC70B9049E56B1337803F00C0392
:1008D000082B0AD12046FFF7BFFDC21E56425641E3
:1008E00001274BE70127002648E70127064645E791
:1008F000B9F8C831B34207D04FF6F770864294BFBB
:100900000026012600273FE7002701263CE705A92E
:10091000A88801F001FC6FE701F00AFE90E70721CB
:10092000204605F092F9FF2383712CB940F6C121CE
:1009300040F2471005F07CFD002300931A46214643
:10094000044884E6002E3FF4ADAD91E72DFC000095
:1009500071150100750E010010B5214B93F8A82107
:1009600093F8A7019C1894F89211FE2929D1FF2130
:1009700084F892110132152492FBF4F104FB112248
:10098000B3F8AA1183F8A821013189B21428A3F879
:10099000AA1107D8013083F8A7011A44002382F86E
:1009A000923110BD981890F89201091AFF28A3F807
:1009B000AA111EBFB3F8AC1101F1FF31A3F8AC11BD
:1009C000EBE710B9012083F8A7011A44013182F83E
:1009D0009211B3F8AA210132A3F8AA2110BD00BFD9
:1009E000CC8C002013B51E4B93F8A72112B901221D
:1009F00083F8A721B3F8AC01421CA3F8AC2193F80B
:100A0000A8211524511C91FBF4F204FB121293F857
:100A1000A71183F8A821142913D8013183F8A7114D
:100A20001A4493F85038002113F0010382F8921110
:100A300005D100931A4619460A4809F0DFFD02B0B5
:100A400010BD991891F89241B3F8AA11FF2CA1EBAF
:100A50000401A3F8AA1118BFA3F8AC01E0E700BF96
:100A6000CC8C0020612902002DE9FF4119210446A8
:100A700005F0EBF805460789204604F063FF0646BB
:100A8000FFF76AFFD5F8123023F00803E12B14D1E9
:100A9000FFF7A8FFEB7D83B1013BDBB2EB7563B1E0
:100AA0008D4B93F84C34DB0707D500238B4800931C
:100AB0001A46214609F0A2FD47E02B7ED5F81280A8
:100AC000FA2B2BD00BD8F72B56D0F82B5CD0E12B80
:100AD0000BD1002300931A4621468148EAE7FC2BFC
:100AE00040D0C0F0A880FD2B4AD0F62B40F2C08049
:100AF000B8F1000F32D03A465FFA88F12046FFF78E
:100B0000FDF873785B0720D5734B7288B188754800
:100B1000A3F82022002204F0A6FE16E06E4D95F800
:100B2000D831072B11D10022FF216F4809F0EAFFCD
:100B300095F8D56166B96C2231466B4809F0F4FD31
:100B4000204685F8FD6101F031FD04B0BDE8F0817B
:100B500040F245120021644809F0E6FD204604F009
:100B600095FEF2E75C4B93F81F13FF2201F00101A1
:100B70002046FFF73DF8E8E7204609F049F8E4E7AA
:100B8000204626F02FFCE0E71921204605F05DF80D
:100B90000721D0F81270204605F057F80646204687
:100BA00004F0D0FE0546002F42D003A9408801F092
:100BB000B3FA48B9039B3BB11A7812F0080202BF9E
:100BC000197A62F306111972434BD3F8E420474BAC
:100BD0001B6803EB830313449A4219D12B7803F06B
:100BE0000303012B05D12846FFF7F7FB2B5C032BF2
:100BF0001ED0AB8833800223B3706B88A6F8033015
:100C0000FF23B371002300931A462146384851E769
:100C10001178C80704D5B2F803706888874201D0FC
:100C20000532D9E7CA06D9D5204602F013FF8CE772
:100C3000002C93D189E7092120462E8905F008F878
:100C40004FF6FF739E4280F800800BD0451C29466A
:100C5000304604F06BFA28B108224FF0FF312846E5
:100C60002FF06BF8002300931A462146214821E714
:100C7000B8F1000F0FD0B8F1DA0F0CD00222B11882
:100C800003A82FF036F8BDF80C004FF6F773984222
:100C900001D827F039FBD5F8121099B1F12911D0FC
:100CA000DA290FD03A46C9B20020FFF727F8D5F865
:100CB0001200C0B2FFF70EF9012201462046FFF7ED
:100CC000A1FB42E7044B93F8E020022A04BF002274
:100CD00083F85928EBE700BFCC8C002059FB0000BB
:100CE00021C0020051390100159D0300F8000020C9
:100CF000152B0100D91E02001C22002101482FF0F3
:100D00001CB800BF5E8E002010B50C46072104F011
:100D10009FFF6FF001014FF0FF3201704270817050
:100D2000C270847110BD0000F0B5002189B0044686
:100D3000FFF7EAFF0546204604F015FE10F8023CD6
:100D40002B71204604F00FFE10F9013C6B71214617
:100D500002A822F0CFFB02210646204604F0A1FEA5
:100D60003146204604F0B9FE0378C3F38303022B17
:100D7000064625D1204604F0EFFD07463046FFF732
:100D80002CFB87421CD09DF81D309A09022A17D1EE
:100D9000C3F38103022B13D1BDF810304FF6F77265
:100DA00093420DD86B80BDF808302B80012300934F
:100DB00000231A462146054809F020FC09B0F0BD81
:100DC000204604F063FD16F061FAF7E769040100BC
:100DD00008B5072104F039FF408808BD07B5144B5A
:100DE00093F8E0208AB1012A07D193F88E01C0431D
:100DF00040F3000003B05DF804FB002211460DF142
:100E0000030304F069F9014610B14FF0FF30F1E738
:100E100001AA9DF8030000F001FF0028F5D1019B15
:100E20005B7813F01C0F14BF4FF0FF300020E1E798
:100E3000CC8C002070B50E46162115461C4604F0D9
:100E400007FFC27C0A4B0680022161F34612C2747E
:100E5000827C058161F3461264F304028274B3F864
:100E6000CA3103829DF8103043750023037570BDAD
:100E7000CC8C00202DE9FF47064604F063FD0721D6
:100E80008046304604F0E1FE90F806902EB940F21C
:100E9000954140F2471005F0CBFAC94F97F8E03082
:100EA000012B9EBF98F8013023F0200388F8013011
:100EB000304604F047FD0023039305464088ADF813
:100EC0000A00AA88B7F8C8319A4209D04FF6F773DA
:100ED000984205D86B7813F0040F08BF4FF0F8095B
:100EE00097F8E030022B4CD197F8D831072B41D13D
:100EF00000242546A24698F8003003F00303012B96
:100F000002D13046FFF7A8FABAF1000F40F05E8137
:100F1000B8F802204FF6F7739A4200F21481304677
:100F200004F010FD42884FF6F7739A42044600F22F
:100F30003481BDF80A20B7F8C811CDF800904FF6FB
:100F4000FF73D31A18BF012343EA85033046FFF726
:100F500071FF62884FF6F7739A4205D81621304622
:100F600004F073FE04230375002300931A463146F0
:100F700094481CE197F8D9110DF10A0003F046FEE0
:100F8000B6E74FF6F773984204D94FF6FF73ADF802
:100F90000A30ADE76C78C4F380045CB32846FFF7F1
:100FA00013FA28444178002900F014810139417076
:100FB000023000EB410102220DF10A002EF099FEF1
:100FC000002211460DF10903BDF80A0004F084F86F
:100FD000014600288CD103AA9DF8090000F01EFEEE
:100FE000002885D1039B5D7885F00205C5F3400597
:100FF00004467FE70DF109032246214604F06CF810
:1010000070BB03AA00219DF8090000F007FE00282C
:10101000E8D0688826F0F4FD044600284ED0037816
:1010200013F0060301D0062B48D1A1780DF10A0078
:1010300003F0ECFD23786FF34203237003F03003D9
:10104000302B7FF455AFA888B7F8C831834215D14B
:10105000BDF80A306A88A988002002F001FC47E741
:101060006B781B07D5D50DF109032246214605F102
:10107000080004F009F90028C3D0CAE7002211468D
:101080000DF1090304F028F8014600287FF430AF81
:1010900003AA9DF8090000F0C1FD00287FF428AFE5
:1010A000039A137803F00C03082B7FF421AF5378D5
:1010B00003F01C03042B7FF41BAFC9E72B78C3F3A9
:1010C00041135BB3F4B1227802F00602022A25D163
:1010D0004946304626F0C4FD824678BB688826F033
:1010E000A9FD20B14288B7F8C8319A4229D000231F
:1010F0001A466988184626F063FF002425466FF0DB
:10110000030AF8E64946304626F0AAFD8246B0B901
:1011100023462246698826F053FFEFE70424019313
:10112000009440F26E4340F2471201214FF0FF302D
:1011300009F0C2FE00254FF0FF3ADCE60024254608
:10114000D9E65446DAE7404625F060F900287FF4F6
:10115000E6AE404625F024F900287FF4E0AE04A96D
:10116000002341F8043DBDF80A0000F0D5FF58B94E
:10117000039B4BB15B7803F00C03042B04D1BDF847
:101180000A202146FEF7BAFDB9F1F60F14D8012264
:10119000CF213046FFF736F90BE097F8E030012B0E
:1011A0003FF6C7AE0023084800931A46314609F0BF
:1011B00025FA04B0BDE8F087304604F067FBF8E795
:1011C000CC8C002081480300416403001AF1040F15
:1011D000C5D1EEE7AB78EA7843EA0223ADF80A30EE
:1011E000EEE600BF022104F074BD00002DE9F84FC7
:1011F0008A78CB78002A80460D460CBF0826102638
:1012000003B10836664B674F1A7897F884319342DA
:1012100009D8D7F8800100230E2404FB03F1934280
:1012200000EB010A03D34FF0000AD1460FE0415C06
:10123000C90704D5BAF802E0E9888E4501D0013328
:10124000EBE79AF801300133B14606EB43062C7800
:101250000CB10E36042495F801B0BBF1000F71D02B
:101260003146404604F0C0FB0222002104462EF025
:1012700064FD6A782378002A00F0838043F0090334
:101280002370BAF1000F14D09AF8013004F8093035
:1012900004EB09009AF8013043709AF801200AF132
:1012A0000401520002302EF024FD637843F0040361
:1012B0006370EB7894F90110002BAB7814BF08220F
:1012C0000022002B14BF102300230A431343DBB278
:1012D000637097F8E020022A05D197F8AF2112B188
:1012E00043F0200363702B785BB1264497F872318A
:1012F00006F8013C637843F0020363704046FFF751
:1013000071FFAB88A380EB8863800123A37197F8FA
:10131000D630E37197F8D630013387F8D630AA7803
:10132000EB788AB30822ABB3A918A0182EF0E1FC21
:10133000082205F1100104F110002EF0DAFC20461D
:10134000BDE8F88F404604F007FB33190B3318440F
:101350007F2809D9AB7813B185F802B0083EEB7845
:1013600013B10023EB70083E404604F0F5FA0B344D
:10137000344404447F2C10D83146404604F075FCB8
:1013800072E743F008037BE7002BD8D00822A918A6
:10139000A018D2E705F11001FAE70024CFE700BF5B
:1013A000F0000020CC8C002070B586B014469DF86B
:1013B00028308DF8003000238DF802308DF803308E
:1013C000204B9DF82C2093F88E618DF80120054666
:1013D000F6060846ADF804009DF83010ADF806405A
:1013E00000D549B393F89011C90700D522B3B3F8DB
:1013F000C831834208D10822134904A82EF079FC91
:1014000001238DF8023004E004A903F08FFE0028C8
:10141000F6D04FF6F7739C420ED802A9204603F08F
:1014200085FE48B9082209490DEB02002EF052FC56
:1014300010B101238DF8033069462846FFF7D6FE28
:1014400006B070BDCC8C0020988E002099660400F8
:10145000F0B50E218BB0064604F0F7FB04462EB91A
:1014600040F2E22140F2471004F0E2FF2CB940F2D2
:10147000E32140F2471004F0DBFF3B4D95F84C248C
:1014800012F0010204D1C2213046FEF7BBFF4EE04C
:10149000A37953B195F8043613F0010305D095F8FC
:1014A0008F3113F0070318BF0123227A012ADBB220
:1014B00022883ED1B5F8C8118DF81030ADF814105F
:1014C000002304A930468DF811308DF812308DF8C4
:1014D0001330ADF81620FFF789FE0746002836D0F6
:1014E000237A012B01BF63898380237BC371A37897
:1014F0001BB995F83A315B00DBB2BB7163795BB124
:1015000022884FF6F7739A4206D87B785B075EBF56
:101510003B7843F040033B70E1793046FFF7F4FB42
:10152000002300931A463146104809F067F80BB0C3
:10153000F0BDE7780093002002900190781E4342AE
:101540004341B5F8C8113046FFF72EFFC5E70090BC
:1015500040F24712012140F23B334FF0FF3009F0D7
:10156000ABFC3A46D3218FE7CC8C0020750E0100EE
:101570002DE9F04786B0044604F0E4F90578074603
:10158000FEF72BFF05F003058046002D59D1C84E0C
:1015900096F8E83253B986F8E8421A460093214695
:1015A000C44809F02BF806B0BDE8F087D6F8E4226D
:1015B000C14F92683968B2EB510F22D202930823CF
:1015C000009340F2471240F6283301214FF0FF30DC
:1015D000019409F071FCD6F8E4325A6813441C7384
:1015E000D6F8E422936801339360D6F8E4023B68AE
:1015F00042685B080132B2FBF3F103FB1123436045
:10160000D1E704230093019440F62E3340F24712B1
:1016100001214FF0FF3009F04FFC15F037FE002C90
:10162000C1D004230093019540F6D33340F2471212
:1016300001214FF0FF3009F03FFC204604F026F96D
:10164000B1E7012D40F031812046FEF705FF042867
:101650000546974E40F08D8008F10101204604F0C8
:101660008CF996F84C3490F800800022D8078DF859
:101670001320059217D511460DF11303B88803F016
:101680002BFD014678B905AA9DF8130000F0C6FAB3
:101690004FEA9813002800F01981D90703D49DF868
:1016A000130003F025FB204604F0F0F85FE0B88853
:1016B000FFF794FB0028F6D17A884FF6F7739A4229
:1016C000F1D896F88F7117F007074FEA581A44D1EE
:1016D0004FF00109B6F8C811CDF808908DE88002E6
:1016E00000234FF6FD722046FFF75EFE80F806905D
:1016F00017B12046FFF776FD012204215FFA8AFA2E
:101700002046FEF7DFFB1AF0010F14BF2023002351
:101710005FEAD81714BF6FF07F02002213430370F3
:1017200096F81F33FC216AF30003204686F81F3326
:10173000FFF7EAFA002300931A4621465F4808F0B3
:101740005DFFA7B93A46FE215D4809F0DBF93A464C
:10175000FE215C4809F0D6F909E096F80436DA076C
:10176000B6D4FF220AF001012046FEF741FA002418
:1017700053E7072808D196F8E030002B3FF44DAF2F
:10178000204628F005FBF2E70C280FD108F10101F3
:10179000204604F0F2F896F8E030022B02467FF47F
:1017A0003CAF3946204608F061FBE0E70A2807D144
:1017B000D6F81832002B3FF430AF20469847D6E7D2
:1017C00096F8E030012B67D801280AD108F1010111
:1017D000204604F0D2F839460246204626F0AEFAFA
:1017E000C5E702280AD108F10101204604F0C5F836
:1017F00039460246204626F08DFCB8E7052805D17B
:1018000042463946204602F033F8B0E7082805D1B1
:1018100042463946204628F071FDA8E7062803D144
:10182000204625F0ADFDA2E70B280AD108F1010101
:10183000204604F0A2F839460246204608F060FB34
:1018400095E7092802D1D6F81432B3E7032826D148
:1018500008F10101204604F090F80678B0F8017014
:10186000022EB9B205D90D2E06D1204624F082F9F8
:101870007DE7084626F080FD0421204604F0E5F9C6
:1018800001230670A0F80170009300231A46214638
:101890000D4808F0B3FE6AE703283FF4BEAE2A46BF
:1018A00039462046FEF700FA61E70025B7E600BF9B
:1018B000CC8C002079010300F4000020750E01009B
:1018C00099A2030091A40300CD180200DB073FF5A5
:1018D000EEAEC8F340139DF8130086F81D3386F86A
:1018E0001C0303F0ABF9084803F0A1FF059B5B78EC
:1018F00013F01C0F7FF4D7AE5FEAD8133FF4D3AEDA
:1019000096F8E030012BDBE689FC00002DE9F0437E
:10191000194C94F88F7185B08846012507F00707A8
:10192000B4F8C81102950195009700234246064677
:10193000FFF73AFD814617B13046FFF753FC89F8AF
:101940000650012204213046FEF7BCFA60230370E2
:10195000FB23B4F8C8110093424630460123FFF739
:1019600069FA002300931A463146044808F046FEFF
:1019700005B0BDE8F08300BFCC8C00208148030097
:1019800010B50F4C94F8B8316FF3040384F8B831F4
:1019900004F5E07004F0F1FCD4F8C03103F07843B2
:1019A00043F0FF6343F4FF23C4F8C03194F8B83127
:1019B00043F0200384F8B8311023A4F8BA3110BDE5
:1019C000CC8C0020082070472DE9F041194B0646C9
:1019D0001868194B17468846D3F8F8224FF0130EB3
:1019E0000123834203D36FF01500BDE8F0810EFBA5
:1019F00003F15518545C14F0010418D12146132248
:101A000028462EF09AF92B78A5F8068043F00303B8
:101A10002B700622094905F108002EF06AF9EB7BCC
:101A200066F30403EB733D602046BDE8F0810133AB
:101A3000D7E700BFEC000020CC8C002099660400A2
:101A400010B5084B084C1A68D4F8FC024FF0FF316F
:101A50002EF073F9052384F809333C2384F80A3304
:101A600010BD00BFD0000020CC8C0020F0B50023BA
:101A70001360114B1F68114B4FF0130ED3F8F8622F
:101A80000123BB4203D3BDE8F040FFF79DBF0EFB2F
:101A900003F57419755D05F00305032D07D1E5887D
:101AA0008D4204D1E57B05F01F05854201D001334D
:101AB000E7E714600020F0BDEC000020CC8C002093
:101AC0002DE9F04F0F4685B0804602A938461646EC
:101AD00002F0A6FFDFF878A0DFF8789001256FF01C
:101AE0001B044FF0130BDAF800309D4213D314F1AE
:101AF0001C0F0CD132464FF6FF714046FFF764FFD2
:101B0000044620B931683846083102F089FF204682
:101B100005B0BDE8F08F0BFB05F2D9F8F832981844
:101B20009B5C03F00303032B10D1C37B03F01F0363
:101B300043450BD102A90830019203F043FB28B1C1
:101B4000D9F8F832019A1344336000240135CAE70A
:101B5000EC000020CC8C002010B5124AD2F8FC32E8
:101B6000FF241C5401EBC10301EB4301D2F8F8320E
:101B70005A5C6FF300025A5403F01CF905F012FB93
:101B80000B2006F003FD0C2006F000FD0F2006F0F0
:101B9000FDFC132006F0FAFC05F012FBBDE8104036
:101BA00008F06CB8CC8C002038B5094BD3F8FC3267
:101BB0005D5CFF2D0C4607D008F08AFA29462046C6
:101BC000BDE83840FFF7C8BFBDE8384003F05EBE4F
:101BD000CC8C002010B50F4CD4F8FC321B5CFF2BD2
:101BE000014614D003EBC30203EB4202D4F8F842DF
:101BF000A25C02F00C02082A05D10022064803F07C
:101C000032FE002010BD1946FFF7A6FFF9E76FF07E
:101C10001B0010BDCC8C0020A91B01002DE9F8434E
:101C200017462C4AD2F8FC321B5CFF2B06461546A1
:101C300040D1002949D0284BD5F8F8121A684FF046
:101C4000130E00235FFA83F94A4503D86FF015009D
:101C5000BDE8F8830EFB09F8013311F8080010F015
:101C60000104EFD1304602F0E9FFD5F8FC3203F869
:101C70000690D5F8F89209EB08051322214628466C
:101C80002EF05BF819F808206B7842F00D0209F885
:101C9000082043F00203032262F3840364F3000389
:101CA0006B702B7AEE7143F070032B727F236B7194
:101CB0003D6007E0D2F8F82203EBC30103EB4103D8
:101CC00013443B600020BDE8F8836FF01B00BDE8C3
:101CD000F88300BFCC8C0020EC0000200A4B0B4A9C
:101CE000D3F8F8321268132101FB0232002093422C
:101CF00000D17047197801F00D01092904BF0130A6
:101D0000C0B21333F3E700BFCC8C0020EC000020FE
:101D10000A4B0B4AD3F8F8321268132101FB023246
:101D20000020934200D17047197811F0010F03D0C1
:101D300009075CBF0130C0B21333F2E7CC8C00203E
:101D4000EC0000202DE9F04F85B00DF110091B4B80
:101D50000024174629F8024DD3F8F862184A834642
:101D60008A462546A0461368984501D2544503D3B8
:101D7000204605B0BDE8F08F337803F00D03092B42
:101D800018D10135EDB25D4514D3F1790192484681
:101D900002F03CFF3B68019A591C3960BDF80E10F7
:101DA000197039684B1C3B60BDF80E3001341B0ABA
:101DB0000B70E4B208F101081336D4E7CC8C002094
:101DC000EC00002037B504460D460DF107012078E0
:101DD00002F090FE014618B16FF01B0003B030BD59
:101DE0002A469DF80700FFF719FF0028F6D0237850
:101DF00001332370E9E70000F0B5037803F0030333
:101E0000032B87B004460E4605D040F20A214FF45A
:101E1000A47004F00DFB564DDEB1564BD5F8F81208
:101E20001B6813225A430026B24212D08B5D13F076
:101E3000010701EB060006F1130E59D121461322CA
:101E40002DF057FF237867F300032370D5F8F8428D
:101E50003444E2884FF6FF739A4204F1080650D0EA
:101E60000622454930462DF035FF0246002841D074
:101E7000314604A802F016FE0DF10F030022E1889E
:101E800004A803F04FFA06469DF80F00002E44D137
:101E9000D5F8FC321B5CFF2B3FD102F0CFFE0C22A9
:101EA0003146A01D2DF049FFD5F8F822334BD5F867
:101EB000FC029DF80F10A21A534343542378627812
:101EC00003F00C01083918BF012161F3410203211D
:101ED00061F384026270227A42F0700222729DF8ED
:101EE0000F20E27166F341032370304607B0F0BD66
:101EF000764699E70DF10F030121E08803F0ECF835
:101F0000C1E7314604A802F0CDFD0DF10F03002218
:101F1000012104A803F0B8F9B5E7D5F8FC32D5F8EB
:101F2000F8121B5C03EBC30203EB4203CA18944292
:101F300010D0CA5C02F00C000C2801BF2078C0F35E
:101F4000810060F38302CA54237803F0FD036FF32A
:101F50000003C9E70423019000934FF4A4724FF4E7
:101F60001C7301214FF0FF3008F0A6FFBDE700BF52
:101F7000CC8C0020EC000020996604001BCA6B2862
:101F80002DE9F743384C394F94F84C3413F0010FD6
:101F9000804614D1012213253B689A4227D205FBC3
:101FA00002F1D4F8F802435C03F00306032E02BFEB
:101FB00003F0FD036FF3000343540132ECE70DF12E
:101FC000070104F1D80002F073FC4FF6FF73984547
:101FD00010D100264FF0000E01254FF013093B6889
:101FE0009D4219D3BEF1000F01D006F073FE03B07D
:101FF000BDE8F08300220DF106031146404603F0D0
:102000006BF80028E5D19DF80630D4F8FC22D65CA8
:10201000FF3E18BF0126DDE709FB05F3D4F8F822DF
:10202000D15C01F00301032902EB030013D1C17B52
:102030009DF807C001F01F0161450ED194F8E01032
:10204000012903D9C188414507D136B90021FFF7DD
:10205000D3FE4FF0010E0135C1E7D15C01F0FD0167
:102060006FF30001D154F6E7CC8C0020EC00002087
:10207000F8B5184F184C002513263A68EBB29A426F
:102080001AD872430021D4F8F8022DF056FE134BF3
:10209000D4F8FC021A6800212DF04FFE0023C4F88A
:1020A000003384F8083307F047FE0D4803F0BFFB08
:1020B000BDE8F840FFF7C4BC7343D4F8F822D11848
:1020C000D35C03F00303012B02D1C87902F072FE46
:1020D0000135D2E7EC000020CC8C0020D00000209D
:1020E00045A101000A4B1B6898420DD200EBC003CA
:1020F00000EB4300074BD3F8F8321A181B5CDB07E0
:1021000002D50A60002070476FF01B00704700BFC7
:10211000EC000020CC8C002013B500220C460DF101
:102120000703114602F0D8FF014628B922469DF860
:102130000700FFF773FD08B16FF01B0002B010BD80
:1021400013B500220C460DF10703114603F09CF86D
:10215000014628B922469DF80700FFF75FFD08B148
:102160006FF01B0002B010BD30B50B4B1C680B4B61
:10217000D3F8F8321325A0420BD205FB00F29918D0
:102180009A5CD20703D54A78920700D530BD01305A
:10219000F1E74FF0FF3030BDEC000020CC8C002088
:1021A000F0B5134B1D68134BD3F8F84213264FF6C6
:1021B000FF77A94218D206FB01F3E218E35C13F0A3
:1021C000010F0FD0527802F00C0EBEF1040F09D1AE
:1021D00003F00C03082B05D1B84203D1930701D4B7
:1021E0000846F0BD0131E4E74FF0FF31F8E700BFEA
:1021F000EC000020CC8C0020F0B5114B1E68114B78
:102200001327D3F8F8420023B34202D16FF01B002A
:10221000F0BD07FB03F2A518A15CCA070ED56A78CA
:1022200012F0200F0AD001F00C01082906D102F0AB
:102230001C02042A02D105600020F0BD0133E3E74F
:10224000EC000020CC8C002030B50A4B19680A4BFA
:102250000020D3F8F842132503468B4200D130BD4D
:1022600005FB03F20133A25CC2F300021044C0B2CA
:10227000F3E700BFEC000020CC8C00202DE9F041FA
:10228000134EDFF850E0074600226FF01B004FF0BE
:10229000130C33689A4201D3BDE8F0810CFB02F1C4
:1022A000DEF8F842635C03F00308B8F1030F04EBB7
:1022B00001050AD1ED7B05F01F05BD4201BF03F00A
:1022C000FD036FF30003635400200132E1E700BF18
:1022D000EC000020CC8C00202DE9F04FDFF890803E
:1022E000224F87B00025C246D8F80030013B9D42FE
:1022F00038D200264FF013092BE0D7F8F83209FB4B
:1023000004F419191A5D02F00302032A20D104F122
:10231000130B03EB0B0013F80B3003F00303032B39
:1023200016D10A7903799A4212D2132201A82DF00C
:10233000E0FCD7F8F802132200EB0B0120442DF04B
:10234000D8FCD7F8F802132201A958442DF0D1FC8B
:102350000136DAF80030013BF4B25B1BA342CCD863
:102360000135C1E7002007B0BDE8F08FCC8C00201C
:10237000EC00002090F905207F2A1FBF5523891A01
:102380004B434FF480711BBF93FBF1F39B184171DA
:102390004371704707B501A9FFF7BEFE30B9019B35
:1023A0005878C0F3820003B05DF804FBFF20FAE721
:1023B00007B501A9FFF7C4FE30B9019B5878C0F3F7
:1023C000820003B05DF804FBFF20FAE707B501A91E
:1023D000FFF7A2FE30B9019B1878C0F3810003B06B
:1023E0005DF804FBFF20FAE707B501A9FFF7A8FE97
:1023F00030B9019B1878C0F3810003B05DF804FB8D
:10240000FF20FAE707B501A9FFF786FE30B9019B67
:102410005878C0F3400003B05DF804FBFF20FAE7F2
:1024200007B501A9FFF78CFE30B9019B5878C0F3BE
:10243000400003B05DF804FBFF20FAE737B514460F
:1024400000220D460DF103031146019202F044FEF5
:10245000D8B901AA29469DF80300FFF7DFFBA0B910
:10246000019B5A78C2F3820222701A78C2F3810269
:1024700062705A78C2F34002A2701A78C2F3031253
:10248000E2705B78C3F30003237103B030BDF7B58E
:1024900000220C460DF103031146019202F01CFECE
:1024A0000546002841D1014601AA9DF80300FFF727
:1024B000B5FB0546002838D1019A20785378C3F33C
:1024C0008201814213D116786178C6F381078F4269
:1024D0000DD1A778C3F34001B94208D1E178B1EB3F
:1024E000161F04D1217903F001038B421DD05378CC
:1024F00060F384035370019B61781A7861F383025F
:102500001A70019BA1785A7861F341025A70019BBD
:10251000E1781A7861F307121A70019B21795A78D1
:1025200061F300025A7006F0D5FB284603B0F0BDF7
:1025300013B501A9FFF7F0FD044630B9019BD87926
:10254000FFF748FB044606F0C5FB204602B010BD6D
:1025500013B501A9FFF7F4FD044600BB019BD87930
:10256000FFF738FB019A537803F01C03042B044651
:1025700015D113780B4803F00C03042B0A4B0BBF47
:1025800093F83C2193F83D2102F1FF3202F1FF3232
:102590000CBF83F83C2183F83D2103F048F9204625
:1025A00002B010BDC1850300CC8C002073B5264C51
:1025B00094F8EC5215F02005064606D0012384F865
:1025C000FE3100283BD102B070BD28B91F4802B0CF
:1025D000BDE8704003F02BB90F2103F036FB94F8EF
:1025E000EC3284F8FE5143F0200384F8EC3294F886
:1025F000FD31013384F8FD3102230370D4F8F83142
:10260000DB88A0F80130B4F8CA31A0F809302022E4
:10261000C27205734573857394F8FD31012B06D1A1
:102620000B48314602B0BDE8704008F07DB8009517
:102630002B462A463146064807F0E0FFC3E702B0C2
:10264000BDE8704003F022B9CC8C0020AD2501001C
:102650001D2E030038B51C4D1C4B002229688A42F0
:1026600028D393F80111002262F3000183F80111CD
:1026700093F80B1183F8362162F3000183F80B11F4
:1026800093F8151183F8372162F3000183F81511CF
:1026900093F81F1162F3000183F81F1193F82911B9
:1026A00062F3000183F8291125F016FABDE83840DD
:1026B00023F0DABF02EB8201D3F8E400445C6FF34D
:1026C000000444540132C9E7F8000020CC8C0020FB
:1026D0002DE9F0418AB000230A210693064603F053
:1026E000B4FA674C01460A2207A82DF002FB94F8C1
:1026F0004C3413F001030CD1009340F249124A23E9
:1027000001214FF0FF3008F0D7FBC2254FF0FF3317
:1027100007E008225B4907A82DF0DCFA30BB002552
:102720002B4694F8E020002A3ED163B9069A002A8D
:102730003CD1009340F249128F2301214FF0FF302A
:1027400008F0BAFBC225304603F08AF90921304669
:1027500003F07EFA082207A900F8015B2DF0C9FA00
:10276000002300931A46314647486BE0082204F5DF
:10277000E67107A82DF0AEFA0028D0D094F8E0302A
:10278000012B0FD806A907A8FFF7DAFC50B9069A63
:10279000137803F00C03082B04D1537803F01C03C7
:1027A000142BBCD1C825B1E7002BCCD194F88F7184
:1027B000069B07F00707002B49D194F81F239DF8CB
:1027C0002510009761F3000284F81F23B4F8C811A4
:1027D0000122029201924FF6FD723046FEF7E4FDAF
:1027E000804617B13046FEF7FDFC01252A4688F8E1
:1027F000065004213046FDF765FB002303709DF869
:102800002530002B14BF2023002303709DF82420C3
:1028100062B3069A2AB1157805F00C05083D18BF79
:10282000012543EAC5150570069B0BB345F040052D
:102830000570FB213046FEF767FA0023134800932A
:102840001A46314607F0DAFE0AB0BDE8F081D979C0
:102850000DF1160002F0DAF9012302930193BDF89D
:102860001620B4F8C81100970023B6E71546D8E73C
:10287000002FDED094F80436DB07DAD4CD2562E7EA
:10288000CC8C0020A1660400D91E0200750E010048
:102890002DE9F3410221064603F0D7F905781B4CD8
:1028A000CDB194F8E030012B01D8FFF7D3FE94F8B6
:1028B000D8310A2B01D0FFF7DBFB07F0DFF900234B
:1028C00000931A463146124884F8D83107F096FE34
:1028D00002B0BDE8F08147780121304603F0B5F938
:1028E0000122804629462DF028FA012388F800307D
:1028F0002A4600952B463146064807F07FFE1FB159
:102900000A2384F8D831E3E70923FAE7CC8C0020C6
:10291000151902003D25030073B5144C94F8D83105
:102920000A2B054608D094F8D5610020FDF70EFA71
:1029300084F8D561FFF79CFB94F8E030012B01D8B7
:10294000FFF788FE4FF49072002109482DF0F5F949
:10295000002003F08BFD07F091F9002300931A4645
:102960002946044807F04AFE02B070BDCC8C002016
:10297000A48E0020151902002DE9F043DFF89080A5
:1029800098F8EC4214F0200485B0074603D198F87B
:102990004C34DB070DD4C221384603F0DFF90023A5
:1029A000194800931A46394607F028FE05B0BDE8DD
:1029B000F0830F2103F049F904AE0546052138469E
:1029C00026F8024D03F041F998F8EC32D0F8019066
:1029D00098F8D91143F02003304688F8EC3202F021
:1029E00015F9BDF80E30A5F8013002232B70B8F8A8
:1029F000CA31A5F80930C5F80B9023460094224649
:102A000039460248D0E700BF657402001D2E03005E
:102A1000CC8C002013B5044603F098F9104B93F8C2
:102A2000EC226FF3451283F8EC2293F8D821072AA1
:102A30000DD193F8FE31204623B102B0BDE810401D
:102A4000FFF7B4BD02B0BDE8104002F01FBF002385
:102A500000931A462146034807F0D0FD02B010BD8E
:102A6000CC8C00206574020037B503F081F9274D46
:102A7000044695F83833A8B313F0010315D140F29A
:102A8000491201214FF0FF30009340F2E72308F094
:102A900013FA03F099F995F8383343F0010385F8F8
:102AA000383308F073FAC5F8300308F06FFAD5F838
:102AB0003043174B001B984210D808F067FAD5F83E
:102AC0003043001B41F67864A04294BF00200120EF
:102AD000D0B103B0BDE8304003F076B908F056FA43
:102AE000201AEFE7DB070FD5009040F22F3340F2BA
:102AF000491201214FF0FF3008F0DEF995F8383324
:102B000064F3000385F8383303B030BDCC8C00206B
:102B1000FEFFFF7FF0B5072185B0274F054603F084
:102B200094F897F88F610288B7F8C811002304461B
:102B300006F0070601200293019000962846FEF752
:102B400033FC97F83A315B008371037843F040031C
:102B5000037016B12846FEF745FBB4F803204FF684
:102B6000F7739A4225D8A378132B0CBF04220322B3
:102B700003212846FDF7A6F9A3780370B4F80330C3
:102B80004FF6F77299B2914206D8A0F80130A378B7
:102B9000132B04BF6379C370A1792846FEF7B4F8FC
:102BA000002300931A462946044807F027FD05B084
:102BB000F0BD0122DCE700BFCC8C0020750E0100C7
:102BC00007B5074B0D2283F8D82100230146009357
:102BD0001A46044807F012FD03B05DF804FB00BF7D
:102BE000CC8C0020912C01002DE9F0470D4603F11B
:102BF0000B011E4691460746DDF8208002F0F4FEE8
:102C000004460570002545708670324649460B30F3
